:020000040800F2
:1000000000A00020090601085DC500084DF70008A2
:100010005BC5000859C5000857C50008000000006E
:1000200000000000000000000000000055C50008AE
:1000300053C500080000000051C500080BC00008AF
:1000400071060108710601087106010871060108B0
:1000500071060108710601087106010871060108A0
:100060007106010871060108710601087106010890
:1000700071060108052E00083F29000871060108D5
:100080007106010871060108710601087106010870
:10009000BDC5000871060108710601087106010856
:1000A00011B5000851B5000801B5000879B5000880
:1000B00041B5000831B5000821B5000871060108F6
:1000C0007106010871060108710601087106010830
:1000D000710601083DB7000831B700087106010834
:1000E00019C000087106010831F600087106010800
:1000F0007106010871060108710601087106010800
:10010000000000000000000000000000710601086F
:1001100071060108710601087106010871060108DF
:1001200071060108710601087106010871060108CF
:1001300071060108710601080000000000000000BF
:10014000710601087106010871060108000000002F
:10015000000000000000000000000000000000009F
:10016000000000000000000071060108710601088F
:1001700071060108000000000000000000000000FF
:080180000000000071060108F7
:100188002DE9F04F2DED028B6B4D6C4B2B60A3B01E
:1001980000236B600DF0AEFE18B90DF0CFFE07F02E
:1001A800EFFE07F0ABFF664B664C1A7842F001028F
:1001B8001A70654A4FF47001C2F88810002209923B
:1001C8000A92226842F4803222600493236803F47E
:1001D80000330A93099B013309930A9B1BB9099BB6
:1001E800B3F5A04FF2D1236813F4003318BF0123ED
:1001F8000A930A9B012B69D0DFF84C81534BC8F84E
:100208000C30636AAB60636A514FDFF870A1DFF8A6
:10021800709143F080736362636943F4FC0322AE18
:10022800636103238DF83A3041F6FF7326F8503D99
:100238004FF09040314602F0F9FD4FF6FF73384613
:100248003146ADF8383002F0F1FD4248314602F04F
:10025800EDFD4148314602F0E9FD4048314602F0E3
:10026800E5FD31463E4802F0E1FD304606F0F4FF78
:100278000E9B3C4AB3FBF2F33B4A3C4913603C4BB0
:1002880000221A603B4B5960F02188F823109A60CD
:1002980007221A60DFF8EC80DAF80830C8F8003076
:1002A80099E80300636986E8030043F480236361E7
:1002B8004FF48053BB610E980FA902F0B7FDD8F830
:1002C800003013F0080F574629D163E02A4B122259
:1002D8001A606368636063686360636843F480639B
:1002E8006360636823F47C136360636843F4881372
:1002F8006360236843F0807323602268114B970181
:10030800FBD55A6822F003025A605A6842F002028A
:100318005A60636803F00C03082BFAD16CE79AF86B
:100328009231012B36D8044A9AF89331926812F028
:10033800805A00F0E7872DE0600800203178000837
:10034800E82600200010024000ED00E00005FA0554
:100358000004004800080048000C0048001000484D
:100368000014004840420F008C2000203F19010073
:100378009020002010E000E000200240B41100208E
:100388003042010870260020C24B002283F89321D6
:1003980008F056F864200BF02AFE4FF48C72BE4821
:1003A800002112F0DAF8E369BC4A43F00703E3617D
:1003B800A36943F4E123A361636943F4C023636140
:1003C80002F1E00C937B506892F80FE003F007010C
:1003D800DB0800EB83038900186A4FF00F0A0EFA56
:1003E80001FE0AFA01F120EA01011962196A1032C4
:1003F8004EEA010162451962E4D10022A8490023AE
:10040800535401320E2AF9D1DFF8C4A20AF11A02B4
:10041800FF2199540133072BF6D1A24AA24B13604E
:10042800DFF8B0B2A14A03930321117058460021A6
:10043800242212F092F814228BF800209C49039B86
:10044800D8F8008001228BF8182097F805B081F8B9
:1004580000B0A3F5F071CAF824109649A3F590737B
:100468000B60954B03EBCB0318F0200F5B78CAF8B1
:10047800283018BFCAF828200023904A40F2DC51DF
:1004880022F813100133082BF7D1304600211C2223
:1004980012F063F8BBF10E0F04D00BF0EF0BBBF1B9
:1004A800080F02D101238DF84830022006F064F8C5
:1004B80018B14088003018BF0120C8F340038DF8F8
:1004C8003E30C8F380138DF84030C8F340338DF8C0
:1004D8003830C8F3C03300F001008DF83B3018F411
:1004E80000638DF83D0004D097F886315E1E734294
:1004F80073418DF83C30C8F300438DF84130AB6A46
:10050800B7F84801ADF84C00003318BF01238DF847
:100518004230C8F300538DF84330B7F84A31ADF88C
:10052800463018F4805FB7F8563118BF5948ADF80F
:100538004430C8F380438DF83F30B7F854311CBFBE
:10054800B0F85001ADF84C00B3F5FA7FADF84A3079
:1005580084BF0023ADF84C30594897F8D63185F858
:100568002C30002385F82D3043709DF8483008F072
:100578000101002BC8F3C0028DF839108DF83A201C
:100588000CBF0023022301B902B1013309EB83092F
:10059800D9F80830A3F1020B1A3305934FF000097C
:1005A8003BF8023F4FF6FF72934200F033811A0A7C
:1005B800022AD0B202D19DF8382003E0012A04D1E2
:1005C8009DF83920002A00F021819DF84220DBB2F5
:1005D80062B19DF848204AB99DF840200AB11A1F17
:1005E80001E0A3F10802012A98BF04202B4F9DF8CF
:1005F80043104FEA031807EB08063A4631B19DF855
:10060800481019B9043B032B40F2E980012863D153
:100618004244FF234FF0000A517B85F8743085F877
:10062800753050688DF82E1002F108031289ADF864
:100638002C200BA9022285F878A0C5F884600393C2
:100648008DF82F2085F830A0C5F834A0C5F838A05B
:10065800C5F83CA0C5F870A085F876A085F877A005
:1006680002F0E4FB039B57F808009978524602F021
:100678000FFB30460EF04EFC124B1349C5F888307C
:10068800124BC5F88C30C5F890A030460A1D0AF008
:10069800F1FFBBE0B4110020C42000205C60010819
:1006A8006C080020A0240020A8130020911100202D
:1006B800EC0300205822002080630108021100206A
:1006C8008D08002081260008E8080020612700081E
:1006D80060080020A4240020022847D15FFA89F38B
:1006E8004FF01C0A0AFB03F3EF180393974B87F8A4
:1006F8007990012187F8781003EB08014FF0000A80
:10070800D1F804C091F80DE08DF82F0001F108022E
:100718000989ADF82C1060460BA987F87AA087F8EC
:1007280082A0C7F884608DF82EE00793069202F045
:100738007DFB079B069A53F808009178524602F011
:10074800A7FA30460EF0E6FB8149C7F888108149C0
:10075800C7F88C10039B8049C7F890A0194430460D
:100768000A1D0AF087FF09F101094FE0032834D177
:100778009DF83F30794FDFF81C823BB197F82EA0E7
:10078800304608214FF6FF7200231AE0BDF84A20D0
:1007980097F82EA0BDF84C30B2F5FA7F0BD9704906
:1007A800B1FBF2F23046082192B202F068FB6D4BC1
:1007B80048F82A000AE06C49B1FBF2F23046012100
:1007C80092B202F05CFB694B48F82A00C36097F8C4
:1007D8002E30013387F82E3018E0042816D195F80A
:1007E8002D70BDF84420604B93FBF2F23046BDF803
:1007F8004630012192B202F042FB95F82D3005EB0C
:1008080087070133C7F8580185F82D30059B9B45AC
:100818007FF4C6AE95F82D3085F87831544B554F96
:1008280093F800E0AEF117030026022B3E7018D8AB
:100838006B6A3344D3ED007AF5EE407AF1EE10FAA4
:1008480002D1AB6A53BB24E04B4A06EB020C0FCB38
:100858008CE80F003B7810360133C02E3B70E7D18F
:10086800EFE7464B13F83EC087F800C003EBCE0312
:10087800D3F80480B8F1000FE3D06645E1DA3E4AC8
:10088800330103EB020943440FCB013689E80F001B
:10089800F3E73B4E3368DD0424D41DE0394B3A4A74
:1008A80013F83E00107003EBCE035D68002DF0D006
:1008B80000238342EDDAC3EBC3016A18DFF8D8C01E
:1008C800D2F8008041F80C8001EB0C069188B180C9
:1008D8009279B2710133ECE70EF0EF03082B2B4F3E
:1008E8001FD121E03A78012AF6D9294B03EB0212ED
:1008F800103210339342EFD053ED047AB6EE007AFB
:1009080067EE877A43ED047A53ED057A67EE877AC6
:1009180043ED057A53ED037A67EE877A43ED037A60
:10092800E7E7BEF10E0F09D13B7843F010033B70A7
:10093800BEF1180F32D10BF025FD2FE03B7823F0E4
:1009480010033B70BEF1190FF4E700BF5C600108AB
:10095800952D000859260008E808002060080020A6
:1009680000127A008127000840420F007127000812
:10097800EC0300208A20002028030020806301085F
:1009880070260020C0460108E4210020E01800205D
:100998003003002094200020E52100200BF0D6FC35
:1009A8003368DFF84883C54D58035EBFC44B012246
:1009B8001A70049B049A1B7843F0040313704FF4D5
:1009C8008063ADF82C3011238DF82E3063694FF019
:1009D800020943F480230BA98DF82F9040466361E8
:1009E80002F024FAB74BB84A1A6000200BF018FB43
:1009F800B64B1D60636943F480236361E36943F484
:100A08000013E361236B23F010032363236B43F08C
:100A180010032363D8F8203023F07063C8F820301F
:100A2800D8F8203043F08063C8F82030D8F8203058
:100A380023F07043C8F82030D8F8203043F08043C2
:100A4800C8F82030032300248DF831304046402375
:100A58000BA98DF832408DF833400B938DF8309008
:100A680006F068FD802340460BA90B9306F062FD53
:100A78002B6823F001032B602A68954B13402B60E9
:100A8800944B2B612B6843F001032B60AC60EC6046
:100A9800AC60AB68904C43F40043AB602B682B60B0
:100AA8006B6823F0784323F400436B602B6843F0B2
:100AB80001032B60B4F85C31002B40F05684B4F984
:100AC8005E21002A40F05184B4F96021002A40F0E8
:100AD8004C8400210C22814811F03FFD0021142292
:100AE8007F4811F03AFD7F4B002201201A7005F073
:100AF80063FF7D4B1A7842F002021A707B4A4FF46A
:100B0800805191614FF00A089946784DAB8A9BB2A3
:100B180083F48053AB8219200BF069FA01200BF0A3
:100B28007FFA19200BF063FA08F1FF3800200BF068
:100B380077FA18F0FF08E8D14FF48053AB616C4B9B
:100B48009FED6C8A1B686C4D1B7B00EE103AB8EE6B
:100B5800C00A20EE080A07F01DF9DFED687A20EEDA
:100B6800270A11F009FF664B9FED667A1880664BDD
:100B7800C5F87C315A4BD3ED047A644B67EE887A1A
:100B8800FF2167EE877A1B22C3ED007A604B184677
:100B980011F0E3FC5F4ADFF880E1126880F800801A
:100BA800012112F0020F8EF800101FBF41700321BF
:100BB8008EF80010022118BF8170510748BF9EF8B7
:100BC8000010734641BF01F1010E83F800E04FF0B9
:100BD800030E00F801E012F00A0F0ED01A78042173
:100BE8008154511CC9B24FF0050E00F801E0D11C28
:100BF8000232D2B219700621815431688A0641BF87
:100C08001A7802F1010E83F800E04FF0070E48BF92
:100C180000F802E00A060ED51A784FF0090E00F81F
:100C280002E002F1020E0132D2B283F800E04FF086
:100C38000A0E00F802E094F805E0BEF1080F02D0B1
:100C4800BEF10E0F08D11A7802F1010C83F800C02A
:100C58004FF00B0C00F802C01A7811F0040F4FF097
:100C68000C0800F8028002F1010C1CBFDFF8A88014
:100C780002325FFA8CFC83F800C01FBF88F800209E
:100C8800234A4FF0100802F80C801A7802F1010C80
:100C98005FFA8CFC4FF0120811F4806F83F800C0E3
:100CA80000F802803FD094F81082B8F1000F3AD0D3
:100CB800DFF86480023288F800202FE000540040FA
:100CC80058080020F42600205DB70008D410002042
:100CD800FFE0CF007A25E000B41100206C2300204B
:100CE8005C1D0020AC010020E8260020000400481C
:100CF8003802002035FA8E3C60080020000080434E
:100D080054020020BD378635A88980363402002079
:100D1800E1100020DC180020E0100020884A4FF085
:100D2800130802F80C801A7811F4007F4FF01408A9
:100D380000F8028002F1010C1CBFDFF86482023265
:100D48005FFA8CFC83F800C01FBF88F800207C4A3B
:100D58004FF0150802F80C80BEF1180F14D11A785C
:100D68004FF0160C00F802C002F1010C5FFA8CFC7F
:100D78004FF0170800F80C8002F1030C0232D2B2CF
:100D880083F800C000F802E00A0341BF1A7802F1B4
:100D9800010E83F800E04FF0190E48BF00F802E09A
:100DA800CA0541BF1A78511C19701A2348BF8354C9
:100DB80000219822634811F0D0FB0DF090FD624BA2
:100DC800624A1A60624BB4F85211198061490023D3
:100DD8000B808B7060490A60B4F8982190B25F4923
:100DE80021F813000133122BF9D13368D8045CBF02
:100DF800B4F89E0108801B0740F1058194F89231F0
:100E0800062B00F2FA80DFE803F004070E3D59795B
:100E1800790045F2F05201E042F6F822504B1A8070
:100E28000DF013FEE8E007EE902ADFED4E6A4C4B1A
:100E3800B8EEE77ADFED4C7AE7EE267A42F6F8214B
:100E480019800023FCEEE77A484A17EE901A42F818
:100E580023100133122BF7D1454A46491160464AFF
:100E68004020137005F070FC002800F0C6800123B4
:100E78004FF0070890F90000404A8DE8080140212A
:100E88003F4BB4E0364B42F6F8221A80384B3D4AC5
:100E98001A60394B102240201A7005F055FC0028C2
:100EA80000F0AB8001234FF0000C90F90000364AA7
:100EB8008DE8081040214FF4E13398E0284B42F6C2
:100EC800F8221A802A4B314A1A602B4B08224020FC
:100ED8001A7005F039FC002800F08F8001234FF0CC
:100EE800000E90F900002A4A8DE8084040214FF48E
:100EF800E13305F001FAC5F880017AE0184ADFF815
:100F0800A480DFF8A4C0DFF8A4E0224842F6F82164
:100F1800118019490C22062B0A7049D0002388F841
:100F280000308CF800308EF800301B2303701A4B09
:100F38001A701A4B05221A704FF4E13847E000BFC7
:100F4800E1100020FC230020B80A00203E130020F6
:100F5800BC0A0020BC260020B0260020101B002060
:100F6800A4020020CDCCCC3F0000B0C4C81A002099
:100F7800AC0000203D6C000898240020A96E0008F1
:100F8800A0860100296C0008FD6D0008116C00089E
:100F9800B16D0008561B0020531A0020571B002073
:100FA800E0100020541A0020551B0020541B00207C
:100FB800002188F800108CF800108EF8001021210C
:100FC8000170AA49DFF824830A70A94A1370A94B53
:100FD800A94A1A60402005F0B7FB70B1012100232F
:100FE800A64A90F900008DE80A004021434605F022
:100FF80083F9003018BF012028B9082006F08EFFB9
:101008009C4B9F4A1A6033689E4A13F4804F1FBF57
:101018000821117097499C4818BF086042F20101E5
:10102800194003F0010003F4005EA1B1974944F6AA
:10103800206CA1F800C0BEF1000F06D00821117085
:101048008C49DFF8ACE2C1F800E020B10C21117046
:1010580088498F4808601178043951701A0662D59A
:101068004FF0000ADFF88C82DFF88CB28948C5F8A7
:1010780084B15146152288F801A0C8F804A0C8F820
:1010880008A011F06AFA844A0392ABF105035046AE
:1010980013600AF0A3F8814B02201B68C8F80C30D3
:1010A80005F052FB039A964618B9802006F036FFE1
:1010B80031E098F8013090F805C079490C2202FB1C
:1010C80003125278624504D00133DBB2042BF4D901
:1010D800002388F80130DEF8003098F801201B78EA
:1010E80090F90000002B4FF00C0303FB021314BF10
:1010F8004FF0030E4FF0010E00225B78CDF800E0B0
:101108000192022105F0F8F8664B18600028CCD04F
:1011180001200AF063F8644B1868644B00F5C57247
:101128001A600AF009F933685B055CD5604BD5F89D
:10113800A0A1C3F800A0042005F006FB0421C5F80F
:10114800A40105F0DBFA5B4B85F8A8010820C3F879
:1011580000A005F0F9FA584BDFF8A08118600821C3
:1011680005F0CCFA002185F8A9012C22404611F09F
:10117800F4F98E227C2388F801204FF07D0BE022C1
:1011880088F8003088F8032088F82BB0DFF87081E1
:1011980003932C220021404611F0DFF9039B88F8C5
:1011A80000308A2388F801301020A02388F8033003
:1011B80088F82BB0C5F8ACA105F0C6FA1021C5F81F
:1011C800B00105F09BFA85F8B4012020C5F8B8A154
:1011D80005F0BAFA2021C5F8BC0105F08FFA85F8A8
:1011E800C0010BF0FDFD3368344A13F4002318BF27
:1011F800012313700AF0D4FE314B18606379052B74
:1012080002BF304B4FF4C8721A802F4B4FF47A72DA
:101218001A803B782D4A43F008033B70137823F07B
:1012280002031370326840F6020313406BB1284B77
:10123800284A1A60284B03221A70284B01221A7078
:10124800274A00231380274A1380A3683360264B5C
:1012580001221A7099F8003063F07F0389F8003092
:1012680023B0BDEC028BBDE8F08F00BF531A0020FD
:10127800571B0020AC0000202D6B0008916C000863
:101288004DF6000898240020716C0008A402002084
:10129800816C0008E8090020A401002094260020A1
:1012A800743E0108C81C002014110020100B0020F7
:1012B800D01800202819002074190020CA24002002
:1012C80084020020CA0A00200827002010270020D6
:1012D800C8180020301300202C190020FC00002022
:1012E800A8100020AA1000205808002090D0030061
:1012F80041F6000884010020A8130020F8180020F7
:101308002D190020013B092B3FF644A8D9F81800F5
:10131800306031464FF0904001F088FD4FF0904327
:1013280008229A613C200AF062FE97F893319A45A8
:10133800BFF62AA8214A4FF0904B4FF4805108235A
:101348009161782006910592ABF8283003930AF052
:1013580043FE059A0699039B11857820CBF818302F
:101368000AF03AFE0AF1010ADFE71BB207EE903AEB
:10137800DFED136AB4F95E31124AF8EEE77A07EE48
:10138800103A67EEA67AB4F96031CDED0B7A07EE24
:10139800903AB8EEC77AF8EEE77A002127EE267A77
:1013A80067EEA67A11700BA807498DED0C7ACDED82
:1013B8000D7A06F0F7FCFFF78CBB00BF000400486D
:1013C80035FA8E3C68000020EC1B0020804A2DE98D
:1013D800F04F15687F4C05F59C4320332DED028BAB
:1013E80023607D4B196889B011F4804F05929846A7
:1013F80005D10EF075F910B9237901332371774BB4
:101408001F78C7B1764A1268954240F2FF80013FC3
:101418001F70FBE0D9F800307248072D98BF595D5E
:10142800714B88BF29461B689847032D0BD904EBDD
:1014380045050137E8806B4BDFF8C8911E78FDB28F
:10144800AE42E7D820E0D9F8002005F10E0302EB00
:1014580083039988DA880028E9D04FF47A73401A10
:101468005843531A90FBF3F040F6C90300F57A701D
:10147800984205DC40F2EE239842B8BF184601E0D6
:1014880040F6CA0080B2D2E70F23277984F82A30C1
:1014980094F82B300193032594F82C30B7FBF5F51D
:1014A80005EB45057D1B0393D9F800300293DFF85F
:1014B80058A1EBB204930025B54254DA4B49019B7D
:1014C80031F815B04FEA450953B90EF009F928B1BA
:1014D800039B002B08BF4FF0000B01E0DDF804B0C0
:1014E800029B988A584502D8D88A58450ED2E8B245
:1014F8000EF0AAF8032D8346DFBF94F82AE00120F6
:10150800A8402EEA0000D8BF84F82A000EF0E8F8B8
:1015180018B1374829F800B021E0049B94F8760008
:101528002AF813B028B9022F15D92A49012081F8C1
:101538007600BAF80210BAF800000844BAF80410A5
:1015480008442C4980B229F8010000B2032190FB1D
:10155800F1F080B200E05846254929F8010001352C
:101568000AF1060AA8E794F82A202348234BA2F197
:101578000F0EDEF1000242EB0E0284F890206AB1F1
:101588001F4A1268570109D40268D9689A60521A2A
:10159800C82A3BD9012283F8212037E002689868DD
:1015A800DA605B68121A9A4288BF144B4FF0000148
:1015B80084F82B1088BF83F821100025B54225DA5E
:1015C800E8B20EF041F80A4B23F815000135F5E7AB
:1015D800F0260020240A002070260020B8260020CB
:1015E800B426002098240020AC0000202A0A0020FD
:1015F800101B00209C0A002094260020BC260020F6
:10160800DC100020B0260020520A0020D8F8003054
:10161800DE0405D58C4B1B68DD0701D40DF028FCD2
:101628008A4B1A68937A2BB3013B8949127B31F8AC
:1016380013301AB1C3F53B6308339BB21BB2A3F551
:101648007A73B3F57A7FA8BF4FF47A7323EAE3730A
:1016580007EE903A9FED7F7A7F4AF8EEE77AC7EE79
:10166800877A9FED7E7A67EE877AFCEEE77A17EE47
:10167800903A1380D8F80030794F13F4807F00F047
:101688000481059BDFF8E0911A68764B9A4205D9E8
:1016980099F8022012B9012289F8022099F802204B
:1016A800002A00F0F280704A3E7892F82150664A8B
:1016B800681E454211684541002DC1F38063C6F399
:1016C80080060193924614BF4FF0000B4FF0030BB6
:1016D80099F82020052A00F2D280DFE802F0034DB5
:1016E800527584A1002E3AD0D4F89400B4F898101A
:1016F80005F0CDF8012809D15C495D4A09681268EE
:10170800C988642000FB0122C9F81020019B6BB135
:10171800564A126812794AB109F0EAF9032289F89F
:1017280020204FF47A72C9F81C20D1E7002D40F030
:10173800A6804F4AD9F8101010684B4A88420AD937
:10174800029209F0D5F9029A032182F8201040F696
:10175800B831D161BCE7012182F82010B8E7019BBC
:101768004FF4806013B106F0C9FB01E006F0B5FB49
:101778000022C9F8102082E0002D46D109F0B8F9FE
:10178800A6E725B1052289F82020012000E0284697
:1017980066B1D4F89420D1892D4A11805180918066
:1017A800324909684988D1804FF0020B304A1168E4
:1017B800D9F81420914201D8002E5DD147F2305259
:1017C800C9F81C20032221E03A7842F002023A705C
:1017D8000DF04EFB264AD9F81C1012680A44C9F8C5
:1017E8001820042212E0224A9DB11168D9F8182065
:1017F800914244D91F4A12781AB9DAF80020D10761
:101808003DD43A7822F002023A70052289F8202065
:101818005EE71268D9F81C100A44C9F818202EE0AF
:101828001249134A09681268C988642000FB01221A
:10183800C9F810204FF48060002289F8202089F828
:10184800032006F04AFB43E7DC100020B026002006
:10185800101B002000007A443011002000C07F4493
:1018680010270020404B4C00BC260020941D00206F
:10187800942600201000002000287FF429AFBBF137
:10188800000F02D0584605F05DF8AD4D05F5C5705E
:10189800B5F8521104F0FBFF834668B909F01AF94C
:1018A800A84BC3F800B0C3F804B0C3F808B0A64BFF
:1018B80000221A605A609A603B785A0736D5D8F8E1
:1018C8000030DB0632D5A14B1B78DE062ED4A04BA8
:1018D8001B7893B195F8E231BBF1000F15D17BB1BC
:1018E8009C4B1A68D4F89C309B1A002B08DA0DF030
:1018F800BFFA994B83F8A0B018E0BBF1000F0DD1E7
:10190800102005F01FF801230EE03BB1914A126840
:101918004FF47A7101FB0323C4F89C3094F8A0308B
:1019280023B104F0F9FF002384F8A030002295F8D1
:10193800E0A195F8E111B5F89AE1B5F89CC1134614
:10194800864E019636F912009B087045C4BF63F0B5
:101958007F03DBB201326045B8BF43F04003042A7D
:10196800EED194F8A1207C489A4205D190F8A220A3
:10197800F92A04D8013200E0002280F8A22084F875
:10198800A130734B764E1A789946E2B93368D80776
:1019980008D5BBF1000F16D13B78D90713D50DF048
:1019A800F5F810E03B785A070DD56B4B93F82B30C0
:1019B8004BB16C4BDB7833B911B10DF059FA02E039
:1019C800BBF1000FF9D094F8A230634ADFF8A4B154
:1019D800142B40F0898099F800301AF1000A18BFDA
:1019E8004FF0010A6BB392F8A1305F2B11D13B780D
:1019F80003F0040303F0FF0113B10DF039FA08E016
:101A08000B200391029204F09DFF029A039982F839
:101A1800A210BAF1000F14D094F8A1307D2B10D188
:101A28003B7803F0040303F0FF0213B10DF020FA32
:101A380007E00B20029204F085FF474B029A83F8D7
:101A4800A2203B7803F0040303F0FF01002B4BD1E5
:101A580094F8A130404A572B11D1434B4FF47A7276
:101A68001A80D8F800301B0601D509F0C7FC3F4B97
:101A78001B6813F0080337D13D4A138034E0D8F8C7
:101A88000000400717D55A2B15D192F8A3302BB177
:101A9800012382F8A31082F8A43025E092F8A5303B
:101AA80083F0010382F8A5300BB10C2000E00D2073
:101AB80004F048FF18E05D2B00F000855B2B00F078
:101AC8001B855E2B00F01A85562B01D106F0B8FC59
:101AD80099F80030002B00F0C48494F8A1306F2BE3
:101AE80040F0B9840DF052F8D8F800305A0752D5B2
:101AF80094F8A530184A93B13B785B070FD5019B42
:101B0800B3F90610B5F89A31994208DD336813F035
:101B1800010302BF3221A2F8A81082F8A530336869
:101B2800D80329D594F8AA200B4B2AB993F8A320F7
:101B380012B93222A3F8A820012384F8AA302AE097
:101B4800B4110020EC1F002070200020E0180020B5
:101B58001000002094260020240A0020101B0020DA
:101B6800DC100020BC26002008270020DC180020FC
:101B7800A81100201411002094F8A330B74A53B1DB
:101B88003B7803F0040303F0FF0123B9012382F833
:101B9800A31082F8A430DBF800A0002333600AF118
:101BA8007B090AF1CB0B99F8002099F8013019F854
:101BB800010C9A420BD2494604F032FE38B119F8AA
:101BC800022C012303FA02F233681343336009F14C
:101BD8000409D945E7D1A24B1B7843B1A14BA24ECA
:101BE8001A6812F0020F994640F03E8335E30AF175
:101BF800CA060AF589793278737816F8010C9A4280
:101C080025D2314604F00CFE08B3B37896F804E008
:101C1800964A96F803A091480C21013B01FB0E411E
:101C280003EB43031344D1F8B0209A420FD0C1F814
:101C3800B030002390F8DC20C1F8B430012303FA57
:101C48000EF322EA030381F8ACA080F8DC300636F4
:101C58004E45D0D1864B1E68864B1B68039394F87B
:101C68002B300493844B019300230293019B1B6840
:101C7800002B00F0E78293F800A0BAF1000F00F003
:101C8800E182019A039952688A1A002A0CDB01F54D
:101C9800FA7201994A60029901228A4094F8DC108C
:101CA80021EA020284F8DC20049A002A00F0CA82A1
:101CB800019A597812F8042C0432D2B2002940F063
:101CC80080826E4931F91210B5F8982102F1C800E6
:101CD800814202DD93F802B015E0C83A914203DA76
:101CE8009978C1F1000B0EE0029A0123934094F811
:101CF800DC2022EA030384F8DC30039B019A03F515
:101D0800FA7353609EE294F8DC30029A1341D907C3
:101D180000F19882BBF1000FCCBF0220012004F033
:101D280033FE0AF1FF33DFF83491132B00F282827D
:101D3800DFE813F01400250037004B0064006B0047
:101D4800EB004E01B501E501150280024B005A0077
:101D58006B00EB004E01BB002001850196F8009056
:101D6800D944B9F1FA0FA8BF4FF0FA0929EAE9797D
:101D7800304686F8009004F039FD01200FE096F80F
:101D88000190D944B9F1640FA8BF4FF0640929EA5A
:101D9800E979304686F8019004F028FD022049468A
:101DA800DAE196F803A0DA44BAF1640FA8BF4FF05D
:101DB800640A2AEAEA7A86F803A03046D9F8E010DD
:101DC80004F0CAFC03205146C6E1717959446429DC
:101DD800A8BF642121EAE17171710D2004F088FD2A
:101DE800BAF10D0F00F02682317959446429A8BF51
:101DF800642121EAE17131710E20ADE1B1795944D4
:101E080081F30801B1710520A6E1D9F8E4301A7808
:101E1800022A3BD107EE90BAF8EEE77AB2EE040A4E
:101E280087EE800AD3ED097A30EE270AB5EEC00AAC
:101E3800F1EE10FA09D4DFED137AB4EE670AF1EE89
:101E480010FAC8BFB0EE670A01E09FED0F0A83EDF4
:101E5800090A0F2004F036FD23E000BF240A002001
:101E680011270020DC100020DC180020B8420108EF
:101E78003411002094260020D40A0020101B0020D2
:101E880000007A440000C8420000000099785944D4
:101E9800C829A8BFC82121EAE17199700F2004F070
:101EA80027FDBAF10F0F00F0C581D9F8E4301A7890
:101EB800022A20D107EE90BAB8EEE78AB2EE040AF9
:101EC80088EE008A93ED080A38EE000AB5EEC00ADB
:101ED800F1EE10FA09D45FED157AB4EE670AF1EE67
:101EE80010FAC8BFB0EE670A01E01FED190A83EDCA
:101EF800080A122058E159785944C829A8BFC821AE
:101F080021EAE1715970122026E1D9F8E4301A78F3
:101F1800022A20D107EE90BAB8EEE70A5FED277AD9
:101F280093ED0C7A80EE270A30EE070AB5EEC00A68
:101F3800F1EE10FA07D4B4EE670AF1EE10FAC8BF52
:101F4800B0EE670A01E01FED300A83ED0C0A10209D
:101F580004F0B8FC0AE0197B5944C829A8BFC82175
:101F680021EAE1711973102004F0C2FCBAF1100FD4
:101F780000F06081D9F8E4301A78022A1ED107EE01
:101F880090BAB8EEE78A5FED417A93ED0B0A88EED6
:101F9800278A38EE000AB5EEC00AF1EE10FA07D427
:101FA800B4EE670AF1EE10FAC8BFB0EE670A01E0B6
:101FB8001FED4B0A83ED0B0A1320F5E0D97A59443B
:101FC800C829A8BFC82121EAE171D9721320C3E04A
:101FD800D9F8E4301A78022A22D107EE90BA1FED18
:101FE800580AF8EEE77A87EE800AD3ED0F7A30EEDA
:101FF800270AB5EEC00AF1EE10FA09D45FED5F7A50
:10200800B4EE670AF1EE10FAC8BFB0EE670A01E055
:102018001FED630A83ED0F0A112004F053FC0AE058
:10202800997D5944C829A8BFC82121EAE171997549
:10203800112004F05DFCBAF1110F00F0FB80D9F813
:10204800E4301A78022A20D107EE90BA1FED740AFC
:10205800B8EEE78A88EE008A93ED0E0A38EE000A99
:10206800B5EEC00AF1EE10FA09D45FED7A7AB4EE53
:10207800670AF1EE10FAC8BFB0EE670A01E01FED7B
:102088007E0A83ED0E0A14208EE0597D5944C82932
:10209800A8BFC82121EAE171597514205CE0D9F87C
:1020A800E4301A78022A20D107EE90BAB8EEE78A0F
:1020B800B2EE040A88EE008A93ED0A0A38EE000AA6
:1020C800B5EEC00AF1EE10FA09D45FED927AB4EEDB
:1020D800670AF1EE10FAC8BFB0EE670A01E01FED1B
:1020E800960A83ED0A0A09205EE0D9785944C8297E
:1020F800A8BFC82121EAE171D97009202CE0D9F8DC
:10210800E4301A78022A1ED107EE90BAB8EEE78AB0
:102118005FEDA47A93ED0D0A88EE278A38EE000A5F
:10212800B5EEC00AF1EE10FA07D4B4EE670AF1EE84
:1021380010FAC8BFB0EE670A01E01FEDAD0A83EDE3
:102148000D0A0A2030E0597B5944C829A8BFC82184
:1021580021EAE17159730A2004F0CAFB6AE0D9F850
:10216800E4301A78022A22D107EE90BA1FEDBC0A91
:10217800B8EEE78A88EE008A93ED100A38EE000A76
:10218800B5EEC00AF1EE10FA09D45FEDC27AB4EEEA
:10219800670AF1EE10FAC8BFB0EE670A01E01FED5A
:1021A800C60A83ED100A0B2004F08CFB42E0D97DAF
:1021B8005944C829A8BFC82121EAE171D9750B2063
:1021C800CAE7012936D19878BD4B33F91230B3F5F7
:1021D800617F05DB40F633029342A8BF134601E056
:1021E8004FF46173BAF10C0F24D14FF4966292FB4D
:1021F800F0F0B44AA3F5617393FBF0F35FFA83F947
:1022080013784B4516D0B9F1040F34BF4B4602235F
:102218001370AD4A0AFB035303F2EA63136005F037
:1022280049FF5046494604F063FB09F10100C0B27A
:1022380004F0AAFB029A0123934094F8DC2013438C
:1022480084F8DC30029B01330293019B0C33019329
:10225800029B042B7FF40AADC0E4D8F80030DA05FD
:1022680010D59A4BDB786BB133689B070AD5984B2E
:102278001B8813F0010A0AD108F02CFC012005F094
:102288003DFE04E0012005F028FE012300E00023C4
:10229800D9F8002050070DD563B1012005F01DFEC7
:1022A8008B4B1B88990708D408F014FC022005F012
:1022B80025FE02E0022005F010FE33689A0609D4D4
:1022C800D9F800301B0540F194804FF4807005F078
:1022D80015FE92E07F4BDFF8F8A11B7813F0020F90
:1022E80053D07D4B1B78042B4FD9D9F8003013F409
:1022F800007B0FD0BAF80030DE063AD4102005F083
:10230800FDFD202005F0E9FD7448011D08F0CAFF15
:1023180002232AE0BAF8006006F01006B6B22EB121
:10232800102005F0DAFD012684F8E8B0D9F800306D
:10233800580512D5D4F8EC3069495A89B1F90030FA
:10234800002BB8BF5B42934207DAB1F90230002B89
:10235800B8BF5B429342C0F2F880BAF800309906E1
:1023680008D5202005F0B9FD002384F8E8300126BF
:1023780000E0002694F8F030BBB90E2004F0E2FA31
:10238800584B012283F8F0200FE0BAF8003003F030
:102398003003002B94D0102005F09FFD202005F07D
:1023A8009CFD002384F8E83001E0002E88D04E4BD5
:1023B800002003F1280603F150044C4A002122F8BA
:1023C80010104B4A596022F810100432716022F83C
:1023D800101000221A609A603260B2602260616058
:1023E800A26014331436143400287FF469AF012036
:1023F800E3E74FF4807005F070FD6B79082B01D08E
:102408000E2B02D1402005F068FDD8F800305A059F
:1024180040F1B18095F810321BB93B7813F0040FE6
:1024280003E0D9F8003013F4002F0BD0314B002211
:102438001A703C200CF052FB002800F09C800BF036
:102448004FFAF6E70AF0CCFC09B0BDEC028BBDE808
:10245800F04F0CF044BABAF1000F02D07E2B3FF4D3
:1024680041AB94F8A130972B06D11E4B4FF4C8729C
:10247800A3F8A620FFF738BBA72B06D1154A137877
:1024880043F004031370FFF72FBB0022BB2B079206
:1024980001D1022303E0B72B04D14FF6FE73ADF848
:1024A8001E303BE0BE2B01D1022304E0BD2B7FF49C
:1024B8001BAB4FF6FE73ADF81C302FE001201EE079
:1024C800101B00204C23002034110020BC260020C3
:1024D800A4190020E0180020E61800203C11002074
:1024E800AC110020240A0020180B00200A27002025
:1024F800900B00209D240020022000E003205FFABA
:1025080080F909F1FF3385F8E83605F039FD05F063
:10251800F5FD484604F038FAFFF7E6BADBF8003074
:10252800BDF81C10B3F858200A44A3F85820BDF889
:102538001E10B3F85A200A44A3F85A2005F080FF69
:10254800002384F8A230FFF7CFBABAF800309B0610
:102558003FF510AF202005F0D1FC0948094B011DBB
:102568001A685B684360026008F09CFE064B01260F
:1025780083F8E860FEE609B0BDEC028BBDE8F08F99
:1025880044110020E8180020240A0020026BC168CA
:10259800034610B5406942B11A6C8C1A013A005DC5
:1025A80008BF0A46C0B21A6410BD1A6A805C0132BC
:1025B8008A4228BF0022C0B21A6210BD436B13B111
:1025C80090F844007047836A406A1B1A5842584181
:1025D8007047036B13B15B68016C01E0C369016A62
:1025E8008B423CBFC2689B18581AC0B27047836AB6
:1025F8008169426B1944D160416A99429DBF016962
:10260800CB1A5360CB1A96BF0023536083624FF0F6
:10261800000380F84430136888BF816243F00103E7
:1026280013607047436A8269D154436A026901336F
:10263800934228BF00234362436B1BB11B68DB072F
:1026480005D4D4E7026D136843F080031360704724
:1026580010F80A3C0133DBB20A2B84BF10F8131CB4
:10266800044A00F80A3C82BF002322F8113000F81F
:102678000A3C7047341B0020334A136C9068194495
:10268800081A40F68C23984270B513469160D060C2
:1026980051603BD9127893F945108A4210460BD104
:1026A800111F082908D893F84610182901D80131B4
:1026B80003E083F8442002E0002183F8461093F9F0
:1026C80044402149A24219D191F84740B4B10C3194
:1026D8000024944206DA1D4D51F8046F25F8146061
:1026E8000134F6E70C2805D01849002421F81040D9
:1026F8000130F7E7164801780131017083F8452069
:10270800002201211A7083F8471070BD92F8471013
:10271800C9B1A0F2EF2440F2DA518C4208D81178FE
:102728000B2905D80B1D0131117042F8230070BD2B
:10273800002283F84720074B03F13002002143F8B9
:10274800041F9342FAD170BD90080020341B00206A
:102758007C0100209C080020024A136C01331944B4
:102768001164704790080020024B53F820301B6812
:102778001960704794200020064B53F820301A68DF
:102788001B89A1F57A7159434FF47A7391FBF3F1E0
:102798001160704794200020F0B5046D86682368A6
:1027A80023F0010323608379054613F0020F407973
:1027B8000CBF4FF0000E4FF4005E13F0040F14BF6F
:1027C8004FF48067002710F0010F14BF0421002187
:1027D8008307206820F001002060626822F44052DC
:1027E8004EEA02026260226822F4B05323F00C031E
:1027F80048BF41F008013B430B432360A36895B0F1
:1028080023F44073A360684604F026FD284B9C42DD
:1028180001D10C9B0EE0274B9C4201D10D9B09E096
:10282800254B9C4201D10E9B04E0244B9C420CBFDB
:102838000F9B109B2268A879170448BF5B00B3FB65
:10284800F6F206FB1233B3EB560F236828BF0132AA
:102858001E0441BF4FF6F073C2F34201134041EA30
:1028680003026B7992B213F0020FA28100F001010A
:1028780014BF4FF400320022DC0748BF42F4803214
:102888002B6D11B159680A4302E0596821EA020226
:102898005A609A6801074CBF42F0080222F0080209
:1028A8009A601A6842F001021A6015B0F0BD00BFC4
:1028B800003801400044004000480040004C0040FF
:1028C800417169E7816067E7026D036B70B5044683
:1028D800D5699BB9A90611D5C36A1BB1908C80B282
:1028E80098470BE0E169928C40694E1CD2B2E661D0
:1028F8004254E169E268914228BFE361616BA1B982
:102908002A0612D5636AA26A9A42236D09D0501C1E
:10291800A669A062B25C1A852369984205D3A162B0
:1029280003E01A6822F080021A602B0742BF236D69
:1029380008221A6270BD0D4B0D484FF400525A60C0
:102948000C4A11684FF6FE730B401360426B116816
:102958004FF6FE730B401360426A836A9A4200D0B6
:1029680045E6012380F84430704700BF000002406C
:10297800781F0020440002402DE9FF471D46B24B56
:102988009DF8306098428846174640F08680AF4BE5
:10299800AF4A1A60AF4A5A6102F580729A614FF4E1
:1029A8008072DA601A61AC4A1A63143A5A63A2F563
:1029B8004842203ADA6404329A649F601865A74B4B
:1029C8009A6942F480429A615A6942F001025A6156
:1029D80002238DF80C30032316F0010A8DF80D3010
:1029E8004FF000038DF80E3014BF02230123310786
:1029F8008DF80F301BD54FF090444FF40079CDF887
:102A080008908AF001038DF80E30636A23F0F00312
:102A18006362636A43F070036362204602A904F0AC
:102A280089FDBAF1000F28D1C4F8189025E0AA074B
:102A380010D504A94FF4007341F8083D4FF09040B9
:102A4800436A23F0F0034362436A43F0700343622E
:102A580004F070FDEB0710D504A94FF4806341F82A
:102A6800083D4FF09040436A23F470634362436A21
:102A780043F4E063436204F05DFD0E238DF80430F7
:102A88000022012301A88DF805308DF806208DF865
:102A980007306E4C0CF020FA75E0714B984240F00C
:102AA800F380704B6A4A1A604FF48072DA601A61D8
:102AB8006D4A5A6102F580729A61684A9F6018658A
:102AC800D36943F40033D36102238DF80C30032318
:102AD80016F0010A8DF80D304FF000038DF80E3016
:102AE80014BF0223012334078DF80F301AD55F4C29
:102AF8004FF02009CDF808908AF001038DF80E30C8
:102B0800236A23F470032362236A43F4E0032362F5
:102B1800204602A904F00EFDBAF1000F24D1C4F832
:102B2800189021E0A8070ED504A9202341F8083DF4
:102B38004E48036A23F470030362036A43F4E00314
:102B4800036204F0F7FCE9070ED504A9402341F815
:102B5800083D4648036A23F070630362036A43F042
:102B6800E063036204F0E6FC26238DF804300022BB
:102B7800012301A88DF805308DF806208DF807305F
:102B88000CF0AAF9374CC4F82C80012384F844309F
:102B980000232362E361A36263626571A760A67183
:102BA8002046FFF7F9FDEA0729D5206B00B3D4F8D2
:102BB8004C80E668676904F0C3FA236B216D1A68D4
:102BC80022F4FF4222F0700242F48552B6B21A6033
:102BD8005E60C3F80880DF601A6842F001021A607C
:102BE8008A6842F040028A605B689BB2236406E010
:102BF800236D20221A621A6842F020021A60AB077D
:102C08003BD5606B002833D0A66C256904F098FA90
:102C1800636B1A6822F4FF4222F0700242F4845275
:102C280042F010021A60ADB200225D609E60DA6068
:102C3800196841F0020119605A605A60226D936860
:102C480043F08003936018E000380140781F0020AB
:102C5800F4420108980B002058000240001002407E
:102C680000440040241F0020980D0020000C00485C
:102C7800226D136843F080031360226D136843F0DC
:102C880001031360204600E0002004B0BDE8F0878F
:102C98003D4B1B78012B30B514BF00240324B1B978
:102CA800036A23F0010303628169036A21F0F301D7
:102CB80023F00A0341F0010142F001021A4341EAFC
:102CC800041181610262836923F00C031BE004296B
:102CD8001DD1016A4FF6EF730B4003628169056AE3
:102CE800120121F473414FF65F7342F0100241F470
:102CF80080712B4092B2134341EA0431816103622F
:102D0800836923F4406383618369836130BD082943
:102D1800016A1AD14FF6FF630B400362C169036A67
:102D28009BB289B223F4206343F4807321F0F3014A
:102D380043EA022241F0010192B241EA0411C16161
:102D48000262C2694FF6F37319E04EF6FF730B4047
:102D58000362C369056A40F6FF41194045F6FF73EF
:102D68002B4043F4805343EA023241F4807192B21B
:102D780041EA0431C1610262C2694FF2FF33134074
:102D8800C361C369C36130BD8C08002038B510F831
:102D98000E2C50F8043C044652B9012200F80E2CBF
:102DA80020F80C1C997A18680222BDE838406FE7B1
:102DB80030F80C2C20F80A1C891A89B220F8081C53
:102DC800074A10F80F0C002522F8101004F80E5CC2
:102DD8001868997A2A46FFF75BFF04F8065C38BD45
:102DE800341B0020044B53F820301BB107289CBF2C
:102DF8001B681960704700BFB8090020084A1368AB
:102E08009B050BD5074B00211970074908684FF639
:102E1800FE7303400B604FF400735360704700BFAC
:102E2800000002400F2700203000024073B506461C
:102E38000D46002401232A88A34013421AD0AA78F9
:102E4800009302F003038DF80430EB78022B03D0D3
:102E5800032B0CBF032301238DF805303046C2F342
:102E680001136946C2F381028DF806308DF80720F8
:102E780004F060FB0134102CDCD102B070BD2DE9E8
:102E8800F743DFF81C9299F8004405468E4600681F
:102E98001146164698467246631C89F8003408F0B5
:102EA8006FFB2B89ADF8043001A9022368688DF8FF
:102EB80006308DF80730FFF7B9FFAB7A2A6809F2B8
:102EC80004472401274449460C2B00F2B780DFE869
:102ED80003F007B5B5B53EB5B5B56AB5B5B5930058
:102EE800136ADFF8C0C123F001031362136AD2F832
:102EF80004E0906920F4803020F07300624540F0CF
:102F0800700012D00CF5006C62450ED00CF5406CC8
:102F180062450AD00CF5806C624506D00CF5806CD1
:102F2800624502D043F0030307E023F00E032EF4BA
:102F3800407E43F003034EF4807EC2F804E09061C3
:102F4800C2F834801362936943F0080329E0136AD6
:102F5800DFF850C123F010031362136AD2F804E0BB
:102F6800906920F0807020F4E640624540F4E0402B
:102F780006D00CF5006C624502D043F0300307E040
:102F880023F0E0032EF4406E43F030034EF4806EDD
:102F9800C2F804E09061C2F838801362936943F480
:102FA800006393614AE0136ADFF8F8C023F4807382
:102FB8001362106AD2F804E0D369624523F0730300
:102FC80043F0700306D00CF5006C624502D040F463
:102FD800407007E020F460602EF4405E40F44070DA
:102FE8004EF4805EC2F804E0D361C2F83C801062FF
:102FF800D36943F0080320E0136ADFF8A8C023F47C
:1030080080531362106AD2F804E0D369624523F44E
:10301800E64343F4E04340F4405003D00CF5006C21
:10302800624501D14EF4804EC2F804E0D361C2F883
:1030380040801062D36943F40063D3612B7B1BB1DA
:10304800536C43F40043536413889BB243F0010369
:103058001380AB7A0C2B19D8DFE803F0071818187F
:103068000B1818180F18181813000B1902F1340050
:103078000AE00B1902F1380006E00B1902F13C00D6
:1030880002E00B1902F14000C3F804040C4438466E
:10309800A4F80C64C4F8082403B0BDE8F08300BFAA
:1030A800980B0020002C01402DE9F04FC14BB3F9DB
:1030B8000610C14B2DED028B1F687A8987B09142AB
:1030C80001930EDBB1F5FA6FFC79BDBF8B1A634330
:1030D800A2F5FA64C4F16404BCBF93FBF4F464344D
:1030E80000E06424B54AB64BB2F898A192F962217F
:1030F8001868049092B20592054600220293AD4BDF
:1031080033F912300393CAEB030303F2F31640F2C8
:10311800E63086424FEA420B03D8002BB8BF5B4229
:1031280001E04FF4FA73022A049E4FF064002FD096
:1031380096F811E1BEF1000F04D07345CCBFCEEB79
:1031480003030023DFF8C0E293FBF0FC6FF0630990
:103158003EF81C809B4E09FB0C390CF1010C3EF922
:103168001CE00FFA88FCCCEB0E0E0EFB09FE9EFB52
:10317800F0FEC64426F80BE0BE1836797343924E2B
:1031880093FBF6F364339BB2634393FBF0F02EE0BA
:1031980096F812E1BEF1000F04D07345CCBFCEEB18
:1031A80003030023DFF84C8293FBF0F06FF0630C0D
:1031B8000CFB003938F910E00130002B38F9100009
:1031C800CEEB000000FB09F9BDF8140099FBFCF9EF
:1031D800CEEB090919FB00F97A48A0F80490B879F0
:1031E800B8BF5B424343784893FBF0F064306B7898
:1031F800764E4FF0640E434393FBFEF3B354744E84
:10320800EB7A434393FBFEF3B3546B7D6D4E584307
:10321800704B90FBFEF0022A98546F4B0FD183F845
:1032280002E0039B53450EDB644CB4F89A219142AB
:1032380015DBB1F5FA6FA8BF4FF4FA6110E09C54A2
:10324800039B534504DA36F80B305B4226F80B3003
:103258000132032A05F101057FF451AFE4E7114675
:10326800891A4FF47A73DFF8A4E1564D59436FF089
:1032780063036427C2F5FA62B1FBF2F191FBF7F23E
:103288003EF8120003FB0211013203B23EF912208C
:10329800D21A514391FBF7F30344F3804F4B1B8839
:1032A8005F0635D54E4B4F4A1B881288DFED4E7AA4
:1032B8009B1A1BB208EE103AB8EEC88A28EE278A85
:1032C800B0EE480A04F066FDF0EE408AB0EE480A17
:1032D80004F0FDFCB5F9023006EE903AB5F900307D
:1032E800F8EEE66A07EE903A20EE667AF8EEE77AAC
:1032F800A7EEA87A67EE807ABDEEC77AE6EEA87ADE
:1033080017EE103AFDEEE77A2B8017EE903A6B80B5
:10331800364D2B68980740F1A180354B354F1A6818
:103328007B6945F20721D31A8B4240F397807A6173
:1033380004F0EEF9304BDFF8D8901A78032A984653
:10334800B9F8003022D10A2B2AD90023282088F87E
:10335800003008F04CFE04F0DBF9284B188804F024
:10336800C1F9274B1A68D37890FBF3F0013008288D
:10337800244BA8BF08201870537980B213FB00F3C0
:103388003B83137913FB00F0788309E00A2B07D8F5
:1033980003231C4A88F80030002313703B837B8387
:1033A80098F80030144A012B3DD033D3022B4CD06F
:1033B80054E000BF101B002034110020B41100207D
:1033C80014110020AC1100200CFEFFFF8420002007
:1033D8009E10002087200020CC1F0020A419002068
:1033E800A8110020C824002035FA8E3C7026002041
:1033F800F0260020901000202C190020101C00201E
:10340800C8180020FC000020FA190020E21900204A
:10341800CC1800203A8BB9F800309A421EDD0123FF
:1034280088F800300FE0B9F800107B8B8B4202DD82
:10343800022313700FE09B4B1B8B0133994202DD73
:10344800002313700AE0082006E07B8BB9F80020FF
:1034580001339A42E3DC072003F074FA2F68390538
:1034680070D5914B8F4D1A68EB69C3EB020845F292
:103478000723984566DD8D4BB6F906B0D3F8009062
:10348800EA6199F80A30B4F85211894E012B4FF4C9
:103498007A70ABF57A7B98FBF0F803D03BD3022B1C
:1034A80019D03AE02A6A082192FBF1F3D31A0022D4
:1034B8002B62AA8493FBF1F340F6E4429BB2534398
:1034C800B9F80820C2EB13335843B9F9063090FB1A
:1034D800F3F0306021E0774BB9F808A01B78C6F804
:1034E80000A05A0719D5744803F0D1F920B917F08C
:1034F800100F18BF4FF0000B32220BFB0BF393FB9E
:10350800F2F3B9F906205B445A434FF47A7392FBFD
:10351800F3F3534400E000233360D5E90A0133682C
:10352800664A03FB08F84FF47A7398FBF3F810EB3C
:10353800080041EBE8710023C5E90A010CF01CF909
:103548005F4B18605F4E3368DB0427D53F0622D5F2
:103558005D4B1B789D071ED55C4B187804281AD93B
:1035680000225B4BD7180521951C4FF00A0E122A32
:10357800D154E9B287F801E004D0B0EB510F2A46E4
:10358800EFD800E014215A18322002F8010CFF226B
:103598005A540F2000E00A2003F0D4F94D4D2A6850
:1035A800002A50D04C4B4D4F1868396881429846D4
:1035B80049D84B4BDFF8349119785268E1B94FF08C
:1035C800010A83F800A0B9F80030D35C23B3504651
:1035D80008F026FD434B83F800A00CF08DF8B9F8ED
:1035E8000030CBB92B681B78053B534514D808F03D
:1035F800D7FC3D4B18600FE04FF0000A83F800A09D
:10360800B9F80030D35C3BB1504608F009FD354BA2
:1036180083F800A00CF070F82A68B9F800305268F6
:103628003248D25CFE2A01D100230BE0FF2A02D1E6
:1036380003F072F907E0D8F800500A2111FB025292
:103648003A60013303801B4D2B78580704D5284B6B
:103658004FF480521A8561E03268D1075CBF43F0AD
:1036680001032B70184B1B781F075EBF2B7823F0C4
:1036780001032B70D60242BF2B7823F001032B7075
:103688001C4B1A88174B1AB11B4A1268900702D4B0
:103698001A4A1288A2B302221A702B7823F0010367
:1036A8002B7032E090100020F0260020C81800206F
:1036B800D4180020102700203E130020407E05006B
:1036C800D8180020DC100020E0180020E6180020A0
:1036D80078230020141A0020942600200C1A0020B9
:1036E800081A0020E02600204C260020101A00208E
:1036F80000040048CA0A0020DC180020082700201F
:103708002978C90758BF02221A7008F049FCB64B3D
:103718001B68C01A002801DB0BF0EEFFB34F09F05D
:103728005FFB3E78002E00F0AF80B14E3368002B6F
:1037380000F09286306808F082FC002800F08C8641
:10374800AB4BAC4C186808F077FC092801D03F282F
:1037580054D14FF0000AD4F80090A74DD046B9F1E3
:10376800000F05D0A54829684A460EF043FF20B946
:10377800AA46B8F1000F00D1A846A14B10359D42CA
:10378800EDD3B8F1000F18D0D8F800E0DAF800C08F
:1037980023681EF803501CF80300A8420DD15A1CD8
:1037A800964938B92D2B05D8924D2A602025CD543D
:1037B800885402E0CD542260EAE723680BB1D04573
:1037C80011D090480AF080F9D04507D858F8100B66
:1037D8000AF07AF909200AF06FF9F5E78A480AF041
:1037E80073F94FF0000923689945A3D2834B13F866
:1037F80009000AF061F909F10109F4E72368002BCF
:1038080040F00F86042840F04A867C4804F05CFFAC
:1038180000F022BED9F80000DFF8F8A108F00FFC8C
:1038280040B3DAF8000008F007FCDBF8003093F842
:1038380048100246002937D124286ED1012283F886
:103848004820DBF80030DFF8ECA193F84820062A7E
:10385800E0D193F8490000F0B1FE002800F086801E
:10386800D8F8003098790AF078F8D8F800300022B3
:1038780083F84820654B93F83730002B40F0BF851C
:103888004C36982E00F0E885614BF21892F84A10F1
:103898000129F5D1DFF89C81F358C8F800205D4A6A
:1038A800C34613609146B5E7012904D14D2814BFDA
:1038B80000220222C3E7022904D13C2814BF0022B7
:1038C8000322BCE703290CD140284FF0000102D99C
:1038D80083F84810B5E758711971D97198710422A5
:1038E800ADE7042906D1997983F849004A409A71CD
:1038F8000522A4E70529A4D158791979884298792D
:1039080006D950409871481C18710B441A7298E7F0
:1039180090420CBF0622002291E72B783E495807B7
:103928008FD4232ADAF8003013D1012038703048B8
:103938000491036035480392036338480AF0C4F8D9
:1039480031480AF0C1F80499039A0B7843F002034E
:103958000B70334B1B681B78934201BF314B324AC3
:103968001A60324B04BF324ADA606AE7DAF800209C
:1039780092F849304E2B00F0C38400F29C80372B1C
:1039880000F0FC8421D8292B00F0698409D8252B64
:1039980000F04084272B00F04484232B40F07B85E3
:1039A80029E22D2B00F06C8407D82B2B40F073856F
:1039B80009F0B6FF607100F01DBD332B00F0CC8418
:1039C800352B00F0538200F066BD412B00F0C9840E
:1039D80032D83C2B00F000813E2B00F0EE80392BD2
:1039E80040F0598500F02ABCE42600201127002069
:1039F80068230020FC1C0020D8440108CC1C0020AF
:103A0800684601083C6101084161010890100020E6
:103A1800FC2300208819002010270020716101086C
:103A2800A0240020FC9F0020EFBEADDE00ED00E0EA
:103A38000400FA0584190020442B00F0D78426D806
:103A4800432B40F0288509F06BFF0023A3606071C9
:103A580009F07AFFA3681843A06009F061FF84F8B1
:103A6800920109F067FFA4F85C0109F063FFA4F86C
:103A78005E0109F05FFFA4F8600109F05BFFA4F89C
:103A8800820109F057FFA4F8840100F0B3BC4A2B67
:103A980000F09D804C2B40F0FE8409F041FF84F833
:103AA800D80109F03DFF84F8D90109F043FFA4F8D3
:103AB800DA0100F09FBCD12B00F06D831AD8CC2B13
:103AC80000F0128209D8C92B00F03E83CA2B00F0FF
:103AD8009180C82B40F0DF8442E0CE2B00F0278392
:103AE800C0F01C83CF2B00F05382D02B00F00B8347
:103AF80000F0D1BCD62B00F0848207D8D32B29D074
:103B080015D3D42B00F0898200F0C5BCEF2B44D02C
:103B180005D8D82B40F0BF844FF0000AFDE0F22B07
:103B280000F0C982FA2B00F00B8300F0B4BC2B78AC
:103B380003F0040303F0FF09002B40F05B8409F055
:103B4800EFFE022884F8E80640F2E382DB4B83F8B4
:103B5800E896DEE209F0EEFED94B988600F04ABC02
:103B680092F805904FEA5909B9F1120F03D90AF0F2
:103B7800B1FF00F03FBC4FF0000ACA4507D209F078
:103B8800D9FED04B23F81A000AF1010AF5E7CC4B0D
:103B9800012283F8362000F02DBCDFF82C93D9F8E9
:103BA80000A009F0C7FEAAF85A00D9F8009009F059
:103BB800C1FEA9F8580000F01DBC09F0B1FE84F858
:103BC800E20109F0ADFE84F8E10100F013BC09F050
:103BD800B1FEA08100F00EBCDFF8EC92D9F800A08D
:103BE80009F09EFE8AF80000D9F80030187808F02D
:103BF80067FCFFE3B44B1A681278022A4FF0000AF8
:103C080099466FD1D9F800B009F08AFE07EE900AFC
:103C1800F8EE677AB2EE048AC7EE887A0BEB8A0B65
:103C2800CBED087AD9F800B009F07AFE07EE900AD1
:103C38009FEDA67AF8EE677A0BEB8A0BC7EE877AC8
:103C4800CBED0B7AD9F800B009F06AFE07EE900ABE
:103C58009FED9F7AF8EE677A0BEB8A0BC7EE877AAF
:103C68000AF1010ABAF1030FCBED0E7ACAD1BAF103
:103C7800070FD9F800B01CD109F052FE07EE900AE0
:103C8800F8EE677AC7EE887ACBED117AD9F800B0EA
:103C980009F046FE07EE900AF8EE677AC7EE887AD2
:103CA800CBED127AD9F800B009F03AFE8BF84C0047
:103CB80012E009F035FED3448BF80100D9F800B0C2
:103CC80009F02EFED3448BF80B00D9F800B009F0A8
:103CD80027FED3448BF815000AF1010ABAF10A0F3E
:103CE800C5D187E3D9F800B009F01AFED3448BF8A0
:103CF8000100D9F800B009F013FED3448BF80B008B
:103D0800D9F800B009F00CFED3440AF1010ABAF15F
:103D18000A0F8BF81500E5D16CE3DFF8AC919FED45
:103D28006C8AD9F800B009F005FE07EE900AF8EEA3
:103D3800677A0BEB8A0BC7EE887ACBED087AD9F84D
:103D480000B009F0F7FD07EE900AF8EE677A0BEB82
:103D58008A0BC7EE887ACBED0B7AD9F800B009F058
:103D6800E9FD07EE900AF8EE677A0BEB8A0BC7EECF
:103D7800887A0AF1010ABAF1030FCBED0E7ACCD199
:103D8800BAF1070FD9F800B01CD109F0D3FD07EE3E
:103D9800900AF8EE677AC7EE887ACBED117AD9F8EF
:103DA80000B009F0C7FD07EE900AF8EE677AC7EE93
:103DB800887ACBED127AD9F800B009F0BBFD8BF800
:103DC8004C0012E009F0B6FDD3448BF80100D9F895
:103DD80000B009F0AFFDD3448BF80B00D9F800B060
:103DE80009F0A8FDD3448BF815000AF1010ABAF1CD
:103DF8000A0FC5D1FEE209F093FD132883463FF66A
:103E0800B6AEDFF8C4A0DAF8009009F089FD002307
:103E1800304A0C2101FB0322117A814222D10FFA88
:103E28008BFB09EB8B09137889F8793009F078FD59
:103E380089F87A0009F074FD89F87B0009F070FDB3
:103E4800254B264A1A6089F87C00254BDAF80000D1
:103E580018600021793002F009FD224B80F0010042
:103E68001870C7E201331C2BD2D180E609F058FD47
:103E78000B2882463FF67BAE134BD3F8009009F02F
:103E88004FFD03283FF673AE062303FB0A9989F812
:103E9800CE0009F045FD89F8C90009F041FD89F80F
:103EA800CA0009F03DFD89F8CB0009F039FD89F811
:103EB800CC0009F035FD89F8CD009BE2B411002053
:103EC80090100020101B0020141100200000C84290
:103ED80000007A443C430108040B0020F81200203B
:103EE800080B0020100000205379092B7FF63FAE05
:103EF800019BD3F8009009F013FD019B89F800009D
:103F0800D3F8009009F00CFD89F8010009F008FDCC
:103F1800019B64281B68A8BF6420187109F000FD84
:103F2800019B64281B68A8BF6420587109F0F8FC3D
:103F3800019BFF281B68A8BFFF20987109F0F0FCBF
:103F4800019B6428D3F8009028BF642089F80700F3
:103F580009F0E6FC019B89F80200D3F8009009F00B
:103F6800DFFC019B89F80300D3F8009009F0E2FC1C
:103F7800DAF80030A9F80A005B790A2B40F23A8295
:103F8800D14BD3F8009009F0CBFC89F8080031E256
:103F980009F0D0FC6FF4AF6283189BB2C62B98BFB0
:103FA800A4F8980109F0C6FCA4F8440109F0C2FC81
:103FB800A4F8460109F0BEFCA4F8480109F0BAFCCF
:103FC800A4F8DA0109F0ACFC84F8EF0109F0A8FCC8
:103FD80009F0A6FC84F8F00109F0A2FC84F8870136
:103FE80009F09EFC84F8940109F09AFCB74BD3F8C9
:103FF800009009F09FFC00EB80004000A9F85600F3
:104008001CE1814609F096FCB14B23F8190009F12F
:104018000109B9F1080FF5D1ECE153790F2B7FF4C1
:10402800A6AD09F07DFC072881463FF6A0AD029BAE
:10403800D3F800A009F07EFC0E2303FB09F9CA445B
:10404800029BAAF81901D3F800A009F073FCCA442E
:10405800029BAAF81B01D3F800A009F06BFCCA4424
:10406800029BAAF81D01D3F800A009F059FCCA4424
:10407800029B8AF81F01D3F800A009F051FCCA443A
:10408800029B8AF82001D3F800A009F049FCCA4431
:10409800029B8AF82101D3F800A009F041FCCA4428
:1040A800029B8AF82201D3F800A009F04DFCD14404
:1040B800C9F823019EE109F033FC0F2881463FF639
:1040C80056AD09F02DFCC9EBC909A14489F8D40003
:1040D80009F026FC89F8D50009F022FC89F8D600F9
:1040E80009F01EFC89F8D70009F01AFC89F8D800F5
:1040F80009F016FC89F8D90009F012FC89F8DA00F1
:1041080008F040F976E12B785B0700F1738109F03C
:1041180015FF03F035FF03F0F1FF6BE12B7858072B
:1041280000F168816B4B4FF4C8721A8062E12B78FA
:10413800590700F15F81684A137843F0040328E0C7
:104148002B785A07E5D5A6E109F0EAFB624B1A7805
:1041580010B142F0020201E022F002021A7009F0E6
:10416800DFFB5E4BDFF89491187009F0EDFBC9F89E
:10417800000009F0E9FBC9F8040009F0DBFB584B23
:10418800188009F0D7FB574B574A1880137843F02B
:10419800020313702EE109F0C3FB039009F0D4FB6E
:1041A800834609F0D1FB824609F0CEFB814609F02F
:1041B800C1FB09F0BFFB09F0B3FB039BA3B94B4B51
:1041C8001020C3F800B0C3F804A003F086FE424AEA
:1041D800137843F001031370B9F1000F00F00A815E
:1041E800434BC3F8009005E1102B40F00381414B8D
:1041F800C3F800B0C3F804A0B9F1000F02D03C4BDB
:10420800C3F800903B483C4B0222011D1A7007F08E
:1042180049F8EFE0A06009F097FBA3681843A06095
:10422800E8E009F087FBA4F85C0109F083FBA4F837
:104238005E0109F07FFBA4F86001DBE009F070FB88
:1042480084F87C0109F06CFB84F8800109F068FBB4
:1042580084F87F0109F064FB84F88101CAE009F061
:1042680069FBA4F8820109F065FBA4F8840109F050
:1042780057FB84F8860109F05DFBA4F88801B9E0D2
:1042880009F04EFB84F8920109F054FBA4F89C0154
:1042980009F050FBA4F8980109F04CFBA4F89A0126
:1042A80009F03EFBDAF8003084F893015B79082BBB
:1042B80040F2A08009F03EFBA4F89E0109F03AFB09
:1042C800A4F8A00196E000BF3411002014110020CA
:1042D8004E230020CA0A0020E0180020E61800201B
:1042E800E4180020E21800203A1100203C110020B8
:1042F8004C110020441100200C0B0020E81800206D
:1043080092F805A00323BAFBF3FABAF1120F3FF6AD
:104318002EACDFF8A4B28146D1456BD209F000FB80
:104328008BF8A20109F006FB40F2ED23984205DD67
:1043380040F6CA039842A8BF184601E040F2EE20B2
:10434800A0F2EE20192309F1010990FBF3F00BF11B
:10435800020B8BF8A101DFE709F0E2FA84F8940177
:1043680048E0814609F0DCFA04EB090309F1010988
:10437800B9F1080F83F88A01F4D13BE053794FF083
:10438800070AB3FBFAFACAEBCA029B1A13F0FF0F2B
:104398007FF4EDAB5FFA8AFA0AF1FF3A5FFA8AFA1C
:1043A800BAF1FF0F26D009F0BBFA5FFA80FB4FFA8B
:1043B8008BF002F0E1F8814600283FF4D8AB80F892
:1043C80000B009F0B7FAA9F8020009F0A9FA89F8CB
:1043D800040009F0A5FA89F8050009F0A1FA89F89E
:1043E800070009F09DFA89F80600D5E7604B01221D
:1043F80083F83720002009F0DFFAFFF731BA5D4B68
:10440800985907F013FE18B9322007F0F0FDF6E7C7
:1044180007F078FF03F08AFD574B584ADA60FFF738
:104428002FBA0C283DD00A283FD1554D554809F0E0
:104438004BFB284623210EF0C6F808B1401B20602C
:104448002368002B34D14E482360002130220EF01F
:1044580084F83B78002B5FD14B4B1B689B060FD52C
:104468004A4B43491B688A6B9A1A002A08DB484A58
:104478001278042A82BF03F5123303F5F8738B63AD
:10448800444B9B68002B6ED0434807B0BDEC028BB1
:10449800BDE8F04F18470AF01DFBFFF7E1B90C28FB
:1044A80048D13E4809F010FB36E00D2836D1BCE76C
:1044B8005A1EA95C202901D11346C2E7304A23605D
:1044C8000021D154364B374DD3F800A0D5F800B0B1
:1044D800DFF8AC9058460EF084F8804642464846CD
:1044E80059460EF087F8304A28B919F8083053446D
:1044F8005B785B0703D010359542E7D307E0954218
:1045080005D208F10100EB684844984702E02748C3
:1045180009F0DAFA002396E7254807E07F280DD14D
:10452800013B174A234823600021D15409F0CCFAF3
:10453800FFF700B97F2804D1FFF7FCB82F2B3FF60F
:10454800F9A8A0F12002D2B25E2A3FF6F3A813B967
:1045580020283FF4EFA85A1C2260094AD05409F0D9
:10456800ABFAFFF7E7B807B0BDEC028BBDE8F08FF8
:1045780090100020FC23002000ED00E00400FA0564
:10458800CC1C00206D6C0108DC180020F0260020EF
:10459800E61800205C1D0020AA11002046610108D1
:1045A8000C010020D844010868460108516101083F
:1045B800416101086D610108B41100202DE9F0473F
:1045C80064282DED028B044600F0868100F29C8061
:1045D800342800F0778451D8222800F0518423D859
:1045E800032800F0458114D8012800F035810228FD
:1045F80040F0BA86042009F0DFF9432009F0ADF94C
:104608004C2009F0AAF9462009F0A7F94C2000F03F
:1046180023BE042800F03681052840F0A5861A201C
:1046280009F0CAF900243EE1282800F0AE8515D823
:10463800242800F09585262840F09686AE4C062062
:1046480009F0BAF9B4F85C0109F0B9F9B4F85E01F7
:1046580009F0B5F9B4F8600100F02FBE2C2800F07D
:10466800A785322800F0F2852A2840F07D860120AF
:1046780009F0A2F9A04B587900F0EEBD402800F0EF
:10468800EE8521D83A2800F08E820BD8362800F023
:104698003386382840F06886042009F08DF9964C56
:1046A80000F064BD3B2800F0E4833D2840F05C86C0
:1046B800914C022009F080F994F8E20109F04DF9D3
:1046C80094F8E10100F0C8BD462800F034860BD804
:1046D800422800F0D285452840F04686132009F08C
:1046E8006BF9002400F031BE4B2800F080854D287E
:1046F80000F08C85492840F03786022009F05CF9E3
:104708007D4B988900F0D9BD722800F05A8455D89D
:104718006A2800F09A842FD8672800F0B7811CD83F
:10472800652800F00181662840F01E86734C12202F
:1047380009F042F9208809F042F9608809F03FF948
:10474800A0886F4C09F03BF9A08D09F038F9E08D8D
:1047580009F035F9208E00F0F9BC682800F00582D0
:10476800692840F00186674D2878400000F0FE0077
:1047780009F022F9002404E26D2800F00D8213D814
:104788006B2800F082846C2840F0EE855E4C062091
:1047980009F012F9208809F012F9608809F00FF978
:1047A8005A4B188800F089BD6F2800F04982C0F084
:1047B800FE81702800F06E8200F0D6BD782800F0E7
:1047C800728119D8752800F0488309D8732800F039
:1047D8003184742840F0C8854FF0000801269EE314
:1047E800762800F06384772840F0BE85444D287C05
:1047F80009F0E2F80024DCE3A42800F07C8414D853
:104808007B2800F0D082A02840F0AE850C2009F06B
:10481800D3F83F4B186809F0DBF83E4B186809F0ED
:10482800D7F83D4B186800F09BBDF12800F0778160
:10483800FE2800F08784F02840F09685304C04204C
:1048480009F0BAF8636CB3F85A0009F0B8F8636C69
:10485800B3F8580000F031BD032009F0ADF800208E
:1048680009F07BF8204609F078F80D2000F0F4BC38
:1048780009F0A2F8012009F070F80A2009F06DF893
:1048880000F037BC062009F097F8412009F065F8D8
:10489800462009F062F8462009F05FF8332009F055
:1048A8005CF800F05BBC1D4B185D013409F055F84D
:1048B8000B2CF8D100241A4B185D013409F04DF87F
:1048C800082CF8D10024174B185D013409F045F87D
:1048D800072CF8D100F046BD072009F06DF8E72055
:1048E80009F03BF8044B587909F037F8002009F033
:1048F80034F8042000F034BDB4110020A2110020C7
:10490800D01000209824002066260020A81100203E
:10491800ACF7FF1FB0F7FF1FB4F7FF1FA25D010838
:10492800AE5D0108835D0108B84C0B2009F044F81E
:10493800208809F044F86268B54B9A420CBF208978
:10494800608980B209F03BF8B24B1B68C3F3C00022
:10495800C3F38002800040EA4200C3F340021043E0
:10496800C3F3401240EAC20003F01003184309F0F1
:1049780026F8A94B1A88E368247C02F0080103F49E
:10498800475949EA010903F4804149EA010903F456
:10499800004149EA010903F4803149EA010903F4B5
:1049A800003149EA010903F4802149EA010903F4C5
:1049B800002149EA010903F4801149EA010903F0D9
:1049C800007349EA0303DFF8749299F8009012F033
:1049D800010FC9F3800914BF4FF002084FF0000817
:1049E80043EA090312F0020F43EA080314BF4FF029
:1049F800040C4FF0000C12F0040F43EA0C0C14BF27
:104A08004FF0100E4FF0000E12F0400F14BF202789
:104A180000274CEA0E0E12F0100F14BF4FF4007668
:104A280000264EEA070712F0200F14BF4FF48065E6
:104A380000253E4312F4807F14BF4FF4006000202D
:104A4800354312F4007F14BF4FF4001100212843AE
:104A580012F4806F41EA000114BF4FF08063002315
:104A6800002019430346A3420AD26C4A9D5C0122E6
:104A780002FA05F50D421CBF9A4010430133F2E7D4
:104A880008F0A6FF664B93F8E806E5E3102008F067
:104A980093FF0024634B185D013408F05EFF102C6F
:104AA800F8D100F05FBC702008F086FF0026574D53
:104AB8000E246B6C744323440136B3F8190108F0D3
:104AC8007EFF6B6C2344B3F81B0108F078FF6B6C16
:104AD8002344B3F81D0108F072FF6B6C234493F86C
:104AE8001F0108F03AFF6B6C234493F8200108F08B
:104AF80034FF6B6C234493F8210108F02EFF6B6C94
:104B0800234493F8220108F028FF6B6C1C44D4F866
:104B1800230108F05DFF082EC9D100F023BC7020E6
:104B28003F4C08F049FF04F1700594F8D40008F0F0
:104B380014FF94F8D50008F010FF94F8D60008F098
:104B48000CFF94F8D70008F008FF94F8D80008F094
:104B580004FF94F8D90008F000FF073494F8D30054
:104B680008F0FBFEAC42E0D1FCE3102008F024FF83
:104B780000242D4B185D013408F0EFFE102CF8D1FD
:104B8800F0E32B789C4280F0ED83284B33F8140037
:104B980008F015FF0134F4E7062008F00DFF0020A7
:104BA80008F016FFDAE2042008F006FFD7E3072032
:104BB80008F002FF1E4B1888FF28A8BFFF20C0B2CC
:104BC80008F0CBFE1B4B18684FF6FF74A042A8BF35
:104BD800204620EAE07080B208F0F1FE0B4BB3F8F3
:104BE800600008F0ECFE0E4B93F88721124B186812
:104BF8003AB10A235843A042A8BF204620EAE070F1
:104C080001E000F30F0080B257E300BFD01000208E
:104C180000540040DC180020A4190020E1100020F6
:104C2800B41100200211002018110020101B0020D0
:104C3800CC180020D8180020D418002010270020F5
:104C4800C64C0B2008F0B8FE636E187808F085FE95
:104C5800636E587808F081FE002625466B6EBF4CBF
:104C680033440136187908F078FE032EF6D1636EC6
:104C7800D87908F072FE636E987808F06EFE636E5D
:104C8800D87808F06AFE636E588908F098FE636E5B
:104C9800187AE1E2B14C1E2008F08EFE636C1B7896
:104CA800022B4FF000056BD1636C03EB850393ED8A
:104CB800080AB2EE048A20EE080A0DF05DFE80F3C1
:104CC8000800C0B208F049FE636CDFEDA57A03EB7B
:104CD800850393ED0B0A20EE270A0DF04DFE80F3B5
:104CE8000800C0B208F039FE636CDFED9E7A03EB72
:104CF800850393ED0E0A20EE270A0DF03DFE80F3A2
:104D08000800C0B2013508F028FE032DCCD1072DCC
:104D1800636C23D193ED110A20EE080A0DF02CFEE6
:104D280080F30800C0B208F018FE636C93ED120A15
:104D380020EE080A0DF020FE80F30800C0B208F04B
:104D48000CFE636C93F84C3000EE103AB8EE400A53
:104D58000DF012FE80F30800C0B20BE02B44587827
:104D680008F0FBFD636C2B44D87A08F0F6FD636C01
:104D78002B44587D013508F0F0FD0A2DC7D1F1E22A
:104D8800636C2B44587808F0E8FD636C2B44D87AA0
:104D980008F0E3FD636C2B440135587D08F0DDFD18
:104DA8000A2DEDD1DEE23C2008F006FE00246B4D12
:104DB8009FED6C8A6B6C03EB840393ED080A20EE7D
:104DC800080A0DF0D9FD80B208F0F9FD6B6C03EB11
:104DD800840393ED0B0A20EE080A0DF0CDFD80B296
:104DE80008F0EDFD6B6C03EB840393ED0E0A20EEE7
:104DF800080A0DF0C1FD013480B208F0E0FD032C73
:104E0800D5D1072C6B6C16D193ED110A20EE080A48
:104E18000DF0B2FD80B208F0D2FD6B6C93ED120A72
:104E280020EE080A0DF0A8FD80B208F0C8FD6B6CF2
:104E380093F84C000BE02344587808F0C0FD6B6CE5
:104E48002344D87A08F0BBFD6B6C2344587D0134A9
:104E580008F0B5FD0A2CD4D184E22F2008F0ACFD6F
:104E6800414C14F8010F002800F07C8208F075FD11
:104E7800F7E7012008F0A0FD384B5B6C1878EBE1F0
:104E8800502008F099FD0025344B5C6C374B04EB3F
:104E980085040C2194F8792001FB0233013593F83D
:104EA800380008F05AFD94F87A0008F056FD94F896
:104EB8007B0008F052FD94F87C0008F04EFD142D9C
:104EC800E2D14FE2482008F077FD0025234B5C6CC7
:104ED800062303FB0544013594F8CE0008F03DFD98
:104EE80094F8C90008F039FD94F8CA0008F035FDB7
:104EF80094F8CB0008F031FD94F8CC0008F02DFDB3
:104F080094F8CD0008F029FD0C2DDFD12AE2002EFF
:104F180000F028825FFA88F008F04EFD002600278E
:104F28000E4B1A7C9742F2DA11330024FA5C0F4DCB
:104F38000C2305F130016343595C914207D12B449E
:104F4800586B0DF04EFB82462EB9B14610E0013485
:104F58001C2CECD119E0804417E000BFD0100020D1
:104F68000000C84200007A440B4301080C430108C2
:104F7800D1450ADA0C2303FB04535B6B13F80900D1
:104F880008F0EBFC09F10109F2E70137C8E7013144
:104F98001C290DD0CA480C2200F1300702FB01F38E
:104FA800DA5DB242F3D1034493F8380008F0D5FC37
:104FB80001342B7C9C4280F0D581C24B0021E65CF9
:104FC800E8E7C14C162008F0F7FCB4F8980108F09F
:104FD800F6FCB4F8440108F0F2FCB4F8460108F015
:104FE800EEFCB4F8480108F0EAFCB4F8DA0108F07D
:104FF800E6FC94F8EF0108F0B0FC002008F0ADFCE6
:1050080094F8F00108F0A9FC94F8870108F0A5FCD1
:1050180094F8940108F0A1FC002008F09EFCAB4B2A
:105028005B6C0A20B3F9563093FBF0F080B208F0BD
:10503800C6FC9BE0082008F0BFFC0124E0B2013464
:1050480008F08BFC092CF9D18CE1102008F0B4FC95
:105058009F4BA04C187800F0020008F07EFC9E4B95
:10506800187808F07AFC206808F0B2FC606808F04C
:10507800AFFC9A4B188808F0A2FC994B188808F0E6
:105088009EFC924BB3F8680017E1052008F094FCE9
:10509800944B188808F093FC934B188808F08FFC01
:1050A8008A4B93F86A0000F00100D5E008F038FC5C
:1050B8000746122008F080FC844C17B9E66E256F6D
:1050C80005E0102F13BF0025666FA56F2E463846E2
:1050D80008F043FC304608F07BFC284608F078FCD2
:1050E800E06F08F075FC002008F069FC002008F06B
:1050F80066FC0020B0E0754D95F880008000013016
:10510800C0B208F059FC95F8800008F026FC00248D
:105118002E4696F880309C4280F02481734D285D9D
:1051280008F01BFC05F11003185D08F016FC05F1EA
:1051380020033035185D08F010FC285D08F00DFCE0
:105148000134E6E7082008F037FC002008F037FCB7
:10515800002008F034FC002008F031FC0020ACE00E
:10516800042008F029FC584B9868F9E094F87C0171
:1051780008F0F3FB94F8800108F0EFFB94F87F0146
:1051880008F0EBFB94F8810166E04F4C072008F02B
:1051980013FCB4F8820108F012FCB4F8840108F09A
:1051A8000EFC94F8860108F0D8FBB4F8880184E076
:1051B800454C0C2008F000FC94F8920108F0CDFB57
:1051C800B4F89C0108F0FBFBB4F8980108F0F7FB71
:1051D800B4F89A0108F0F3FB94F8930108F0BDFBCA
:1051E800B4F89E0108F0EBFBB4F8A00165E0364C7A
:1051F800042008F0E1FB94F8D80108F0AEFB94F81D
:10520800D90108F0AAFBB4F8DA0156E0384C394D58
:10521800207800EB4000C0B208F0CEFB00262378CF
:105228009E4205F1020580F09D8015F8020C08F0F9
:1052380094FB15F8010C00EB800000EB800000F2F5
:10524800EE2080B208F0BBFB0136E8E7012008F049
:10525800B3FB1D4B93F8940108F07FFB82E0082014
:1052680008F0AAFB0024184B2344013493F88A0160
:1052780008F073FB082CF6D174E0134C102008F0EA
:105288009BFB607908F069FBA06808F0A1FB94F823
:10529800920108F062FBB4F85C0108F090FBB4F8E6
:1052A8005E0108F08CFBB4F8600108F088FBB4F8E4
:1052B800820108F084FBB4F8840108F080FB51E017
:1052C8000C430108E1100020B4110020D010002088
:1052D800E0180020E8180020E6180020E418002054
:1052E800E21800205A1900205C19002051110020F2
:1052F80098240020561300202A4B2B4C93F8C10009
:10530800C0EBC000C0B208F057FB04F11805274AEB
:1053180094F8F60192F9001043B2994226D092F916
:105328000C10994222D092F918209A421ED00834C3
:10533800AC42ECD116E00D2008F03EFB002008F04E
:105348000CFB002008F044FB06E0194B185D013403
:1053580008F003FB0B2CF8D1002008F039FB0020E3
:1053680008F036FB012018E0002016E008F0F5FAF6
:10537800B4F8F80108F023FB94F8FA0108F0EDFA04
:1053880094F8FB0108F0E9FA94F8FD0108F0E5FA51
:1053980094F8FC0108F0E1FAC9E7BDEC028BBDE81E
:1053A800F08700BFD0100020B4110020A4240020F2
:1053B800A25D01082DE9F047D44CD54E237886B07C
:1053C8000746002B00F0FE8132686368D31A7C2BF5
:1053D80040F2F881237A626001332372002505F1D7
:1053E8002400DFF82883C0B207F0EAFC08F10A03BA
:1053F8009FEDC87A33F9153007EE903AFAEECC7A79
:10540800013567EE877AFDEEE77ACDED037ABDF9CF
:105418000C0007F0C3FC032DE1D1302007F0D0FCCD
:10542800002007F0BBFC07F0C3FC98F8085015F003
:10543800030520D1D8F8042041F288339A420BD9C9
:10544800102007F0BDFC284607F0A8FC212007F033
:10545800B7FC284607F0A2FC142007F0B1FCB4F909
:10546800100007F09BFC1C2007F0AAFC002007F0A6
:1054780095FC07F09DFC237ADFF890825B0740F0EB
:105488007E81022007F09CFC0A23B8F9120090FBE9
:10549800F3F007F083FC0320B8F91A50DFF8909274
:1054A80007F08EFC9C4B1B7813F0040F4FF0050A95
:1054B80095FBFAF5ADB20DD008F5D370394601F079
:1054C800E6F928B9D9F8003013F0100F18BF0025F5
:1054D80028B205E0D8F830379889B0FBFAF000B266
:1054E80007F05CFCD9F800309F0740F18A80DFF8AC
:1054F8004492B4F8367799F80030B4F83427834DDD
:105508003F014FF06408BFB208FB02325B00B2FBF8
:10551800F3F347EA0327BFB2C3F303231F4306206D
:1055280007F04EFC38B207F039FCB4F8363799F872
:10553800001001339BB293FBF1F201FB1233A4F884
:105548003637D4F838379B7B012B05D1392007F043
:1055580037FCB5F934071AE0B5F834576E233A200A
:105568005D43152707F02CFC95FBF7F5AFB2B7FBA9
:10557800F8F528B207F012FC08FB15753B2007F078
:105588001FFCA8B2451D0A2095FBF0F000B207F0F9
:1055980005FC282007F014FCD4F83C375B4D0A20A2
:1055A80093FBF0F000B207F0F9FB042007F008FCC9
:1055B800D4F83037D5F840079A894FF6FF739842E8
:1055C800A8BF1846C2B10028ACBF131A134607EE8D
:1055D800903A9FED527AF8EEE77A67EE877A07EE0F
:1055E800102AB8EEC77AC7EE877AFDEEE77A17EE8B
:1055F800900A6428A8BF642020EAE07000B207F08F
:10560800CDFBD4F84437414F9D0640F1AD8097F863
:10561800483798071DD5112007F0D2FBB7F84A077D
:105628003F4B4FF4F365684390FBF3F000B207F08B
:10563800B5FB192007F0C4FBB7F84A0745436420B7
:1056480095FBF0F595FBF0F300FB135000B207F063
:10565800A5FB94F84837B4F84C5713F0020F08BF6D
:105668000025012007F0ACFB28B207F097FB0920C2
:1056780007F0A6FB002007F091FB2A4B94F84E5741
:105688001A88B2F5967F0AD9204B1B7A03F00F03CC
:10569800072B04D842F20F75954228BF15460520FE
:1056A80007F08EFBD4F838375B7B0BB928B21CE0C7
:1056B800A5F1200307EE903A9FED1B7AF8EEE77A02
:1056C800F6EE006AC7EE877ABEEE007AF5EEC07A8B
:1056D800F1EE10FA58BFB0EE667A77EE877AFDEEF3
:1056E800E77ACDED037ABDF90C0007F057FB94F883
:1056F8004827064B910703D493F84F27012A1DD159
:10570800012384F84F37094835E000BF981100207D
:105718009426002000007A44102700200000C84288
:10572800A0860100FE0000206666E63FE81800201B
:1057380070260020FC0000208096184BD3F83837DC
:105748005FED036A93ED017AD3ED027A27EE267AAC
:1057580067EEA67ABDEEC77AFDEEE77A8DED047A9C
:10576800CDED057A04A806E0B74A92E8030004AB39
:1057780083E80300184604F04DFA07F019FB237A72
:10578800282B1FD1B14B00221A723C2733684FF4E3
:105798007A70B3FBF0F8172007F012FBB8FBF7F5A7
:1057A800B5FBF7F007FB1050000200B207F0F6FA5D
:1057B800182007F005FB07FB158000B207F0EEFA8A
:1057C80007F0F6FA94F85837A04D002B00F05D81E9
:1057D80006F0E6FBD5F85C379D4AC31A93420746A4
:1057E80040F2C680002385F8623785F86437B5F83B
:1057F8003437DAB21B0A85F87E2785F87F3785F8B3
:10580800742785F87537D5F88C2733689A1AD5F830
:105818009037D97B4FF47A734B439A420ED38D4B12
:105828001B68C5F88C3795F89437013B012B9FBF4F
:10583800102385F86237022385F864370A20D4F8E4
:105848003C2792FBF0F284F87C27121284F87D271B
:1058580094F84827D4F8403793FBF0F384F880375E
:105868001B1284F88137920794F84E37774984F8E9
:10587800AF3703D42D2381F8B03777E0042BD4F861
:105888005097D4F85467DFF8DC81734A8CBF332310
:10589800322381F8B0374FF0060C704B99FBF3F0C8
:1058A80096FBF3F308FB009108FB036803EB830303
:1058B8000CFB01F103EB830391FBF2FE642502FB71
:1058C8001E119B0091FBF5F184F8A11709120CFB3E
:1058D80008FC84F8A2179CFBF2F143FA81F39BB20F
:1058E80002FB11C292FBF5F284F8A627121284F883
:1058F800A43784F8A7271B0AB4F84A2784F8A537E1
:105908002423534393FBF5F5B4F8C23784F8A8373A
:1059180000EB80001B0A00EB8000800084F8A937A8
:105928000A22B4F84C37B3FBF2F303F5FA739BB2CF
:1059380040FA8EF080B284F8AA371B0A4FEAD97968
:1059480084F89F07F60F000A84F89C5784F8AB3751
:10595800C5F30725B4F8C43784F89E9784F8A007E0
:1059680084F8A36784F89D5784F8B137C4F85C7746
:1059780094F8C687354DB8F1000F0DD1D5F8CC078E
:1059880006F05DFB012807D90228354E00F0538246
:1059980004F032F901233370D4F8D0272B4D002AB4
:1059A80073D095F8C6673EB1D5F8D83740F6B73109
:1059B800FB1A8B4219D868E00123D5F8CC0785F883
:1059C800C63700F07EFCD5F8DC3793F900000223D7
:1059D8008DE84800082132464FF4964300F08CFCCD
:1059E80085F8E067C5F8CC074DE095F8D467CEB9DF
:1059F800D5F8CC07C5F8D06785F8C66700F061FC14
:105A0800D5F8DC3793F9000001238DE84800082118
:105A180032464FF4964300F06FFCC5F8CC0704F00B
:105A2800EBF830E0013EF6B285F8D46795F8E01758
:105A380095F8E137C6B94A1C013385F8E02785F89F
:105A4800E137D5F8CC071CE09844010898110020EC
:105A58003F0D03009426002040420F0080969800D6
:105A680011000020806967FF12F8016BC5F8D02784
:105A7800701885F8E0070133D5F8CC0785F8E137C9
:105A8800314606F0DFFAC4F8D87794F8E2379D4D2E
:105A9800F3B1D5F8E437DBB1D5F8E837C3B1C5F8C9
:105AA800EC371B68984AC5F8F037D5F8F437134433
:105AB800187AFEF783FDD5F8EC37987907F04DFF93
:105AC800D5F8F4370133092B88BF0023C5F8F4371C
:105AD8008E4D94F8F8272E688A4B002A00F0E6814C
:105AE800D3F8FC27002A00F0E18193F80038013B45
:105AF800012B00F2DB81D4F8FC07824F06F09FFAF5
:105B0800E0B1D7F8FC0706F097FA97F80138D5F80E
:105B180000907E2B80460ED102231B2887F8003880
:105B280009D1D7F8FC0706F08AFA20B90123C7F88B
:105B3800049887F8083884F80188DCE7D7F804283F
:105B48002B689B1A41F6583293421ED9032387F8D3
:105B58000038ABE16E4A32F8130010B903464FF42F
:105B680003600133B0F5C06FDBB271D01ED9B0F558
:105B7800006F77D033D9B0F5036F40D184F8093876
:105B8800D4F844375F4F9A0640D494F8081894F82C
:105B98000938002900F04C812A68921B012AD9D9BA
:105BA80084F80938002384F808387FE1B0F5007FCD
:105BB80044D008D8B0F5807F00F08780B0F5887FA2
:105BC80000F08380E5E7B0F5806F00F0A580B0F5C0
:105BD800826F00F0EA80B0F5047FDAD123E0B0F5F7
:105BE800E26F00F08280B0F5E46F00F08380B0F5DA
:105BF800E06FCED184F80938B4F90A107EE0B0F528
:105C0800046F6BD0B0F5026FC3D1FAE097F848374C
:105C18009B07BAD5B7F84A1724234B43123364219C
:105C280093FBF1F1FEE084F809383A4B354F1B68D5
:105C38009907AAD5B7F834370A21F2E084F8093869
:105C4800344B304F1B681A059FD5D7F83C17E9E04D
:105C580084F809382F4B2B4F1B681B0595D5D7F8AF
:105C68004017DFE0D4F84417264A84F80938880634
:105C78008BD592F84817890787D5DB0712D5D2F854
:105C8800543783EAE371002BA1EBE37101EB510177
:105C98004FF01902B1FBF2F1ACBF41F0004141F005
:105CA80040410FE0D2F8503783EAE371A1EBE3718A
:105CB800002B01EB51014FF01902B1FBF2F1B8BF13
:105CC80041F080414FF400608AE084F80938D4F844
:105CD80044375F077FF559AF00215FE0B4F9101032
:105CE80084F80938642359437AE084F80938B4F908
:105CF8000C1003E0B4F90E1084F809382C2391FB3A
:105D0800F3F16DE0981100209844010894260020D2
:105D18008E6201087026002084F8093894F80A3841
:105D2800644A0133DBB2032B88BF012382F80A38A7
:105D380094F80A1842F2107359435F4B1B78D8073E
:105D480048BF01319A0748BF02315F07B4F80C38E1
:105D580048BF0431D80748BF0A319A0748BF1431F1
:105D68001F0648BF2831D80548BF28315A0748BF01
:105D780064311F0748BFC831980548BF01F5C8718D
:105D88009A0648BF01F57A71DF0648BF01F5FA6146
:105D9800580648BF01F57A614FF4806003F0F8FEB9
:105DA800444B002283F80828EFE6D4F84417DFF8BC
:105DB800048184F8093811F0200717D098F848278B
:105DC80012F0020F14BF4FF47A71002112F0010F84
:105DD80014BF4FF4FA6300230B4494F84E17194488
:105DE80003F0D6FE002384F80838CEE6334B1B6850
:105DF80019067FF5CAAE394603F0CAFE88F8087856
:105E0800C3E684F80938D4F844372A4F9A067FF550
:105E1800BCAE97F848379B077FF5B7AEB7F84C3755
:105E28006421594303F0B4FE002387F80838ACE630
:105E380084F809383AE0337823B1C5F8C87786F88A
:105E48000080A9E5D5F8C837FB1AB3F57A6FFFF4D7
:105E5800A3AD0123D5F8CC07337006F0EDF806465C
:105E6800D5F8CC0706F0E8F876067FF495AD8A28D1
:105E780002D08E280DD08FE5D5F8443799067FF5E6
:105E88008BAD95F8C637002B7FF486AD05F2957378
:105E980006E095F8C637002B7FF47EAD05F5EC6378
:105EA800C5F8D0372D2385F8D43775E506B0BDE899
:105EB800F08700BF981100201027002070260020CE
:105EC800F8B504460E4617460025204620210CF05A
:105ED8007AFB0446D0B1013420460CF0D9FBB0F56A
:105EE800617F05DB40F634039842A8BF184601E0FD
:105EF8004FF46170A0F56170192390FBF3F00DB9B0
:105F0800307000E070703B7801333B700DB90125AB
:105F1800DBE72046F8BD7FB504780646E4B9364B82
:105F28001B6803EB8403192193F87B0093F87C60CA
:105F380093F8792093F87A304FF4617511FB00508B
:105F480011FB0651009001912C482146013401F0C3
:105F580090FE142CE3D14CE00CF09AFB1328054674
:105F680041DC254B701C1C68202100238DF80F3064
:105F78000CF029FB1E35064670B1013630460CF090
:105F880087FB1A289FBF04EB850358709DF80F30D4
:105F9800013398BF8DF80F30304620210CF013FBE9
:105FA800064670B1013630460CF072FB0D289FBFD3
:105FB80004EB850398709DF80F30013398BF8DF876
:105FC8000F3004EB85043046E11C0DF10F02FFF79A
:105FD80077FF9DF80F30042B0BD0601C00210422A2
:105FE8000CF0BBFA05E0064806490022132301F02D
:105FF80040FE04B070BD00BF14110020AE6201085D
:10600800C3620108E2620108014807F05DBD00BFF4
:10601800E8620108F0B5047887B006461CBB524B0D
:106028001968062303FB0411192091F8CA5091F846
:10603800CB7091F8CE2091F8C9304FF4617610FBFF
:10604800056510FB07600095019091F8CC0002905F
:10605800C8314648497903912146013401F009FEC7
:106068000C2CDCD17DE00CF013FB0B28044672DC11
:106078003D4B701C1D68202100238DF817300CF053
:10608800A2FA064680B1013630460CF001FB03281F
:106098009FBF062303FB045383F8CE009DF81730F7
:1060A8009CBF01338DF81730304620210CF08BFA55
:1060B800074680B1013738460CF0EAFA0D289FBF31
:1060C800062303FB045383F8C9009DF817309CBFCF
:1060D80001338DF8173006266643A9193846CA31A8
:1060E8000DF11702FFF7ECFE20210CF06CFA0746C1
:1060F80070B1013738460CF0CBFA14289FBF9DF8D1
:1061080017307619013386F8CC0098BF8DF8173010
:10611800384620210CF057FA78B101300CF0B8FA63
:106128000D289FBF062303FB045383F8CD009DF879
:1061380017309CBF01338DF817309DF81730062BA8
:106148000FD0062202FB04500021C9300CF005FADA
:10615800FFF75AFF05E00648064900220B2301F025
:1061680088FD07B0F0BD00BF14110020F6620108D9
:10617800C3620108E26201082DE9F3470478064684
:106188004CB9204601A908F04FFC0134FFF7F4FF91
:10619800122CF6D17AE00CF07BFAC5B2112D6FD82B
:1061A8003C4C05F1D00704EB4703701C202193F801
:1061B8000280394E0CF007FA034630B9A8F1020202
:1061C800D2F1000848EB020845E000F1010A5978CD
:1061D80030460CF0F8F960B1032D8CBF032300237F
:1061E800801B334453FA80F090F80490B9F1030F00
:1061F80002D1FFF709FF49E0A9F10203D3F1000832
:1062080050464FF0200148EB03080CF0DCF9D8B1F8
:10621800B8F1000FEDD001300CF03AFA40F2ED235E
:1062280080B2984205DD40F6CA039842A8BF1846D6
:1062380001E040F2EE2004EB4703A0F2EE20192221
:1062480090FBF2F0D87002E0B8F1000FD1D104EB66
:10625800470383F8029004EB4704A378F25CB8F193
:10626800000F08D0E3780D48294640F2EE2419259E
:1062780005FB034308E02946094801F0FAFC05E05C
:10628800084809490022112301F0F3FC02B0BDE8D7
:10629800F08700BFB4110020B44401081663010858
:1062A80028630108C36201089B6E010810B5044603
:1062B800204605F0BBFE18B90A2005F098FEF7E75E
:1062C80010BD0C4B5A6882421A4607D01B6983429C
:1062D80006D0D36983420BD1022302E0002300E0F9
:1062E80001230021C1620C2000FB032319725960AD
:1062F800704700BFA42400202DE9F04F06468B48C4
:1063080090F9004087B0B44289469DF84450114640
:106318001A469DF840300AD090F90C40B44209D092
:1063280090F91840B4420CD14FF0020804E04FF045
:10633800000801E04FF001080C2404FB0800047A6F
:106348000CB10020EEE0012E00F0DA80142E05D00A
:10635800002E40F0E68000957548D3E0DFF814A2DF
:10636800DAF8183043F00103CAF81830DAF81430B4
:106378004FF0904543F40033CAF814300127032244
:106388004FF4805B04A94FF090408DF815200392DC
:10639800CDF810B08DF814708DF816708DF8174080
:1063A80001F0C8F8A5F828B0C82005F020FEC5F807
:1063B80018B0DAF81430039A43F40033CAF81430EA
:1063C80028464FF4C0534FF0020B04A904938DF8EC
:1063D80015208DF814B08DF816408DF8174001F08F
:1063E800A9F86B6A23F470436B626B6A43F46043E9
:1063F8006B626B6A23F470236B626B6A43F46023ED
:106408006B624C4B4C4D4FF480221A6002F1804273
:10641800A2F53F3212232B63082385F83530136821
:1064280085F8367023F480231360536823F480239F
:10643800536095F8343003F1804303F582331A68CA
:1064480042F480221A602A6B3C4B22F01F0002F0B3
:106458001F02C15807FA02F221EA0202C2502A6B4F
:10646800374922F01F0002F01F0250F801E007FA36
:1064780002F22EEA020242502A6B22F01F0102F0B9
:106488001F02C85807FA02F20243CA502D4B2E4A7F
:106498001C60DAF81C3043F40003CAF81C302B4B9C
:1064A80004A8DA608DF810608DF811B08DF81240EC
:1064B8008DF8137008F010FD2A238DF810309DF820
:1064C80013308DF811708DF812401BB104A808F034
:1064D80003FD04E01E4B4FF48062C3F884201D4A7C
:1064E8001D4B136002221A721C4A1D4B13601D4A71
:1064F8001D491B68116098471C4B2B600E4806E02D
:106508001B480095FCF738FA00283FF41AAF074BF0
:1065180006710C2202FB083888F80890C8F80400B5
:1065280000E0204607B0BDE8F08F00BFA42400209B
:106538000038014014040140A81900200804014053
:106548000C040140D80042420005FA0500ED00E0C5
:1065580000E100E0982300209C2300207022002006
:10656800CC0000206C22002014000020C044010848
:1065780000440040001002400C4B1B6893F90220B5
:10658800824209D093F90A20824207D093F9122057
:10659800824208D1022002E0002000E0012003EB43
:1065A800C000023070470020704700BFA0240020C0
:1065B800F0B5027887B0AAB94C4C04F118064C4BD8
:1065C80094F9F61193F900208A4272D093F90C20BD
:1065D8008A426ED093F918308B426AD00834B4429C
:1065E800EDD180E0002204920592451C0CF050F891
:1065F800C4B260B2FFF7C0FF074618B18DF810406B
:10660800012400E00446284620210BF0DCFF054663
:1066180038B1013528460CF03BF80134ADF81200CA
:10662800E4B20026284620210BF0CDFFB0B3451C6C
:1066380028460CF02DF800222E4951F822308342CA
:106648005FFA82FE04D00132082AF5D1002300E067
:10665800734651F82320824220D1022E0FD0032EF8
:1066680012D05A1E012ED2B204D0042A13D88DF8A3
:1066780014300EE0042A0ED88DF8153009E0052BE9
:1066880009D88DF8173004E09A1E052A03D88DF82A
:1066980016300134E4B20136042EC3D1052C03D8D8
:1066A80007B0BDE8F040AFE404AB03CB38607960D5
:1066B80019E094F8FB010F4B94F8FA5153F82000B5
:1066C800B4F8F821009094F8FD0153F820000190E7
:1066D80094F8FC0153F82000029053F8253006483E
:1066E80001F0C7FA7AE707B0F0BD00BFB411002087
:1066F800A42400208C5C01083763010838B1438862
:1067080011EA030003D08B420CBF0120022070471E
:1067180030B50B4B0B491C6891F83820022A0BD86E
:10672800134604EBC303551CEAB29D882842F5D0F2
:1067380081F83820981C30BD81F83820002030BD01
:10674800A0240020A8190020024B002283F838203A
:10675800DEE700BFA81900202DE9F047877890F8F8
:1067680003C0214DBBB2C7F1640E03EB83065C4244
:10677800C3F178005FFA8EFE7600CCF16408A4B20B
:1067880080B2A3B20FFA83F9B9F1000F05DC002B30
:1067980014BFBA464FF0010A00E0F24613FB03F3B8
:1067A80003FB0CF21AFB0AF392FBF3F3434403FBDB
:1067B80009F30A2293FBF2F333449BB225F8023F14
:1067C800B1F800904A880A34C9EB020AA4B21AB296
:1067D80002FB0AF24FF47A73844292FBF3F34B44C0
:1067E8002B80CED1BDE8F087E019002010B54478A1
:1067F8000078002202FB02F3193B634303F6C4133B
:10680800534340F6C411434393FBF1F3034921F882
:1068180012300132072AEDD110BD00BFFA1900204D
:106828000430114B33F91000B0F5617F10B506DB69
:1068380040F6330398420246A8BF1A4601E04FF4D7
:1068480061720C78192340F2833013FB04049442DC
:1068580007DA497813FB01039342B4BF00200120F3
:1068680010BD002010BD00BF101B002010B500F1A6
:10687800500302788A4203D18478C278944204D3C0
:1068880004309842F5D1002010BD012010BD0B4BFB
:106898001B6813F4805F0A4BB3F9063005D0C08932
:1068A800421A934207DD084400E0008A8342B4BFDD
:1068B8000020012070470120704700BF702600208B
:1068C800101B00201FB5094B1B681B030AD58DF848
:1068D800040001230D2001A98DED030A8DF8053070
:1068E80002F0F0FD05B05DF804FB00BF7026002043
:1068F8001FB5084B1B681B0309D58DF804000291CE
:1069080000230D2001A98DF8053002F0DBFD05B04C
:106918005DF804FB7026002010B5002005F080FB10
:10692800064B00241C7008F0E7FE054B83F8604016
:106938005C66A3F86840DC6610BD00BFE026002056
:10694800A819002010B510B9BDE81040E4E70023ED
:106958000C225A430A4C1119125D824203D00133AA
:10696800102BF5D110BD074BD86E18B14A78407876
:10697800824204D20022D966A3F868205A6610BD64
:10698800684D0108A819002010B540001428A8BFB8
:1069980014200023074A022199540B4499181424FF
:1069A800834201F8014CF5DBFF21D1540F20BDE8EB
:1069B8001040C7E7782300202DE9F84307460B2449
:1069C800013C36D01D4B4FF480529A617D1C322613
:1069D8004FF00508DFF86490B9F814309BB283F4DF
:1069E8008053A9F81430012005F01AFB304605F051
:1069F800FEFAB9F814309BB283F480530020A9F84A
:106A0800143005F00DFB304605F0F1FAB8F1000F2F
:106A180008D0B8F10108DDD14FF4FA7005F0E7FAB3
:106A2800FA26D7E7013DD5D14FF47A7005F0DFFAA1
:106A3800C6E7034B034ADA60BDE8F8830004004860
:106A480000ED00E00400FA0510B5214A18B91368F2
:106A580002221A8210BD1F4814680023038021787F
:106A680011F07F0102460DD1637A990644BF0221D5
:106A7800017013F0400F037814BF43F0010323F0B3
:106A8800010315E0012921D002291ED1637913F0F1
:106A9800800F03F00F034FEA830303F1804303F5EC
:106AA800B8431B6806D003F03003102B07D101232D
:106AB800137004E003F44053B3F5805FF6E7064B28
:106AC8001B681B699847034810BD184610BD00BFD6
:106AD80098230020181A00206C22002010B5064CBC
:106AE80018B9236801221A8210BD044B1B689B68E1
:106AF800984720680C3010BD982300206C22002095
:106B080010B5064C18B9236801221A8210BD044B2F
:106B18001B681B68984720680A3010BD982300201E
:106B28006C22002003788B4283BF034B03EB4101A7
:106B380048880020704700BF181A002070B500224E
:106B48001346244914180C44A47E83EA0423082419
:106B580013F4004F4FEA430318BF83F4815304F141
:106B6800FF3418BF83F0010314F0FF049BB2EFD188
:106B78000132192AE5D100F1190200F11A050A4477
:106B88000D44967EAA7E02EB062292B29A421FD14B
:106B9800104B93F83B50E2B2AA4216D2431C03EBC7
:106BA8004203DBB2CA1801330B44927E9B7E03EB8F
:106BB80002239BB24FF4AF6253431B13064A03F5FB
:106BC800487322F814300134E5E7012381F83C309A
:106BD80070BD00BF181A00201A1A002003788B42D3
:106BE8000BD9074B1A78074B89001944086C02B176
:106BF800400800F5777080B270470020704700BFEA
:106C08009C240020181A002007299DBF034B03EB82
:106C18008101B1F870000020704700BF181A0020E9
:106C2800034B03EB4101B1F89000C008704700BF67
:106C3800181A00200A4BDFED0B7A03EB810191ED66
:106C48002C7AB8EE477AF6EE046AE7EE267A82B036
:106C5800FCEEE77ACDED017ABDF8040002B070478A
:106C6800181A002000005C44024B03EB4101B1F804
:106C7800F8007047181A0020024B03EB4101B1F8E5
:106C88001C017047181A002070B5334C054605F0F2
:106C980087F9D4F83431C4F83401C31AB3F5FA5F6C
:106CA800C4F8383182BF002384F83C3184F83D3180
:106CB80094F83C312BB9A12D02BF274A012182F853
:106CC8003D1194F83D11244A29B1D118EDB2013390
:106CD8008D7682F83C3194F83C5194F83E31AB42C1
:106CE80039D11D4B93F83F31052B02D0062B03D029
:106CF8002CE00020FFF722FFE37E1E2B26D1002088
:106D08000246C1B26B1E994219DA21448B7E0821D2
:106D1800DBB283EA0206F60744BF83F01803C3F325
:106D2800460301F1FF3154BF5B0843F0800311F0C3
:106D3800FF01C2F34702ECD101301A46E1E72344D0
:106D48009B7E9A4202D10320FFF7F8FE002384F8C5
:106D58003D3184F83C3170BD181A002010B5044646
:106D680005F01EF90F4BD3F84021C3F84001821AF1
:106D780041F288318A42C3F8442184BF002283F853
:106D8800482193F84821074913440F2AE4B218BF51
:106D9800013283F8494112BF81F84821012381F863
:106DA800593110BD181A002010B5044605F0F8F83E
:106DB8000F4BD3F85C21C3F85C01821A41F2883189
:106DC8008A42C3F8602184BF002283F8642193F8C3
:106DD800642107491344142A18BF013283F8654116
:106DE80012BF81F86421012381F87A3110BD00BFF8
:106DF800181A002038B5044605F0D2F8274A274962
:106E0800D2F87C31C2F87C01C31AB3F57A6F84BF1B
:106E1800002382F8803192F8803133B9A82C3BD115
:106E280081F88131A1F8823106E0022B02D181F884
:106E3800844101E0242B02D8D11881F8854192F8C9
:106E48008411164D01330231DBB249008B4282F8BE
:106E5800803118DAB5F88231E0B283EA00200823DD
:106E680010F4004F4FEA400018BF80F4815003F13E
:106E7800FF3318BF80F0010013F0FF0380B2EFD199
:106E8800A2F8820138BD01318B4201BF002385F889
:106E98008031012385F8813138BD00BF181A0020E0
:106EA80010B5044605F07CF8104AD2F8AC3140F62B
:106EB800AC51C31A8B42C4BF002382F8B03192F898
:106EC800B031D11881F8B14123B90F2C0DD1074940
:106ED800C1F8AC010133DBB2192B044982F8B03197
:106EE8000CBF0123002381F8CA3110BD181A0020F5
:106EF8002DE9F843324F3D682A8A2E7AB2B9042E1A
:106F080014D1304C30482378012B0BD12F4B196802
:106F18002F4B89B20B445B0019681A603023038039
:106F2800227048E010230380072644E0AC8AAB694E
:106F3800A24294BF04260226944228BF14461FFA90
:106F480084F840469847214A13689BB203F10053DE
:106F580003F540535B0004F1010E1B689BB203F17B
:106F6800005303F540534FEA6E0E5B000021714554
:106F780000F1020009D010F8019C10F802CC4CEA8C
:106F8800092C23F821C00131F1E71268104B92B2A5
:106F980013445B001A681C602B8AC8EB03032B821E
:106FA8006B8A9844084BA5F8128030221A80094B46
:106FB8004FF440521A803B681E72BDE8F88300BF48
:106FC800982300201227002066220020505C0040F1
:106FD80002300020642200200E4B0F4A1B689BB22F
:106FE80003EBC00002443E294FEA420209D94B098B
:106FF800C80604BF03F1FF339BB29B0243F400436E
:1070080004E04B08C90748BF01339B0211681360AD
:10701800704700BF505C00400630002010B5454B5B
:107028001A68107810F07F0004D1537A23F02003F7
:10703800537210BD02287AD15388002B78D1137966
:10704800002B75D1537923F08000840004F180412E
:1070580001F5B84113F0800F096814BF01F0300141
:1070680001F44051032862D8002960D0927A002A9E
:107078005DD004F1804404F5B8441906226825D58A
:1070880002F03002102A4CD103F07F039B0003F179
:10709800804303F5B8431A68510641BF196840F6A2
:1070A8000F720A4042F4004244BF42F0C0021A6024
:1070B8001A6822F4E04222F0400292B282F03002D2
:1070C80042F4004242F080021A602AE002F4405280
:1070D800B2F5805F25D128B9174B93F82C10FFF72C
:1070E8007BFF11E09B0003F1804303F5B8431A6866
:1070F800520441BF196840F60F720A4042F44042F8
:1071080044BF42F080021A60236823F4804323F0CE
:1071180070039BB283F4405343F4004343F080036D
:107128002360064B1B685B699847002010BD02204E
:1071380010BD00BF98230020CC0000206C22002046
:1071480002684FF6FE731340036000230360436038
:107158008360C360284B984201D1284A27E0284B16
:10716800984201D1254A2AE0264B984201D1234A68
:107178002DE0254B984201D1204A30E0234B98421C
:1071880001D11E4A33E0224B984204D11B4A53686E
:1071980043F470032EE01F4B984204D1174A5368FA
:1071A80043F0706326E01C4B984204D11B4A536895
:1071B80043F00F031EE01A4B984204D1174A536854
:1071C80043F0F00316E0174B984204D1134A536872
:1071D80043F470630EE0144B984204D10F4A53688D
:1071E80043F4704306E0114B984204D10B4A5368AC
:1071F80043F47023536070470800024000000240C7
:107208001C00024030000240440002405800024086
:107218006C00024080000240080402400004024062
:107228001C04024030040240440402405804024056
:10723800084BDA68D10709D4DA68D20608D4DB68C3
:1072480013F0040F14BF0320042070470120704777
:107258000220704700200240994A536803F00C034B
:10726800042B2DE9F04105D0082B06D09549016083
:10727800B3B916E0934B036012E053685468C3F344
:107288008343991CE30349BFD36A8F4B8D4C03F0AA
:107298000F0344BF0133B4FBF3F34B43036000E037
:1072A80000235168894FC1F303117D5C0168EDB279
:1072B80021FA05F444605668C6F30226BE5D24FA36
:1072C80006FEC0F808E05668C6F3C226BE5DF6B2F0
:1072D800F440C460D2F82C80C8F3041808F00F0CEE
:1072E80007EB4C0C18F0100FBCF810C01FFA8CFC00
:1072F80007D0BCF1000F04D0B3FBFCFCC0F810C0F1
:1073080000E00161D2F82CC0CCF3442C0CF00F083B
:1073180007EB48071CF0100F3F8ABFB204D01FB11B
:10732800B3FBF7F7476100E04161176BFF065ABFEF
:10733800644F87618161176BBF065ABF614FC76190
:10734800C161176B7F065ABF5E4F07620162176BF8
:10735800FF0506D5994204D1AE4202D14F004762DB
:1073680000E04462176BFF0406D5994204D1AE428F
:1073780002D14F00876200E08462176BBF0506D513
:10738800994204D1AE4202D14F00C76200E0C46204
:10739800176B7F0506D5994204D1AE4202D14F0042
:1073A800476400E04464176B3F0506D5994204D151
:1073B800AE4202D14F00876400E08464176BBF04BB
:1073C80006D5994204D1AE4202D14B00C36400E015
:1073D8008464156B3A4BAD0701D1046315E01C6B4F
:1073E80004F00304012C01D101630EE01C6B04F0CE
:1073F8000304022C02D14FF4004305E01B6B03F099
:107408000303032B01D12F4B0363146B2C4B14F490
:10741800403F02D1C0F834E018E01C6B04F440345B
:10742800B4F5803F01D1416310E01C6B04F4403493
:10743800B4F5003F02D14FF4004306E01B6B03F4A0
:107448004033B3F5403F01D11E4B4363146B1C4BD3
:1074580014F4402F02D1C0F838E018E01C6B04F493
:107468004024B4F5802F01D1816310E01C6B04F433
:107478004024B4F5002F02D14FF4004306E01B6B03
:1074880003F44023B3F5402F01D10E4B8363146BF3
:107498000B4B14F4401F02D1C0F83CE020E01C6BF9
:1074A80004F44014B4F5801F01D1C16318E01C6BCB
:1074B80004F44014B4F5001F0AD14FF400430EE061
:1074C8000010024000127A0000093D003800002038
:1074D8001B6B03F44013B3F5401F01D1134BC36377
:1074E800126B134B12F4400F03D1C0F840E0BDE813
:1074F800F0811A6B02F44002B2F5800F02D10164E8
:10750800BDE8F0811A6B02F44002B2F5000F02D117
:107518004FF4004306E01B6B03F44003B3F5400F40
:1075280001D1024B0364BDE8F08100BF00127A006C
:1075380000100240F0B500230E681C460125A54046
:1075480005EA060EAE452BD10F797A1E012A15D809
:10755800856803229A4025EA020282604D79826892
:107568009D4015438560828892B222EA0E0282808D
:107578008A798588A2402A4392B2828003220568CC
:107588009A40D2431540056005689F402F43076025
:10759800C7681740CA7902FA03F547EA0502C260CC
:1075A8000134102C03F10203C8D1F0BD38B52DED1C
:1075B800048B4A4C0368C4F8CC318388A4F8D031D2
:1075C800013A0D46072A42D8DFE802F0040A1018EB
:1075D80022292F35B4F8CC310B80B4F8CE3113E022
:1075E800B4F8CE310B80B4F8CC3105E0B4F8CC3126
:1075F8005B420B80B4F8CE315B4205E0B4F8CE3183
:107608005B420B80B4F8CC316B80B4F8D0311DE00C
:10761800B4F8CC315B420B80B4F8CE3112E0B4F848
:10762800CE310B80B4F8CC310CE0B4F8CC310B80FF
:10763800B4F8CE3105E0B4F8CE315B420B80B4F833
:10764800CC315B426B80B4F8D0315B42AB80244BC9
:1076580093F83030002B3ED1B5F9003094ED780A1C
:10766800D4ED757A09EE103AB5F9023008EE103A01
:10767800B8EEC88AB5F90430B8EEC99A28EE000AFF
:1076880008EE903AA7EE890AF8EEE88AD4ED7B7AFC
:10769800A7EEA80A0BF070F994ED790AD4ED767A82
:1076A800288028EE000AA7EE890AD4ED7C7AA7EE96
:1076B800A80A0BF061F994ED7A0AD4ED777A68801C
:1076C80028EE000AA7EE890AD4ED7D7AA7EEA80A6B
:1076D8000BF052F9A880BDEC048B38BD181A0020B5
:1076E80038000020094B1A68137844F6FB7103EB45
:1076F800431300FB03135078C0EB0030B3FBF0F3E7
:107708009078B3FBF0F080B2704700BFC818002033
:107718000748002108B50A22A0F8F81100F5007002
:1077280004F093FC80B2FFF7DDFF024B188008BD20
:10773800181A0020CC180020F0B50124B0FBF4F58D
:107748008D4201D34C43F9E70026D4B1B0FBF4F5E0
:1077580004FB1500B4FBF1F41EB9002D01DC002C6C
:10776800F3D1092D03F1010EEFB204DD002A14BF95
:107778003725572500E030253D441D7001367346F6
:10778800E3E71C70F0BDF0B50124B0FBF4F58D42C1
:1077980001D34C43F9E70026D4B1B0FBF4F504FB60
:1077A8001500B4FBF1F41EB9002D01DC002CF3D157
:1077B800092D03F1010EEFB204DD002A14BF3725AD
:1077C800572500E030253D441D7001367346E3E738
:1077D8001C70F0BD2DE9F843089E002B074688462B
:1077E800144614BF4FF030094FF02009334613F800
:1077F800012B0AB9254603E0002CFBDD013CF6E726
:10780800002D04DD38464946C047013DF8E724EA23
:10781800E4743546A01B284415F8011B11B13846FD
:10782800C047F7E7BDE8F883014B186804F00ABCC5
:10783800C010002090ED017A07EE901AB5EE407A5C
:10784800F1EE10FA01BFF8EEE77A9FED0E7A67EED7
:10785800877AB7EE007A04BFC7EE277AC0ED017ABF
:1078680090ED017AD0ED007A30EE877A30EE670A33
:10787800C0EE870AE0EE807AB0EE670AC0ED007AC3
:10788800704700BFDB0FC94010B50278202A0346B5
:1078980000F10100F9D0092AF7D02D2A03D10346B7
:1078A800BFEE000A04E02B2A08BF0346B7EE000A21
:1078B800DFED387A1A46134612F8010BA0F13001B1
:1078C800CCB2092C0AD807EE101AB8EEC77AF2EE35
:1078D800046AA7EEA67AF0EE477AECE72E2816D1CE
:1078E800F2EE046A1146B0EE666A0B4611F8012BF7
:1078F800303AD0B209280AD807EE102AB8EEC77A6B
:1079080087EE267A66EE866A77EE877AEDE71A784A
:1079180002F0DF02452A35D15A782D2A02D10233E6
:10792800012004E02B2A14BF013302330020013B5D
:10793800002213F8011F3039CCB2092C03D80A24CD
:1079480004FB0212F5E7B2F59A7F28BF4FF49A724A
:107958001346B7EE007A072B05D9DFED0F6A083B0F
:1079680027EE267AF7E702F007032BB1F2EE046A56
:1079780027EE267A013BF8E7F0EE476A20B1C7EE1A
:10798800877A03E0F7EE006A67EEA67A20EE270A08
:1079980010BD00BF0000000020BCBE4C30B52DED6E
:1079A800028B87B0B0EE408A0C220021054603A85E
:1079B8000AF0D3FDB5EEC08ADFED2A7AF1EE10FAAF
:1079C800CCBF38EE278A38EE678ADFED277A28EEB3
:1079D800278A6946FDEEC87A17EE904A84EAE47071
:1079E800A0EBE47007F020F8002CACBF20232D2377
:1079F80068468DF80C300AF0F4FD012807D13023D1
:107A08008DF80D308DF80E308DF80F300CE002280F
:107A180005D130238DF80D308DF80E3004E00328A1
:107A280004BF30238DF80D30694603A80AF0BCFD69
:107A380003A80AF0D6FD0338C4B2224603A9284693
:107A48000AF0FCFD00232B55284608490AF0ACFD36
:107A580003AB284619190AF0A7FD284607B0BDEC64
:107A6800028B30BD6F12033A00007A445663010856
:107A780070B5064615460846B6FBF2F414B1204622
:107A8800FFF7F6FF05FB1464024B1B5D00F8013B92
:107A980070BD00BF586301082DE9F04F814689B0D9
:107AA8008A4616461C4600253178002900F0DD80FC
:107AB800252902D00136484675E07278302A08BF79
:107AC800B278A2F1300319BFB71C4FF0000BF71CB6
:107AD8004FF0010B092B4FF0000819D8A2F1300321
:107AE800D9B2092905D80A2202FB083817F8012B50
:107AF800F4E7A2F16103052B02D8A2F1570305E0D0
:107B0800A2F14103052B03D8A2F137030A2BEADDC2
:107B18006C2A31D13A78642A07F1010600F0838093
:107B28000BD8252A3DD003D8002A00F09E80BBE759
:107B3800582A0CD0632A19D0B6E7732A22D002D863
:107B48006E2A37D0B0E7752A5CD0782AACD1271DC9
:107B58002068A2F1580462424FF01001624155E0DA
:107B68002CD9582A32D0632A2AD13E464846217851
:107B7800271DD04701350FE0642A64D00ED9732A37
:107B880014D13E4623680093484651464246002396
:107B9800FFF720FE271D05443C4685E7252ADFD14F
:107BA8003E4648462521D04701357DE70AD86E2A4A
:107BB80006D13E46236804341D6075E7002A54D078
:107BC8003E4671E7752A26D0782AF9D1A2F15803E2
:107BD80004F1040C5A422068CDF80CC04FF0100193
:107BE8005A4105ABFFF7A8FDDDF80CC03E466446D8
:107BF80005AB00934846514642465B46FFF7EAFD0F
:107C0800054451E72068271D0A21002205ABFFF72C
:107C1800BAFD3C46ECE704F1040CCDF80CC0206832
:107C28000A210022DDE72068002804F1040708DAA9
:107C38002D238DF8143040420DF115030A2100223E
:107C4800E5E705ABFAE72068002804F1040C0ADA36
:107C58002D238DF8143040420DF11503CDF80CC0DA
:107C68000A210022BEE705ABF8E7284609B0BDE8BF
:107C7800F08F0FB413B50B4904AB08680A4953F8E1
:107C8800042B09680193FFF707FF0446074B1868A0
:107C980004F0CCF90028F9D0204602B0BDE8104025
:107CA80004B070476408002060080020C01000205D
:107CB80080EAE073A3EBE0738B4206DB002801DD6A
:107CC800401A704702D00844704700207047FDEE04
:107CD800C07A17EE903A2033402B43D8DFED237A51
:107CE800B4EEE70AF1EE10FA04DDDFED217A30EEAA
:107CF800670AF3E7DFED1F7AB4EEE70AF1EE10FA50
:107D080004D5DFED1B7A30EE270AF3E7DFED1A7AA8
:107D1800B4EEE70AF1EE10FA04DD30EE670A37EE4A
:107D2800C00A0AE09FED157AB4EEC70AF1EE10FA20
:107D380044BF30EE270A37EE400A60EE007ADFEDE6
:107D4800106A9FED107AA7EEA67ADFED0F6AE7EECC
:107D5800876A9FED0E7AA7EEA67A20EE276AA6EE2E
:107D6800070A70479FED0A0A704700BFDB0F4940BA
:107D7800DB0FC940DB0F49C0DB0FC93FDB0FC9BFB1
:107D88009A7C2E36FAAF4FB93587083CA4AA2ABE8A
:107D980000000000DFED027A30EE270A97E700BF07
:107DA800DB0FC93F38B52DED068B90ED008AB0EE9C
:107DB800480A0C460546FFF7EDFFB0EE40AAB0EEC4
:107DC800480AFFF784FFD5ED018AB0EE409AB0EE7D
:107DD800680AFFF7DFFFB0EE408AB0EE680AFFF7E7
:107DE80076FFD5ED02AAF0EE408AB0EE6A0AFFF7F8
:107DF800D1FFF0EE409AB0EE6A0AFFF768FF60EE36
:107E08000A6A69EE297AF0EE665AE7EEA85A29EE70
:107E18008A6A29EE007A69EE889A29EE489A28EE4D
:107E2800400A28EE0A8AC4ED035AF0EE465AE7EEF5
:107E3800685AE6EEA87AA6EE687AC4ED009AC4ED10
:107E4800028A84ED059A84ED088ABDEC068B84EDE0
:107E5800010AC4ED045A84ED067AC4ED077A38BDE8
:107E680010B52DED048B8AB090ED009AD0ED028A02
:107E780090ED018A0446084601A9FFF793FFDDED5E
:107E8800047A9DED017A68EE277AE9EE077A9DED8E
:107E9800077AE8EE877A9DED027AC4ED007ADDED87
:107EA800057A68EE277AE9EE077A9DED087AE8EE1A
:107EB800877AC4ED017ADDED067A28EE278ADDEDB2
:107EC800037AA9EE278ADDED097AA8EEA78A84ED60
:107ED800028A0AB0BDEC048B10BD074B1A8822EA4F
:107EE8000000904210B518801C4602D00120FEF711
:107EF8004BFD208810BD00BFA4190020064B1A882E
:107F08001043904210B518801C4602D00120FEF79D
:107F18003BFD208810BD00BFA4190020024A9368C9
:107F280023EA000090607047B411002008B5104B98
:107F38001A780023D9B2914207D20E4951F823107A
:107F48000968002008600133F4E7322004F04FF894
:107F5800094B1B685A0309D5084B9B685B0305D47A
:107F680040F2DC50BDE8084004F041B808BD00BF4D
:107F78008A2000209420002070260020B4110020C0
:107F88002DE9F34107F09AFB454A6923137040F243
:107F980014735380BE231371EF2382F81137002323
:107FA80082F8123719461646F25C0133514040F206
:107FB80014729342F8D13A4B83F81217394B1A6965
:107FC800120604D5384A5A6002F188325A600427EA
:107FD8000020013F17F0FF0750D0324B3422DA60FF
:107FE800002444B1002356F80480019306F0ECFC09
:107FF8000428EED117E006F0E7FC0428E9D1294D62
:108008002B6943F002032B61284B6B612B6943F00A
:1080180040032B6106F0D8FC2B69042823F00203E7
:108028002B61DFD0D5E71F4D2B6943F001032B618E
:1080380004F1006303F57E331FFA88F21A8006F014
:10804800C3FC042810D11A4B23440193019B4FEA27
:108058001848A3F8008006F0B7FC2B69042823F021
:1080680001032B6105D0B4E72B6923F001032B61D1
:10807800AFE7043440F214739C42B2D1094A136941
:10808800042843F08003136102D105F033FF10B9CF
:108098000520FEF791FC07F0FFFA02B0BDE8F08179
:1080A800B4110020002002402301674500F80308AE
:1080B80002F8030810B50E4C2068FEF797FB2068FD
:1080C800047A002202FB02F3193B634303F6C4134C
:1080D8005343192193FBF1F3064921F81230013279
:1080E800072AEFD10449BDE81040FEF735BB00BFB1
:1080F8003411002090100020F81200202DE9F041E2
:1081080005F0F8FE10B90420FEF756FCAC4CAD4D56
:1081180007F0D4FAAC4940F2147220460AF012FA79
:1081280094F8E836022B84BF002384F8E83694F8E4
:10813800E8264FF4CC7101FB02F303F508702344E1
:108148002044286093F8740203F51C73022801FB8D
:10815800024284BF0020187192F874329B4A13704F
:108168000C2202FB03439A4A03F2EA631360A368F2
:1081780046F209021A401AB9914A43F4005393602F
:10818800A368D80703D54FF40050FFF7C7FEA368CC
:10819800590409D50820FFF7C1FE4FF40050FFF736
:1081A800BDFE0120FFF7BAFEA3681A0706D54FF4F3
:1081B8000050FFF7B3FE0120FFF7B0FEA3689B0451
:1081C80002D54020FFF7AAFE012284F8112294F874
:1081D800E0217B4B2AB193F8E42112B1002283F805
:1081E800E4217C4B7C4E1E604FF0000C674604EB8C
:1081F8000C03B3F8F8E14FEA5E0101F077314FEA7A
:108208009E0303F03333C1EB0E00C11A4FEADE03BD
:1082180003F01133CB1A03EB23131EF0010803F00C
:108228000F324FF0FF0392FBF3F3C3EB032318BFA6
:108238000137A2EB030318BFFFB2012B0ADD022BA3
:1082480040F0BB80B8F1000F00F0B7801EF0BC0F03
:1082580000F0B3800CF1080CBCF1180FC7D1013F36
:10826800012F00F2AA80FFF725FF302200215B488A
:108278005B4F0AF072F95B4BD5F800801F605A4BD0
:10828800002108F17900C3F80080FEF7EFFA574B98
:1082980080F001001870564B07F126021A60554B02
:1082A80007F1CC021A6098F8000004F009F9286870
:1082B800514B00F5C5721A6003F03EF84F4B94F825
:1082C800D801DFED4F6A07F194021A6064214D4B23
:1082D800C82211FB00225A6000229A60DA601A61F3
:1082E8005A619A61DA6183F8202083F82120464B8D
:1082F80007F12C021A602B68444A93ED187A03F2AE
:1083080019111160424A03F289111160414A07F1BB
:1083180008011160404A1760404A07F1A001116046
:108328003F4A07F1AA0111603E4967EE266A0E60CE
:10833800B4F86611B6EE007A07EE901A87EE267A40
:10834800B4F86811101DF8EE677AC2ED027A07EEEC
:10835800901A93F85C10117193F87810517194F891
:10836800E3111174F8EE677AB3F81611C2ED037AC7
:1083780007EE901A2C4908602C49536103F16400F8
:1083880008602B49936181ED007AF8EEE77A9FED5A
:10839800297A29495762C7EE277ABDE8F0419FED4F
:1083A800277A67EE877AC1ED007A03F1680103F254
:1083B8001113D161136207F06FB906F0D1FA52E7D1
:1083C800B41100201411002000F803084C230020E9
:1083D80034110020B02600203E130020D00A0020CF
:1083E800F8120020040B0020080B002010000020C9
:1083F800B0010020000A0020100B0020941D00206E
:10840800DB0F4940BC26002008020020001D002088
:1084180010040020DC210020E0210020240300209B
:10842800A01C0020E8030020380200207002002071
:108438006C02002000006144200300204C3D0F44E2
:1084480008B5FFF79DFDFFF759FE0120BDE808407C
:10845800FEF79ABA38B500240B4D6059254405F04B
:1084680033FB696811B10948FFF703FCA96811B12A
:108478000748FFF7FEFB0748103405F025FBB4F565
:10848800C87FE9D138BD00BFD8440108506401084D
:10849800566401086D6C0108F0B585B004460AF011
:1084A800A0F8082826D1621EE01D1F4912F8013FD6
:1084B80009681944497801F00301022908BF203BE3
:1084C80082421370F1D1254604F1080715F8016BB3
:1084D800164831460AF077F820B1284631460AF0A6
:1084E80072F810B1FDF790FD1CE0BD42EED12046B8
:1084F80006F07CFA0E4805F0E7FA00230D4A1A4404
:1085080004A992F88A210A440849595C02F80C1C0B
:108518000133082BF2D1002307488DF80C3001A94C
:10852800FFF7A7FB05B0F0BD0C010020DD770108BF
:108538005C640108B4110020AF6B01081E4B1F4C8E
:108548001D68206880B5FDF7B1FE2846FDF7AEFE30
:10855800206841798B0704D4036841F002015B6904
:108568009847174B4FF480529A61206803F067FDD3
:10857800A0B1134E4FF480533385104B186803F0A5
:108588005BFD074602F039FB08B104F029FD2846D7
:10859800394603F057FD4FF48053B361284603F082
:1085A8004EFD0028E1D02846266803F045FD014627
:1085B800304603F047FDD8E768230020C81C002098
:1085C800000400482DE9F04705460AF00AF8314E44
:1085D8000446D6F8088090B92F4805F075FA2F4B55
:1085E80053F8241049B10123A34013EA080F02D01D
:1085F8002B48FFF73EFB0134F1E72A4822E02846E2
:108608002949224609F0F6FF58B92848284C05F0B0
:108618005BFA54F8041F0029EFD02148FFF729FB23
:10862800F7E72B782D2B03BF013504F1FF344FF00A
:10863800010A4FF0000A4FF00009184B53F829704F
:1086480027B91C48BDE8F04705F03EBA2846394628
:10865800224609F0CFFFC8B9012000FA09F08305C6
:1086680001D51548EEE7BAF1000F03D0FFF756FC25
:10867800124803E040EA0800B060114805F024FA07
:1086880039461048BDE8F047FFF7F3BA09F1010988
:10869800D3E700BFB41100206264010868460108EE
:1086A8006C6401086D6C0108706401087564010848
:1086B8006446010881640108906401089E64010809
:1086C800A7640108AE6B010810B5084805F0FCF96D
:1086D800074B00241C715C63064B1C7003F036FECC
:1086E80005F0D6FB044B1C6010BD00BFAF64010849
:1086F800C81C0020112700206823002070B50646FA
:1087080000240B4BE518AA8816420AD0E1580948FC
:10871800FFF7AFFA2846002105F063F9064805F08F
:10872800D3F9143440F6BC439C42EAD170BD00BF73
:10873800084F0108DB6401086D6C0108F0B5047886
:108748008BB005460CB1002436E04B4B19680E235C
:1087580003FB041101F58C70B1F91D51B1F9192110
:10876800B1F91B31009591F82051019591F82151EB
:10877800029590F90700039001F590713F4891F92F
:108788000210049121460134FFF773FA082CDCD15A
:1087980070E02D2B14D1072C1BDC284609F078FF3C
:1087A8000AAB661C03EB440424F8100C15F8013FCF
:1087B800303B092BFAD934462B78002BE9D104E059
:1087C800A3F13002092A09D8E5E7082CBDF81820DA
:1087D80009D00BB0BDE8F040FDF716BC202BF8D14E
:1087E80001352646E7E7072AF3D8BDF81A00224BD9
:1087F800A0F2EE2189B240F2DC55A9421B68E8D804
:10880800BDF81C10A1F2EE24A4B2AC42E1D8BDF828
:108818001E6004B237B2A742DBDB0DB2AF42D8DC30
:10882800A542D6DBBDF8247007F16404A4B2C82CB5
:10883800CFD8BDF826E00FFA8EF4112CC9DCBDF8AC
:108848002050B42DC5D8BDF82240B42CC1D812B2DE
:108858004FF00E0C0CFB0233A3F81901A3F81B11FF
:10886800A3F81D6183F8205183F8214183F81F7113
:1088780083F822E10BB0F0BD14110020E564010873
:108888002DE9F041047806467CB9334DB5F8C62188
:10889800B5F8C831314821460134FFF7EAF9042C0C
:1088A80005F10405F2D1BDE8F0812D4909F05EFE1D
:1088B800B0B9294B4FF47A714FF4FA62A3F8C61194
:1088C800A3F8C821A3F8CA11A3F8CC21A3F8CE11A4
:1088D800A3F8D021A3F8D211A3F8D421BDE8F081E0
:1088E800304609F0D5FE032805462DD8304620210C
:1088F80009F069FE044630B10134204609F0C8FE8B
:108908000126074600E006462046202109F05BFEC6
:1089180018B9BDE8F041FDF777BB013009F0B8FEA2
:10892800012EF6D1A7F2EE2240F2DC539A42F0D89B
:10893800A0F2EE229A42ECD8074B703503EB850380
:10894800DF801881BDE8F08106480749002203232B
:10895800BDE8F041FFF78DB9B411002005650108A5
:1089680018650108C36201089B6E01082DE9F041F2
:108978002DED048BAB498AB0044609F0F7FDAA49EE
:10898800002820460CBF0126072609F0EFFDA7495D
:108998000028204608BF022609F0E8FD002808BF85
:1089A8000426F10740F1E380A148A24C05F08CF8B9
:1089B800002004F091FEA04805F086F89F4805F0D5
:1089C80083F863799E4A9F48013B254652F8231055
:1089D800FFF74FF99C48FFF74CF94FF0000827467E
:1089E80095ED058AB5EE408AF1EE10FA04D1974864
:1089F800FFF73FF9002570E09548D5ED069A95ED0B
:108A0800079AD5ED088A4146FFF733F9B5EEC08AD3
:108A1800F1EE10FA02D5202005F04EF8B0EE480A23
:108A280006A8FEF7BBFF01468A48FFF722F9F5EED4
:108A3800C09AF1EE10FA02D5202005F03DF8B0EE0C
:108A4800690A06A8FEF7AAFF01468248FFF711F94E
:108A5800B5EEC09AF1EE10FA02D5202005F02CF8F8
:108A6800B0EE490A06A8FEF799FF01467948FFF7D4
:108A780000F9F5EEC08AF1EE10FA02D5202005F0D3
:108A88001BF8B0EE680A06A8FEF788FF08F101088F
:108A980001467148FFF7EDF8B8F10C0F05F1100524
:108AA8009ED1A4E749B294F8D42094F8D530009127
:108AB80094F8D710019194F9D810029194F9D9102B
:108AC800039194F8DA100491644829460135FFF7B8
:108AD800D0F8102D04F1070403D094F8D61000291B
:108AE800E0D15F485F4C04F0EFFFD7F8088054F8F6
:108AF800041F19B15C48FFF7BCF8F8E70D465B4B5B
:108B080053F8254054B10123AB4013EA080F03D0B2
:108B180057482146FFF7ADF80135F0E7554804F00E
:108B2800D3FF21467B180AAA93F88A311344524A84
:108B38008A5C03F8102C01310829F3D1002306A917
:108B48004E488DF82030FFF794F84D4804F0BCFFEC
:108B58004C48FDF72DFD4C48FFF78BF84020FFF7F8
:108B6800CDFD4A4804F0B0FF4648FDF705FBB207C3
:108B780039D5474804F0A8FF464804F0A5FF414806
:108B880004F0EAFD444804F09FFF3E48FDF7C3F9AE
:108B9800424804F099FF3B48FDF73CFA4048FFF78C
:108BA80068F83848FFF76CFE3E4804F08DFF3548FA
:108BB800FFF7C4FD00270E257D4300243A4A926B37
:108BC8002A440123D2F80A20A34013421ED10134BB
:108BD8000E2CF3D10137082FEDD12B48FFF749F8B8
:108BE8008020FFF78BFD730716D5304804F06CFF23
:108BF8002F4804F069FF234804F088FD2248FFF756
:108C080038F84FF48070FFF779FD05E039462246C1
:108C18002848FFF72EF8DAE70AB0BDEC048BBDE868
:108C2800F08100BF1E6501087E69010825650108FD
:108C38002B650108B4110020396501084B6501084E
:108C4800C45B010857650108626501086F65010882
:108C58007C65010859640108AF6B01089465010837
:108C68008465010864460108B3650108684601087F
:108C7800C1650108CE650108DD770108DA650108DC
:108C8800E3650108706101086D6C0108F26501086F
:108C9800FF65010812660108206601082A660108B6
:108CA8003966010847660108C81C00205366010898
:108CB8006466010876660108F0B504468FB0204660
:108CC80009F08FFCC5B225BBAC48AD4C04F0FCFEE6
:108CD80094F8D61009B9AB4854E049B294F8D420B6
:108CE80094F8D530009194F8D710019194F9D810E0
:108CF800029194F9D910039194F8DA100491A248DA
:108D080029460135FEF7B5FF102D04F10704DFD120
:108D1800E1E720469D49052209F06CFC0546B8B9F3
:108D280029469B48702209F018FC9A4B1968284676
:108D38000E2303FB001301300022082883F82321A7
:108D480083F8242183F8252183F82621F0D113E123
:108D580020469149042209F04DFC05462046002D85
:108D68004AD1202109F02FFC002800F00581461C7B
:108D7800304609F036FC2C460746884B53F82450F9
:108D88002DB987480FB0BDE8F040FEF772BF3046F6
:108D98002946FAB209F02EFC01340028EDD1784AB0
:108DA80002F170011646002382F8DA3082F8D630D4
:108DB80082F8D53082F8D43007328A42F3D1794923
:108DC80001EBC40191F8E821934210DAD1F8EC7173
:108DD800C3EBC302B0183A4400F1D4011768C0F8D5
:108DE800D4709088888092798A710133E7E72946A0
:108DF8006D48FEF73EFF90E06C49072209F0FAFB48
:108E080005462046002D4AD1202109F0DCFB064604
:108E180009F0E7FBC4B274BB6548FEF72AFF214698
:108E280064480134FEF725FF0E2CF8D15548FEF7AB
:108E380020FF002460482146FEF71BFF0025554A05
:108E48005E4811680E2202FB04120123D2F8232186
:108E58005B49AB4013425B4B05F1010508BF19465E
:108E6800FEF707FF0E2DEAD146480134FEF701FF51
:108E7800082CDFD180E03046534909F00DFC2C4620
:108E880000284CD0022C4FD009F002FC06AB4E490A
:108E980043F82400002009F0FFFB0134F0E74A49B9
:108EA80009F0FAFB002460B1082C38D009F0F0FB77
:108EB80006AB454943F82400002009F0EDFB0134D6
:108EC800F1E7082C2BD1069B0F2B28D8DDF81CE0E6
:108ED800BEF1070F23D8089F0D2F20D8099E06F151
:108EE8006402C82A1BD80A9DFF2D18D80B9864283D
:108EF80015D80C99642912D8884210DA0D9C032CD5
:108F08000DD8324AC3EBC303134483F804E05F71FE
:108F18009E71DD71187259729C722D4CCFE60FB09C
:108F2800BDE8F040FDF770B8069B072B20D80799DD
:108F38000D291DD80278722A0DD06E2A18D1154A2B
:108F480012680E2000FB032301228A40D3F8231164
:108F580021EA020209E00F4A12680E2000FB0323EF
:108F680001228A40D3F823110A43C3F8232101E0E0
:108F7800FDF74AF80D4CA2E60FB0F0BD9566010862
:108F8800B41100206D6C0108C0660108186501085D
:108F98008812002014110020DC660108C45B010857
:108FA80081640108D8440108E16601088D6601085A
:108FB8005A640108ED660108C76B0108F2660108EA
:108FC800CE6F010888700108F66601088412002037
:108FD800706101082DE9FF4104780546002C39D15C
:108FE8007348744D04F070FDD5ED057AF5EE407ABE
:108FF800F1EE10FA00F0D98021466F48FEF739FEED
:1090080095ED050A6846FEF7C9FC01466B48FEF770
:1090180030FE95ED060A6846FEF7C0FC0146674833
:10902800FEF727FE95ED070A6846FEF7B7FC0146EE
:109038006248FEF71EFE95ED080A6846FEF7AEFC8C
:10904800013401465E48FEF714FE0C2C05F11005AC
:10905800CAD1AAE05B49052209F0CCFA40B9554BC0
:1090680003F1C0020021596110339342FAD19CE008
:1090780028465549042209F0BDFA04462846002C22
:1090880040D1202109F09FFA002800F08E80451C6D
:10909800284609F0A6FA07464C4B53F824601EB937
:1090A8004B4804F011FD80E028463146FAB209F039
:1090B800A1FA01340028EFD13E4B03F1C0029E46CD
:1090C8000021596110339342FAD1424B03EBC40299
:1090D8009846D2F804C0BCF1000F04D131463E488E
:1090E800FEF7C7FD57E0002718F834309F42F5DA3D
:1090F8003B010EEB030563440FCB143585E80F00E5
:109108000137F1E709F0C4FA0B28064647DC284680
:10911800202109F058FA054650B101352846FEF7D6
:10912800B3FB244B03EB061383ED050A012400E08F
:1091380004462846202109F046FA054648B101357B
:109148002846FEF7A1FB1B4B03EB061383ED060A2B
:1091580001342846202109F036FA054648B1013580
:109168002846FEF791FB134B03EB061383ED070A22
:1091780001342846202109F026FA10B9FCF744FFEB
:1091880013E00130FEF780FB0A4B032C03EB0616B5
:1091980086ED080AF2D11148FFF71CFF05E01048D8
:1091A800104901220C23FEF764FD04B0BDE8F081EC
:1091B800F8660108B411002013670108196701084F
:1091C800AF6B010818650108DC660108C45B01087B
:1091D8008164010880630108E16601087061010883
:1091E800C3620108E2620108284B294A1B68126819
:1091F80010B51A60274A1168596051689268DA6098
:10920800254A996011681961516892689A61234AE0
:1092180059611168D961516892685A62204A196285
:1092280011881985518859859188D288DA851D4A0F
:109238009985118819865188598692889A861A4A7A
:109248001188D986518819871946928821F83A2FAA
:10925800164A10780022824206DA154C34F8124079
:1092680021F8024F0132F6E7124A1288A3F8642067
:10927800114A1288A3F86620104A1288A3F86820B9
:109288000F4A5289A3F85E2010BD00BFE4240020D5
:10929800F02600203C2000204820002054200020F8
:1092A800AC110020FC100020A21100208A20002010
:1092B80018110020101C0020B410002030110020CC
:1092C800021100202DE9F8430E4B93E88003054670
:1092D8000E460024B44213DA7B1933F9140008EB64
:1092E800050333F9142009EB050333F9143013444B
:1092F800022293FBF2F3C01A05F087F90134E9E77B
:10930800BDE8F883E424002070B5472005F0CCF8C8
:10931800174B1B681B0307D5164B174A5B68106869
:109328001B68C01A05F062F9144E154C154D3078BB
:1093380005F05CF923682868C01A05F066F96368C7
:109348006868C01A05F061F90F4B188805F04EF9E6
:109358000E4B188805F04AF90D4B188805F046F9A8
:10936800337823742B68A3606B68E36070BD00BF1B
:1093780038260020E4240020F0260020E6180020EB
:10938800D0240020E8180020E4180020E21800206B
:10939800381100207FB5264C264E274D2749284AEC
:1093A800284B20B128480088B0F5805F31D230883A
:1093B800ADF8040028781E4D91F8201012788DF829
:1093C80006008DF807108DF808201B788DF80930F5
:1093D80001A82946062209F0A5F830B30198BDF87E
:1093E80008302860AB80532005F05EF8208805F02F
:1093F800FDF8A07805F0FAF8E37801932379029351
:1094080001A86379039305F057F80F4B00221A80DF
:109418000BE03088208091F82010287812781B788B
:10942800A070E17022716371DDE704B070BD00BF08
:10943800041D0020A4190020E0180020BC260020EC
:109448004F0A0020B40A00205C260020A0F17D030A
:10945800012B70B504460D460A4E05D830687D21AB
:1094680002F0F0FD84F020043068214602F0EAFDA5
:1094780035B12B881C4404EB142404F0FF042C8021
:1094880070BD00BF941900200A4A13880133138065
:10949800094A136801331360084A138801339BB2E1
:1094A800202B01BF00231380054A138808BF01330E
:1094B800138070475C2600204026002044260020A8
:1094C8004626002038B53A4B1B78083B012B054649
:1094D8000C466BD8452004F0E7FF284604F0E4FF6B
:1094E8000C2D23D004D80A2D0AD014D835B138BD94
:1094F8000E2D4BD02ED3FF2D50D038BD206849E01B
:10950800207804F0D1FF62796378002A14BF8020A4
:109518000020184300E0207804F0C6FFA07804F08B
:10952800C3FFE07804F0C0FF20793BE0B4F9000005
:1095380005F052F8A07804F0B7FFE07804F0B4FF23
:10954800B4F9040005F048F8B4F90600BDE838405D
:1095580005F042B8637820788BB180F0800004F081
:10956800A3FFA468E0B204F09FFFC4F3072004F04F
:109578009BFFC4F3074004F097FF200E12E004F0AD
:1095880093FF6068BDE8384005F03FB8206805F0F3
:109598002DF86068BDE8384005F028B8054804F0A3
:1095A80061FF0020BDE8384004F07EBF38BD00BF31
:1095B800CA240020EF6A01082DE9F04FB54BB64FD9
:1095C8001A888BB00193002A40F09680B7F80E07EE
:1095D800B24D42F20103C11A48424841FFF7DAFE90
:1095E800FFF702FE2C68492004F05EFFAC4B2646CC
:1095F800186804F0FBFF56F8040B04F0F7FF304638
:1096080005F060F904F1100005F05CF904F11C099B
:109618004FF01008A34E0123326803FA08F31342EF
:1096280003D0D9F8000004F0F0FF08F10108B8F100
:10963800130F09F10409EDD104F1280005F032F9FE
:10964800B7F84431B4F92E00C01A04F0CFFF3368DC
:10965800DA0408D5944BB4F864001B88181AC0F3D0
:109668000D0004F0C3FF33689B0403D5B4F866000B
:1096780004F0BCFF3368180403D5B4F8680004F09C
:10968800B5FF04F13000A04605F00CF904F13600EE
:1096980005F008F9B7F8443138F93C0FC01A04F05E
:1096A800A5FF0127814B1B789F4208DA38F9020F82
:1096B800B4F93C30C01A04F0A8FF0137F2E7336868
:1096C800990505D5B4F95E00A0F2DC5004F09DFFC1
:1096D8002A6877486A60AA60121A9110754A4A4344
:1096E800531C032293FBF2F202EB42029A1A6C23F8
:1096F80003FB02032B60ABE16F4B704A1B681168D8
:109708008B4206D00AA9002041F8203D1360FFF7DC
:10971800D9FE019B97F80E171B8897F80F070B4483
:10972800013BB3FBF0F200FB12338B4280F05B810C
:109738005A4D0120FFF72EFEFFF756FD50202F68E7
:109748006E6804F0B1FEAA682B6810681B686A6826
:1097580003441068A3EB400004F057FF72687B686D
:109768009B1A0293B268BB689B1A0393F268FB6862
:1097780002A89B1A049305F0A5F832693B699B1A65
:10978800029372697B699B1A0393BB69B26902A849
:109798009B1A049304F090FE07F11C0B06F11C08B9
:1097A8001024404901220B68A2401A428A4606D07A
:1097B800DBF80000D8F80030C01A04F026FF0134A6
:1097C800132C0BF1040B08F10408EAD107F1260069
:1097D80006F12601002331F9024F30F9022F121B3E
:1097E80002AC44F823200133042BF4D103214FF0B9
:1097F80000094FEA89035FFA83F902AB53F8212085
:109808006AB102F108000F2802D849F0010906E000
:109818008032FF2A94BF49F0020949F0030911F187
:10982800FF31E6D2484604F03FFE00240DF1080B54
:10983800A04609F00302022A16D0032A1DD0012AE5
:109848004FD1B8F1000F05D1DBF800402401E4B294
:10985800904646E0DBF8000000F00F00204304F0DB
:1098680023FE4FF000083CE0B8F1000F0CD0DBF805
:109878000000C0F3031020432DE0B8F1000F1FD102
:109888009BF8010004F010FE9BF8000004F00CFEA9
:1098980027E000BF44260020B4110020E424002063
:1098A8004026002038260020342600208A20002068
:1098B800F024002013DA4B684C26002048260020AC
:1098C800DBF80000C0F30330204304F0EDFDDBF8C3
:1098D8000000C0F3071004F0E7FDDBF800402401A6
:1098E800E4B20BF1040B06AB9B454FEA9909A0D1F2
:1098F800B8F1010F02D1204604F0D6FDDAF80030A5
:1099080013F480541FBFB7F86420B6F86410521AD5
:10991800029218BF01249A040AD50AAA02EB84010C
:10992800B6F86600B7F86620121A41F8202C013400
:1099380018040BD50AAB03EB8402B6F86810B7F825
:1099480068305B1A42F8203C013400E0FCB1012C7D
:1099580003D1029804F059FE19E0631E002002AA00
:10996800400052F82320C0B20AB140F00100013B88
:10997800F5D504F099FD4FF0000802AB53F8280024
:1099880008B104F042FE08F10108A045F5DB3020DB
:109998000321FFF797FC36200321FFF793FC2F4B99
:1099A8003C201978FFF78EFCDAF80030990506D5C7
:1099B800B7F95E00B6F95E30C01A04F026FE2A68D0
:1099C80027486B686A60121A9110264AAB604A43AE
:1099D800531C032293FBF2F202EB42029A1A6C2305
:1099E80003FB02032B60204B1B681A0630D51F4C63
:1099F8001F4D22682B689A420BD162686B689A42A5
:109A080007D1019B1B88102B11D11A4B1B885B06B1
:109A18000DD1482004F048FD206804F0F6FD606888
:109A280004F0F3FD23682B6063686B600EE0124A54
:109A38000F4B11782A7C914208D1104A9968106816
:109A4800884203D15268DB689A4201D0FFF75CFC78
:109A580004F0FAFC0BB0BDE8F08F00BF8A200020AC
:109A6800F024002013DA4B68702600203C110020F7
:109A7800D024002046260020E6180020E818002000
:109A88002DE9F84F0C9E3A4CC2EB030B0B9BF61AD0
:109A98006368002914BF4FF0060A4FF0040A013327
:109AA8000546904613D1236853455ED2314A324861
:109AB80052F82320032B98BF294604F0E3FC63687F
:109AC800013363602D4B002205469A7113E000258F
:109AD80011E02B4A1278954240DA0B9BE3B109FB5F
:109AE80006F2995C01228A40264909680A4213D184
:109AF800636801336360D4F804900A9B1C4F99454E
:109B0800E7DB2BD10A2004F0CFFC3B6801333B6034
:109B18004FF0FF337B6021E0184A917921B12C2066
:109B280004F0C2FC013501E001219171226809FBB2
:109B38000BF308EB030752B958F8030004F092FC42
:109B480097F904104B1C0544D2D00F4802E03A4460
:109B58000E48117904F096FC0544C9E72068504581
:109B68002CBF00200120BDE8F88F0020BDE8F88F49
:109B780050260020104D0108FA6A0108041D002033
:109B88000801002038260020096B0108C76B01086E
:109B980030B585B004AC002524F8025D0091ADF81D
:109BA800060021461020FFF751FC9DF806002146CB
:109BB800FFF74CFC9DF807002146FFF747FC9DF88E
:109BC80000002146FFF742FC9DF801002146FFF7FF
:109BD8003DFC9DF802002146FFF738FC9DF8030084
:109BE8002146FFF733FC9DF80E00C043C0B229465A
:109BF800FFF72CFC05B030BD10B5054C206802F00D
:109C08001EFA18B1206802F017FAF6E710BD00BF77
:109C18006419002013B5044601A9006803F094F8FC
:109C2800132003F0CDF8BDF9040003F0B7F81B20AA
:109C380003F0C6F8BDF9060003F0B0F8232003F0DE
:109C4800BFF82368002BB4BF53204E2003F0A6F8BA
:109C580001A9606803F078F8122003F0B1F8BDF9A3
:109C6800040003F09BF81A2003F0AAF8BDF90600D7
:109C780003F094F8222003F0A3F86368002BB4BF24
:109C88005720452003F08AF802B010BD064B1B7818
:109C980003F0040303F0FF001BB1044B1888C0F362
:109CA800C01000F00100704710270020A419002000
:109CB8002DE9F04F2DED028B87B000260493C14BA0
:109CC8000391B3F90280B3F900300292B8F1000FA2
:109CD800B8BFC8F10008002BB8BF5B429845B8BFB1
:109CE8009846B8F5FA7F0746A8BF4FF4FA7800906F
:109CF800B2460196B1463446B34D2B88990757D0E2
:109D0800B04BB24A33F8143032F91420022013FB56
:109D18000022029B5B429A424FEA440103DB029B0A
:109D28009342A8BF1346AA4A31F902B0049A32F9FD
:109D38001420CBEB030303EB020BFFF7A7FF88B15B
:109D480007EE90BAA34BB8EEE70AB2EE048A185DA4
:109D580080EE080A05F00AF920EE080AFDEEC07A3E
:109D680017EE90BA3B7A642203FB0BF393FBF2F3F2
:109D78003A7F6FF0040909FB02F94B4504DB02EB5B
:109D880082099945A8BF9946934A52F824100BEBCB
:109D9800010342F210718B42A8BF0B468F498B42D8
:109DA800B8BF0B4642F82430BA7C53431B130193C7
:109DB8002D8805F00303012B38D0824B884933F9ED
:109DC80014A0009B51F824E093F801C0854B33F9A7
:109DD800140080EAE073A3EBE073B3F5206F4FEA59
:109DE800840616DC0AEB8A031A0192FBFCF30422B0
:109DF80090FBF2F0181A8644BEF57A5FA8BF4FF4BC
:109E08007A5E794B9E45ACBF41F824E041F8243096
:109E180002E0002341F824308B597D2693FBF6F6A7
:109E2800009BDB7A7343402693FBF6F6AA0711D50D
:109E38000198C8F5FA7208FB0AF308FB06F54FF417
:109E4800FA7102FB093302FB005593FBF1F395FB12
:109E5800F1F505E0EB074DBF019D354653464B46EE
:109E6800604A32F91410042291FBF2F25F49615CF6
:109E78004A436FF04F0192FBF1F297F851101344E7
:109E88004FEA440B08EE103A59B1594B5948D3EDF3
:109E9800000AB8EEC80A00EBC400FDF7CBFCBDEE23
:109EA800C08A504B544A3BF803003BF902302BF868
:109EB800020001B2101D0C32CB1A50F824E0042124
:109EC80093FBF1F152F8243040F8241073440B440A
:109ED80097F8501042F824E04FEA840C00EE103A4C
:109EE80079B1434A4548D2ED000ACDF814C0B8EE1E
:109EF800C00A00EBC400FDF79DFCDDF814C0BDEE00
:109F0800C00A3F4A3F49125D3F4810EE103A53439A
:109F1800202293FBF2F318EE102A2A44D21A2BF8C7
:109F2800012018EE102A4CF80020384A4CF802504C
:109F3800374D5B424CF80530009B013300930CB958
:109F48000124D9E61F4B97F80DE0B3F90440039BB1
:109F58009B790F335B0063435B11224C002B4FF05E
:109F68000406B4F9044094FBF6F41D4EA3EB040474
:109F7800B8BF5B42322BD6F808C00DDC254B0EFB70
:109F880004CE7345A8BF7346DFF890E07345ACBFB5
:109F9800B360C6F808E001E00023B360FB785C43D7
:109FA8001D4B1B78032B4FEAA4143AD9B7F84E304F
:109FB800B3F5FA7F35D25F42BC4231DB9C42A8BF81
:109FC8001C462EE0AC110020A41900200A2700200E
:109FD80066260020284D01080C1D0020F0D8FFFF40
:109FE800EC1F0020FC10002080C1FFFF842000200F
:109FF800E81F0020D01F0020141D00201C20002076
:10A0080087200020342000203C2000204820002009
:10A0180054200020FEFFFF0F8A200020020000F0DD
:10A028003C46B368846043F34F33B3F5807FA8BFE1
:10A038004FF480736FF0FF06B342B8BF3346E6189B
:10A04800936000238E80AB6007B0BDEC028BBDE847
:10A05800F08F2DE9F04F2DED028B85B083460293EA
:10A06800B84B01911D88009205F00205ADB295B17B
:10A07800B54BB3F90250B3F90030002DB8BF6D42AB
:10A08800002BB8BF5B429D42B8BF1D46B5F5007FA7
:10A09800A8BF4FF40075D9460026AB4BAB4C33F83C
:10A0A8001610AB4B54F8267033F9163083EAE37E6A
:10A0B800AEEBE37E08B2BEF5206F4FEA460A4FEAE0
:10A0C80040004FEA860812DC4FF0040E93FBFEF3C3
:10A0D800C31A1F44B7F57A5FA8BF4FF47A579D4B50
:10A0E8009F42ACBF44F8267044F8263002E00023B3
:10A0F80044F8263054F8087099F80B3099F8014064
:10A10800FF115F438F4B1B8844439B074FEAA717F8
:10A118004FEAA41456D0904B33F90A30022011FBB1
:10A128000031009B5B42994203DB009B8B42A8BF36
:10A138000B468A493AF90110591A029B33F916302D
:10A14800CB1808EE103AFFF7A1FD68B1B8EEC80ABF
:10A15800834BB2EE048A80EE080A985D04F006FF8D
:10A1680020EE080ABDEEC08A7E487F4958F80030C4
:10A1780018EE102A42F2107E13447345A8BF7346A6
:10A188008B42B8BF0B4648F800309BF808109BF884
:10A198001C00514300EB8000C911C0F1000E71454D
:10A1A80003DB8142A8BF01468E469BF812104B4341
:10A1B8001B13FF1ACEEB04046F436C4303EB6727B2
:10A1C8000EEB6424624B04213AF9030090FBF1F191
:10A1D8006648805D4143A4EBA1129BF8511008EE3C
:10A1E800102A69B16248634C0393B8EEC80A00EBC1
:10A1F800C600D4ED000AFDF71DFB039BBDEEC08A27
:10A208005D4933F80A303AF901002AF801300FFAAB
:10A2180083FEC0EB0E0E04209EFBF0F001F1040E4D
:10A228000C3158F80E4058F8013048F801402344E2
:10A238009BF8501048F80E00034400EE103A59B14C
:10A248004C4B4E48D3ED000AB8EEC00A00EBC600EE
:10A25800FDF7F0FABDEEC00A49494A48895D4A4C03
:10A2680010EE103A18EE102A4B435B11D119C91A97
:10A278002AF8001048F804204449454A48F8017073
:10A288005B4248F8023009F101090EB9012604E7DA
:10A298002D4B2E4EB3F90450019BD6F808E09B795C
:10A2A8000F335B006B435B11294D002BB5F904504C
:10A2B8004FF0040795FBF7F7A3EB0707B8BF5B421E
:10A2C800322B9BF80D500BDC324B05FB07E5AB42FC
:10A2D800A8BF2B46304DAB42ACBFB360B56001E0C0
:10A2E8000023B3609BF8035005FB07F32B4D2D7833
:10A2F800032D4FEAA3130CD9BBF84E50B5F5FA7FDE
:10A3080007D26F42BB4203DBAB42A8BF2B4600E03B
:10A318003B46B568A36045F34F35B5F5807FA8BFC8
:10A328004FF480756FF0FF06B542B8BF35465E1929
:10A33800002386808D60936005B0BDEC028BBDE87C
:10A34800F08F00BFA4190020AC110020EC1F0020E2
:10A35800FC10002080C1FFFF0A270020662600208D
:10A36800284D01080C1D0020F0D8FFFF8420002094
:10A37800D01F0020E81F0020281D00201C200020DE
:10A3880087200020342000203C2000204820002086
:10A3980054200020FEFFFF0F020000F08A2000205A
:10A3A8002DE9F04F2DED028B87B000260493B24BB8
:10A3B8000392B3F90270B3F900300190002FB8BFCF
:10A3C8007F42002BB8BF5B429F42B8BF1F46B7F51C
:10A3D800FA7F8146A8BF4FF4FA77B0460296B34693
:10A3E8003446A64D2B8899075BD0022C59D0A24B36
:10A3F800A34A33F8143032F91420022013FB002248
:10A40800039B5B429A424FEA440103DB039B93425E
:10A41800A8BF13469B4A31F902A0049A32F91420C6
:10A42800CAEB030303EB020AFFF730FC88B107EE1F
:10A4380090AA954BB8EEE70AB2EE048A185D80EE52
:10A44800080A04F093FD20EE080AFDEEC07A17EE24
:10A4580090AA99F80830642203FB0AF393FBF2F3FD
:10A4680099F81C206FF0040B0BFB02FB5B4504DB27
:10A4780002EB820B9B45A8BF9B46844A52F82430C6
:10A4880042F2107153448B42A8BF0B4680498B425D
:10A49800B8BF0B4642F8243099F8122053431B13D7
:10A4A80002932B8803F00302012A01D1022C3FD129
:10A4B8007848714A30F9140032F914807649019AC3
:10A4C80051F824E0567880EAE075A5EBE075B5F51B
:10A4D800206F4FEA84021EDC022C16D008EB88019C
:10A4E800090191FBF6F6042190FBF1F0361AB64407
:10A4F800BEF57A5F68496948A8BF4FF47A5E864519
:10A50800ACBF42F801E0505007E088EAE875A5EBD7
:10A51800E875642DE2DD002088505F497D26525899
:10A5280092FBF6F6019AD27A7243402692FBF6F62F
:10A538009A0713D5022C11D00298C7F5FA7307FBB6
:10A5480006F507FB08F203FB0B224FF4FA7103FB35
:10A55800005392FBF1F293FBF1F508E0DB0704D519
:10A56800022C02D0029D5A4601E035464246494B2C
:10A5780033F91410042391FBF3F34949615C4B430D
:10A588006FF04F0193FBF1F399F85110D3184FEA8C
:10A59800440A08EE103AB1B1022CB8EEC80A414B91
:10A5A80008D14A0803D09142A8BF114600E0012112
:10A5B8003D4802E03D4800EBC400D3ED000AFDF73A
:10A5C80039F9BDEEC08A334B394A3AF803003AF9F3
:10A5D80002302AF8020001B202F108001432CB1A44
:10A5E80050F824E0042193FBF1F152F8243040F8AC
:10A5F800241073440B4499F8501042F824E04FEAB1
:10A60800840C00EE103A79B1264B2A48D3ED000AA3
:10A61800CDF814C0B8EEC00A00EBC400FDF70AF983
:10A62800DDF814C0BDEEC00A234A2449125D10EEBD
:10A63800103A5343202293FBF2F318EE102A2A44CF
:10A64800D21A2AF801201E4A18EE101A4CF80210E5
:10A658001C4A4CF802501C4A5B424CF80230019BE1
:10A6680001340133032C01937FF4BBAE07B0BDEC7A
:10A67800028BBDE8F08F00BFAC110020A4190020A8
:10A688000A27002066260020284D01080C1D0020FE
:10A69800F0D8FFFFFC100020EC1F002080C1FFFF56
:10A6A80084200020E81F0020E01F0020D01F002089
:10A6B8003C1D00201C200020872000203420002082
:10A6C8003C20002048200020542000202DE9F04F95
:10A6D8002DED088BC94F83B0044600933B88019742
:10A6E80013F0020F0AEE102AF7EE009A4CD0149BD2
:10A6F800C348DD89B0F900305B1B03F2F31640F262
:10A70800E632964203D8002BB8BF5B4201E04FF413
:10A71800FA73B0F90220521B02F2F31540F2E63048
:10A72800854203D8002AB8BF524201E04FF4FA72BA
:10A7380094F84C0058B39342B8BF1346C3F5FA7364
:10A7480007EE903A9FEDAF7AF8EEE77A6423C7EE0A
:10A75800877A93FBF0F307EE103A77EEE97AB8EED2
:10A76800C77AB0EE699AA7EE879AF7EE006AB5EE57
:10A77800C09AF1EE10FA0AD4B4EE669AF1EE10FA25
:10A78800C8BFB0EE669A04E0B0EE699A01E09FEDAA
:10A798009E9ACE1C25464FF0000ABAF1020F16F811
:10A7A80001BF9A4F4FEA4A09F2EE04AA0ED1B7F94F
:10A7B80004209FED977A0BF10A0B02FB0BF307EECF
:10A7C800903AF8EEE77AC7EE877A68E0F8EE4A7AC8
:10A7D8009FED8C6A37F91A30C7EE867A06EE903A02
:10A7E8008C4B33F91A3007EE103A1AEE103AF8EE9D
:10A7F800E66AB8EEC77A5B42A6EEA77A07EE903A09
:10A80800F8EEE77AB4EEE77AF1EE10FA08D4F8EE4B
:10A81800CA7AB4EEE77AF1EE10FAD8BFF0EE477ACA
:10A828007D4B33F9093008EE103A009BB8EEC88A20
:10A8380033F91A3077EEC87A08EE103AB8EEC88ABB
:10A8480037EE888A88EE2A8AFFF720FA40B1734BE0
:10A8580013F80A00B0EE480A04F088FBB0EE408A0C
:10A86800019B1A88D10704D5D4ED117A68EE277AAE
:10A8780015E037F909309FED667A0BF1140B03FBED
:10A888000BF307EE903AF8EEE77A9307C7EE877A6C
:10A8980042BF94ED127A28EE078AE8EE097A604BF7
:10A8A800DFF8ACB133F9093095ED08BA9FED5D8A50
:10A8B80094F85110DFF89C8107EE103A5A4BB8EE25
:10A8C800C77AD3ED186A1AF80B30E7EE667AF0EE1D
:10A8D80048BAF0EE678A67EE8B7A0BEE103AB8EE5C
:10A8E800CBBA27EE8BBA8BEE08BAC1B1BAF1020F18
:10A8F8000AD14B0803D09942A8BF194600E00121AC
:10A90800B0EE4B0A494804E04948B0EE4B0A00EB68
:10A91800CA00D8ED000AFCF78DFFB0EE40BAD8EDBA
:10A92800000A444995ED0B7A4FEA8A0768EEA07A47
:10A93800394467EE877A91ED007AA7EEAA7ADFEDBF
:10A948003E7AB4EEE77AF1EE10FAF0EE47AA09D4AF
:10A95800DFED3A7AB4EE677AF1EE10FAC8BFF0EE9E
:10A9680067AA01E0F0EE67AA89EEA07A344AC1ED41
:10A9780000AAD119D1ED007AC1ED008A78EEE77A04
:10A9880002F10C013944183267EE877A3A4491EDA6
:10A99800007A92ED000AC1ED007A82ED007A37EE76
:10A9A800000A94F8501030EE270A21B1254800EB30
:10A9B800CA00FCF73FFFF0EE087A80EE270A1BF882
:10A9C8000A30D5ED0E7A08EE103A60EE277AB8EE26
:10A9D800C88A27EE880ADFED1C7A80EE2B8AB4EE4F
:10A9E800E78AF1EE10FA37D4DFED187AB4EE678A09
:10A9F800F1EE10FAC8BFB0EE678A2FE0A419002064
:10AA0800101B00200000FA4300000000AC110020D9
:10AA1800000048420A27002066260020284D010829
:10AA2800FC1000200000C8420C1D0020E01F002080
:10AA3800D01F00207020002000007AC300007A4355
:10AA4800701D00201C200020000096C300009643C3
:10AA5800CC1F0020E81F0020B0EE678A3BEE2A0AD0
:10AA68000AF1010A30EE080A07F086FF144AB0F529
:10AA78007A7FA8BF4FF47A709042B8BF1046BDEEF7
:10AA8800CBBA104A1BEE103A22F80900FDEEEAAAEA
:10AA98000D4ABDEEC88ABB500C4A1AEE903ABB501C
:10AAA8000B4A18EE103ABAF1030FBB5005F1040532
:10AAB8007FF473AE03B0BDEC088BBDE8F08F00BF28
:10AAC80018FCFFFF342000203C20002048200020F4
:10AAD80054200020044B00221A605A60034B0022C5
:10AAE8001A605A60704700BF0C1D00207C200020AF
:10AAF80010B50C4C0123E3704FF48060022384F8F6
:10AB08002030FDF7FBF9084A084BD2F888201B686B
:10AB18005178642212FB0133636123880133238057
:10AB280010BD00BFBC2600200C1D0020942600206C
:10AB380007EE900AF8EEE77ADFED0C6A9FED0C0A53
:10AB4800F5EEC07AF1EE10FAD4BFB1EE677AC7EE2F
:10AB5800A67A08B5D8BFC7EE267A27EE800AFDF791
:10AB680019F9044B83ED000A08BD00BF8096184B05
:10AB780035FA8E3C6C0000202DE9F0410369C76866
:10AB880005460E461F40002F35D0B7FA87F24FF022
:10AB98000043D340DB432B611F40A2F11B03042B6E
:10ABA800F1D8DFE803F0221F1C190300746A24B1EE
:10ABB800013C0023A4B2736201E0EC6AA4B2D6F8A7
:10ABC8002080B8F1000FDED0D8F80030404621468A
:10ABD8009847D8F80480F4E73068696B07E0706834
:10ABE800A96B04E0B068E96B01E0F068296C0368C0
:10ABF80089B29847C7E7BDE8F081F8B5994B1B685B
:10AC08000546187818B1012800F06181D9E2242D91
:10AC1800954C0CD006D80A2D00F0D7800D2D00F0E9
:10AC2800D4803FE12A2D06D02C2D04D03AE12070A3
:10AC38006070A07047E18D4B617827788A4A0020C0
:10AC480058542FBB1978D770472921D159785029E2
:10AC58001ED19978472907D1D978472904D119797C
:10AC6800412901D10121D1709978804A522903D113
:10AC7800D1784D2900F0A78299787C4A472907D1D5
:10AC8800D178532904D11279562A04BF0322E270DD
:10AC9800E278754E022A38D0032A4BD0012A40F0B8
:10ACA8008380BA1E072A7FD8DFE802F004080F1352
:10ACB8001A257E2A04F0E8FA606075E01B78532BA9
:10ACC80072D163685B4263606EE004F0DDFAA060F5
:10ACD8006AE01B78572B67D1A3685B42A36063E0E7
:10ACE8001B78302B624B1A788CBF42F0020222F09C
:10ACF80002021A7058E0002004F026FB207353E08B
:10AD0800002004F021FBE0814EE0072F06D0082F39
:10AD18004AD1012004F018FB708245E0012004F0BC
:10AD280013FB41F2184358434FF47A73B0FBF3F026
:10AD3800308239E0022F07D0032F0AD1002004F017
:10AD480003FB4C4B18702FE0002004F0FDFA30751F
:10AD58002AE029D93A1F9210337D0132D2B2013B41
:10AD680002EB8303DBB2102B1ED8F91EC2F10102DD
:10AD780001EB8202D2B2012A0BD0042A11D10020A1
:10AD88005E1E04F0E1FA3C4B98553C4B00229A5564
:10AD980007E05E1E3A4A0020935504F0D5FA394B75
:10ADA8009855A3690133A3612F4B2A2D18BF9A78B0
:10ADB80007F101074FF000000CBF01225540277032
:10ADC80060700CBF1A779D707DE0207F002846D008
:10ADD8002D4B13F8012D2D495A708B42F9D1234A76
:10ADE800214D13785278402B85BF373B1B011B013F
:10ADF800DBB298BF03F0F003402A8CBF373A303AF1
:10AE0800D2B21344A278DBB29A4225D121230B7027
:10AE1800E8782B6A1D4A013301282B620AD00228E0
:10AE28001CD1722313701A4B2A8A1A80194B6A8A0A
:10AE38001A8013E0672313700D4B1B789F070ED5FC
:10AE4800154B6A681A60AA685A60144B2A7B1A70F4
:10AE5800134BEA891A8002E03F230B70002000237D
:10AE6800237730E0A4010020981D00209C260020B4
:10AE7800E0180020501100208111002071110020DD
:10AE88005111002061110020FC090020E809002070
:10AE9800E218002038110020E8180020E6180020E9
:10AEA800E41800206378207F0E2B9FBFAA4A591C04
:10AEB8005170AA4A98BFD554A74A18B993785D40EB
:10AEC800957000E00020003018BF0120F8BDA24BAB
:10AED80093F824100022082900F27381DFE801F0BA
:10AEE800050C101A2B3B5F7B8800B52D40F069815B
:10AEF80083F8252001224FE0622D08BF02224BE093
:10AF0800032283F8242083F8265083F8275083F8F7
:10AF1800285056E1042283F8242093F8272093F838
:10AF2800281083F829502A44D2B283F827200A44EB
:10AF380083F8282045E1052283F8242093F8272068
:10AF480093F828105D852A44D2B283F827200A4452
:10AF580083F8282035E1062283F8242093F8272057
:10AF680093F828102A44D2B283F827200A4483F899
:10AF780028205A8D02EB0525ADB2B5F5AC7F88BF08
:10AF8800754A5D8584BF012182F8251000229A85C3
:10AF9800002D40F01681072283F8242011E193F850
:10AFA800272093F828102A44D2B283F827200A448D
:10AFB80083F828209A8DB2F5AC7F3CBF6649891882
:10AFC80002F1010238BF81F83050598D92B2914296
:10AFD8009A85E0D9F5E0082283F8242093F82730F1
:10AFE800AB4200F0EE805C4B012283F825200FE095
:10AFF8005B4C83F8242014F8012D6270594A94425E
:10B00800F9D193F82810544AA94206D03F23237057
:10B01800554A536801335360D3E0116A92F825000A
:10B028000131116210B13E232370CAE02121217041
:10B0380092F82910062941D004D8022907D00329FB
:10B0480023D0F8BD122959D0302967D0F8BD502136
:10B0580021704649546B4C60946B0C60116C4FF432
:10B068007A7491FBF4F1424C218092F88811414A9C
:10B0780019B1117841F0020102E0117821F00201C2
:10B088001170012283F889218DE05321217092F8F3
:10B098003510CE0705D592F83420D51E6A426A418C
:10B0A80000E0024602F0010183F88811002A7AD1F3
:10B0B80030490A7822F002020A7074E04F212170A8
:10B0C80092F83B10CC0705D592F83A20D11E4A4297
:10B0D8004A4100E0024602F0010183F8881122B9D2
:10B0E80024490A7822F002020A70234A93F85F1072
:10B0F8001170224AB3F85C10118054E05621217077
:10B108001F49546C0C8042F21074916C91FBF4F15D
:10B118001C4C2180012182F88A1144E049212170C8
:10B1280092F83410184A102988BF10211170174955
:10B1380014780022A24233D2154D0E7A5655154D79
:10B148004E7A5655144DCE7A5655144D11F80C6F4B
:10B1580056550132EEE700BF981D00209C260020BE
:10B16800FC090020E809002084010020E8180020DC
:10B17800E4180020E0180020E6180020FE00002057
:10B18800E21800203811002050110020C81D0020AE
:10B19800511100206111002071110020811100203F
:10B1A8009A6901329A6193F889310B4A93B192F8FE
:10B1B8008A317BB1002182F8891182F88A111846F8
:10B1C800F8BD0020F8BD1279432A7FF455AD02225C
:10B1D800E27051E5F8BD00BF981D00200449054BF9
:10B1E8000968187000225A6199611A77704700BF80
:10B1F800942600208401002010B5121A07EE902A28
:10B208005B1A2DED028BF8EEE78A07EE903A184BA1
:10B21800059CB8EEE78AD3ED007A28EE278A28EE57
:10B22800080AA8EEA80A07F0ABFCDFED127A049B27
:10B2380020EE270AF0EE480ABCEEC00A83ED000AA9
:10B24800B1EE680A07F09AFCDFED0B7A9FED0B7AF6
:10B25800E0EE077ABDEC028BFDEEE77A17EE903A46
:10B26800002BBCBF03F50C43A033236010BD00BF07
:10B278006C0000202C7D8E3F00A00C46A00CB3452E
:10B2880044F25063984203DDA0F50C40A0387047A3
:10B29800034B9842BCBF00F50C40A030704700BF7C
:10B2A800B0B9FFFF73B51A4C036823600B6863607D
:10B2B800184D0068184EFFF73BFC184B009395E8B3
:10B2C800030094E80C000196FFF796FF144B3268D0
:10B2D8001A606868636813491B1A07EE903A124BA4
:10B2E800286893ED007A23681B1A0B600F4BF8EE61
:10B2F800E77A1A600E4B67EE877A1B68FDEEE77AED
:10B30800DA880C4BC1ED017A1A8002B070BD00BF1B
:10B31800EC220020E8180020F8220020F422002067
:10B3280034230020FC2200206C0000202C23002065
:10B33800100B0020282300204279DFED2A5A2A4BDF
:10B348009FED2A5A07EE902AF8EE677AC27BC7EE7D
:10B35800A57AB2EE047AC3ED007A07EE902AF8EEE9
:10B36800677A234ADA60C7EEA57AC3ED017A817954
:10B37800204B07EE901AF8EE677A017CDA60C7EE88
:10B38800877AC3ED007A07EE901A817E06EE101ACE
:10B39800F8EE677AB8EE466AC7EEA57A86EE056AD1
:10B3A800C3ED017A83ED026AC179134B06EE901A58
:10B3B800417CDA60F8EE666AC6EE876A07EE101A14
:10B3C800C17EC3ED006A07EE901AB8EE477AF8EE30
:10B3D800677A87EE257AC7EE857A83ED017AC3ED21
:10B3E800027A70470000C8420423002000007A4413
:10B3F8000000FA44142300203823002010B50C4C18
:10B4080023789B0713D50B4B1B78042B0FD90A4ABB
:10B418000A4B106852685A601860FFF789FB084B9E
:10B428001A88084B1A80237843F00103237010BD53
:10B43800E0180020E6180020E81800203C11002041
:10B44800A8110020482300201C4B1B681B0307B5CC
:10B4580030D51B4A1B4BD2ED007A1B788DF8003093
:10B46800B2EE047A67EE877A174B9FED187A1B784D
:10B478008DF80130FCEEE77A0A2017EE903AD2ED0B
:10B48800017A8DF8023067EE877A6946FCEEE77A32
:10B4980017EE903AD2ED027A8DF80330FCEEE77A97
:10B4A80017EE903A8DF80430094B1B788DF805306B
:10B4B800FEF708F803B05DF804FB00BF7026002013
:10B4C80084260020602600208026002000007A4480
:10B4D80064260020054A137883F001031370044A98
:10B4E80000231360034A1360AEE700BF6426002000
:10B4F8007C2600207826002001480249FFF73CBB43
:10B5080000480140B421002001480249FFF734BB3C
:10B51800004001406421002001480249FFF72CBB8C
:10B52800000800403C21002001480249FFF724BBE5
:10B5380000040040142100204FF080400149FFF72B
:10B548001BBB00BFEC20002010B5064C0648214666
:10B55800FFF712FB04F1C8010448BDE81040FFF7EB
:10B568000BBB00BFC4200020002C01400044014058
:10B5780001480249FFF700BB002C0140C42000200D
:10B58800224B10B5224C5A43224BB3FBF2F20388EC
:10B598000139013AA04289B292B29BB20ED004F5A9
:10B5A8000064A0420AD0B0F1804F07D0A4F59834C7
:10B5B800A04203D004F58064A04202D123F07003B6
:10B5C8009BB2154CA04206D004F58064A0421CBF73
:10B5D80023F440739BB203800D4BC16298420285ED
:10B5E8000FD003F5006398420BD003F540639842EF
:10B5F80007D003F58063984203D003F5806398422F
:10B6080001D1002303860123436110BD40420F008E
:10B61800002C014000A24A0400100040134B800A8D
:10B62800984220D00AD84A3B984212D00133984217
:10B6380011D0B0F5801F14D1012070470C4B9842EF
:10B648000BD0013398420AD0023B984209D104201A
:10B658007047022070470320704705207047062076
:10B668007047FE2070470020704700BF4B00100055
:10B6780051001000F8B50468064620460F461546E6
:10B68800FFF7CCFF06284BD8B27A910847B90223B6
:10B698008B40D4F80CE0DB439BB203EA0E03E36073
:10B6A8000A23204A03FB001342F82370043342F8AC
:10B6B800235015463FB1B17AE268890802238B40CE
:10B6C8009BB21343E360282202FB00522032EFF3BF
:10B6D8001286502383F3128803B203EB8303DB0043
:10B6E80003F10C011C3329442B4451F8047F17B192
:10B6F80017600A6804329942F7D100231360F3B245
:10B7080083F31188282303FB0050036A1BB1E36805
:10B7180043F0010303E0E2684FF6FE731340E36071
:10B72800F8BD00BFC42000200148F7F7CDB800BF1E
:10B73800241F00200148F7F7C7B800BF781F002072
:10B74800034B4FF4806208B19A6170471A857047BD
:10B7580000040048034B4FF4806208B11A85704713
:10B768009A617047000400482DE9F04F2DED028BD7
:10B7780085B007460293A04B1B889807934636D599
:10B78800109B9E48DC89B0F900301B1B03F2F315AF
:10B7980040F2E632954203D8002BB8BF5B4201E085
:10B7A8004FF4FA73B0F90220121B02F2F31440F2BC
:10B7B800E630844203D8002AB8BF524201E04FF471
:10B7C800FA729342B8BF1346C3F5FA73052293FB86
:10B7D800F2F30A22643B53433A7FD2105343642264
:10B7E80093FBF2F3134423EAE373DBB200E0642330
:10B7F8000093CB1C0193B8460024019BDFF824A2D8
:10B8080013F8016F0193022C4FEA440905D1BAF9E4
:10B8180004301B365E43761146E079493AF8142025
:10B8280031F91410022012FB0011CBF100029142F1
:10B8380003DB59450A46A8BF5A467249029B31F9AB
:10B848000950551B33F914201544FEF71FFA88B127
:10B8580007EE905A6C4AB8EEE70AB2EE048A105D19
:10B8680080EE080A03F082FB20EE080AFDEEC07A9B
:10B8780017EE905A604A1288D10712D43AF9093063
:10B888001B365E4393074FEA26160DD5BB7C5D43F6
:10B898009DF900305D43642395FBF3F506EB25160F
:10B8A80002E03E7A75432E11584B042533F90930CE
:10B8B80093FBF5F5564BE25C924698F80120751B10
:10B8C80051466A434A43642192FBF1F297F85110BA
:10B8D800D21108EE102AA9B1022CB8EEC80A08D174
:10B8E8004A0803D09142A8BF114600E00121494807
:10B8F80002E0181D00EBC400D3ED070AFBF79AFF1E
:10B90800BDEEC08ADFF808E1434B98F80B60188851
:10B918000EF1200300FB05F253F82410D21206FBA7
:10B928000216B6F5001F3D4AA8BF4FF4001696420E
:10B93800B8BF16460EF12C0243F8246052F82430A2
:10B9480042F82450EB1A0EF138014FF6FF72000945
:10B95800B2FBF0F043430EF1440051F8245050F884
:10B96800242040F824509B112A4441F8243097F8A9
:10B9780050101A444FEA840C761300EE102A79B15D
:10B988000EF15000B8EEC00A00EBC400DEED070A65
:10B99800CDF80CC0FBF74EFFDDF80CC0BDEEC00AB9
:10B9A80098F8153010EE102A18EE101A5A4353461C
:10B9B80053431A463144642392FBF3F3184A1B128B
:10B9C800194422F8091018EE100A02F1080101348E
:10B9D8004CF8010002F114012032032C4CF80160EC
:10B9E8004CF8023008F101087FF407AF05B0BDEC50
:10B9F800028BBDE8F08F00BFA4190020101B0020A7
:10BA08000A27002066260020284D0108FC10002087
:10BA1800CC1F0020E01F0020D01000200000E0FF15
:10BA280034200020AC1100202DE9F04F2DED0A8BB9
:10BA380085B08346039390F85030029101921BB170
:10BA4800322BA8BF322300E0012307EE903AF8EE2C
:10BA5800E7BADFEDDE7ADE4B9FEDDECA1B88C7EE64
:10BA6800ABBA002B08BF012307EE903AB8EEE7AA5D
:10BA7800D94B2AEE0CCA1B887BEE8CBA9807CCEE01
:10BA88002BBA27D5D54AB2F90030B2F9022083EA99
:10BA9800E37182EAE270A1EBE371A0EBE270884205
:10BAA8000446B8BF0C46B4F5E17F16DA88429FED2C
:10BAB800CCBA05DD002AD8BF524207EE902A04E02E
:10BAC800002BD8BF5B4207EE903AF8EEE77A87EE94
:10BAD8008BBA04E09FEDC3BA01E0B7EE00BAC24EDC
:10BAE800DFEDC09ACDF800B006F1080806F110099C
:10BAF80006F11C050024F0EE69AABC49DFF8D8A2BB
:10BB080031F91430B54909EE103AB8EEC99AF5EE94
:10BB1800047A29EE279A31F91430BAF80010BDEEEC
:10BB2800C99A08EE103AF8EEC97A9FEDB19A8907DA
:10BB38004FEA440727EE899AB8EEC88A00F0818058
:10BB4800AC4931F9143007EE903AF8EEE77AB0EEE6
:10BB5800007AE8EE077A019B5842FDEEE77A17EE85
:10BB6800901A814203DB8B42A8BF0B461846A249B4
:10BB7800039B795E401A33F91410084407EE900AC3
:10BB8800F8EEE78AFEF782F848B19C49F2EE049A8B
:10BB980088EEA90A085D03F0E9F960EE298A9BF8A6
:10BBA8001C30DFED976A0AEE903A9BF8083007EEF2
:10BBB800903AF8EE677AF8EE6AAA68EEA77AB1EEDC
:10BBC800047A67EEA67A2AEE877AFDEEE77A17EE10
:10BBD800901AF1EE477AFDEEE7AA1AEE903A9942EA
:10BBE80008DBFDEEC7AA1AEE903A8B42A8BF0B46B7
:10BBF8000AEE903AD5ED007AE8EE8C7ABBEE0E7A32
:10BC0800F4EEC77AF1EE10FAF8EEEAAA09D4B3EE28
:10BC18000E7AF4EE477AF1EE10FAC8BFF0EE477AE2
:10BC280001E0F0EE477AC5ED007A9BF8123009EE94
:10BC3800903AF8EE699A67EEA97ADFED729A67EEA4
:10BC4800A99ABAF80010CA0753D46848385E002881
:10BC5800B8BF4042B0F5206F03DD0020C9F80000EE
:10BC680026E0009B9FED687A5B7868EE077A07EE1E
:10BC7800103AB8EE477A87EE877AD9ED007A37EE30
:10BC8800497AE7EE0C7A9FED617AF4EEC77AF1EE25
:10BC980010FA09D49FED5E7AF4EE477AF1EE10FAC5
:10BCA800C8BFF0EE477A01E0F0EE477AC9ED007AB6
:10BCB800009BD9ED007ADB7A08EE903AF8EE688AB4
:10BCC8008B0768EEA77ADFED538A67EEA88A14D54A
:10BCD80038EE6A8AF0EE6A7AEBEE087A78EEE98A4C
:10BCE800B0EE678AF0EE697AEBEE287AF0EE678AB2
:10BCF80003E0F0EE698AB0EE6A8A474B9FED477A17
:10BD080003F1B801625C9BF8511007EE902AF8EE37
:10BD1800E77A67EEC97AA7EE878A51B1181DB0EEA7
:10BD2800480A00EBC400D3ED070AFBF783FDB0EE29
:10BD3800408A96ED007ADFF8E0A0D8ED007AA6EC0C
:10BD4800019A39EE477A0AF1BB0187EE0C7A635CF7
:10BD580009F10409043509EE103A37EE677AB8EEAE
:10BD6800C99AEBEE877A38EE280AE8EC017A67EE92
:10BD7800897A9FED2B9A27EE899A30EE490A06F0C8
:10BD8800FBFD0AF16801BDEEC88AC85318EE103AE7
:10BD98000AF17001FDEEE88AB1EE499A41F82430C3
:10BDA800BDEEC99A0AF17C0118EE903A41F82430A8
:10BDB80019EE103A0AF18801574641F82430009BE1
:10BDC8000133009374BB012497E600BF83F9223E38
:10BDD800D0100020BD378635A4190020AC110020F2
:10BDE8000000E1430000000060200020FC1000205B
:10BDF800CDCC4C400A27002066260020284D01089B
:10BE08006F12033C0AD7A33D0000A043000040C3C3
:10BE1800000040430AD7233CCC1F0020A69B443B8C
:10BE2800F7CC9238029A584B9479B3F904306400ED
:10BE380028345C43554BB3F9043000EE103ABAEE9F
:10BE4800CF0A06F099FD6411201A002C07EE900A1B
:10BE5800B8BF6442322CF8EEE76A03DD0023CAF863
:10BE6800283029E0BDEECAAA1AEE103A23F00303DF
:10BE780007EE903AB8EEE7AADFED457A9BF80D3069
:10BE8800CAEE277A07EE103AB8EE477ADAF8283081
:10BE980026EE877A67EE277AFDEEE77A17EE902A84
:10BEA80013443C4A9342A8BF13463B4A9342ACBF53
:10BEB800CAF82830CAF82820BB6A5B13B3F5807F1C
:10BEC800A8BF4FF480736FF0FF029342B8BF1346C8
:10BED80007EE903AF8EEE78AFDEEE67A9BF8032043
:10BEE80017EE903A53439B1107EE903A97F8BE30FD
:10BEF800032BB8EEE78A14D9BBF84E20B2F5FA7FC7
:10BF08000FD2FDEEC87A534217EE901A994204DB1D
:10BF1800914217EE903AA8BF134607EE903AB8EE52
:10BF2800E78A9BF8511079B14B0803D09942A8BF12
:10BF3800194600E00121B0EE480A1848D7ED070A73
:10BF4800FBF778FCB0EE408A38EE280ABDEEC00A4E
:10BF58008DED000ABDF9003000EE103AB8EEC00AC7
:10BF680006F00AFDBDEEC88AFDEEE88A0023A7F8B0
:10BF78006C0087ED1E8AC7ED218AC7F8903005B09E
:10BF8800BDEC0A8BBDE8F08FAC110020FC1000203E
:10BF980000803B45FEFFFF0F020000F0E01F00207D
:10BFA80010B50A4A0A4B11689B6800BF1268914293
:10BFB800F7D1084AD2F8C0404FF47A7000FB04F277
:10BFC800D31AB3FBF4F300FB013010BD9426002014
:10BFD80010E000E0CC1F002038B50446FFF7E0FF72
:10BFE8000546FFF7DDFF401BA042FAD338BD10B568
:10BFF80004462CB14FF47A70FFF7EEFF013CF8E7E6
:10C0080010BD024A1368013313607047942600205C
:10C01800024BD3F8C43003B118477047CC1F002037
:10C02800014B1B68184700BFF426002003681B69F2
:10C0380018470368DB68184703689B681847036854
:10C048005B68184703681B6818472DE9F84FB0F973
:10C058000230934218BF00232DED028B18BF0370E6
:10C06800057804460E469146002D40F08B8007EE79
:10C07800902A9FED770AF8EEE77AB6EE008A27EE67
:10C08800800ADFED747A20EE270AA04620EE080A1F
:10C0980006F0E8FCDFED706A60EE266AB7EE006A2B
:10C0A800B0EE667AA0EE007A40F2DC536365D0EE1B
:10C0B800006A1023A4F8523037EE067A76EE866AC4
:10C0C800C6EE077A1823A4F85030274684ED046A90
:10C0D80027EE807A27EE007A77EE075A84ED017A08
:10C0E800C4ED025A70EE005A84ED037AB8EE007A75
:10C0F800A5EE807A27EE877A67EEA67A84ED057A30
:10C10800C4ED067ADFED557A98ED047A27EE277AA2
:10C11800F0EE678AB5EEC07AF1EE10FA4CBF77EE12
:10C12800487A77EE087A013517EE900A03F040FB5B
:10C13800D8ED017A67EEA87AC7E90E01F5EEC07A64
:10C14800F1EE10FA4CBF77EEC87A77EE887A08F1EC
:10C15800040817EE900A03F02BFB032DC7E908012A
:10C1680007F10807CED1A6F2DC531B042367E36767
:10C178006367C4F88030A367C4F884300123A4F847
:10C1880002902370D4F85490B4F95280636A276AF5
:10C19800206FE26FD4F840C0D4F88010C4F8802033
:10C1A800C9EB060606FA08F64FEAE67B734307FB77
:10C1B8000B332667A7FB06671F44636C656F6067D0
:10C1C8004FEAE27B53430CFB0B3EACFB0223734468
:10C1D800B61A67EB0307E36AA26AC4F884104FEA49
:10C1E800E07B434302FB0B3EA2FB00237344B618DB
:10C1F8005F41E36CA06CB4F95020A5674FEAE17B7E
:10C208004B4300FB0B33A0FB01011944636B361A47
:10C21800206B4FEAE57B05FB03F300FB0B3367EB71
:10C228000107A0FB050119448019794103F096FA2A
:10C2380008F1FF3201239340E067C01841EBE37136
:10C24800424603F08BFABDEC028B4844BDE8F88FF8
:10C258006F12833ADB0F4940F404B53F0000804B6E
:10C268002DE9F8430024244B93F8BE60E0B2B042B5
:10C278000DD203EB8003214AD3F8C83032F81010EE
:10C288001BB10B2801D8DB6898470134EBE71C4B3E
:10C298001B685B032DD500242346E2B2B24228D2A4
:10C2A800DFF8549009F1C8074FEA840857F82420AA
:10C2B80055689D4215D02846FFF7B0F9EFF3128371
:10C2C800502282F3128828216A6A01FB0090013209
:10C2D800C0F81C216A6942F001026A61DBB283F38B
:10C2E800118857F808301B6800221A6001342B4661
:10C2F800D3E7BDE8F88300BFCC1F00201811002049
:10C308007026002008B50E4B1B6813F4805F0D4B98
:10C3180014BFD3F81022D3F8142293F8BE109288D1
:10C328000023D8B2884204D2074820F813200133EA
:10C33800F7E7FFF795FF3220BDE8084057E600BF52
:10C3480070260020CC1F0020181100200A4B1A6804
:10C358000A4B30B502F48052D3F81042D3F8145285
:10C3680000230AB1A18800E0A988054820F8131025
:10C3780001330C2BF5D130BD70260020CC1F0020D6
:10C388004E23002070B5124D0024214605F21920D5
:10C39800702285F8184206F0E0F82146D5F88C326C
:10C3A8000B4A0B4493F9020080B102F219241E686B
:10C3B8000E5108199C8884809B79837192F81832F1
:10C3C80007310133702982F81832E7D170BD00BFF8
:10C3D800CC1F0020094B1A680E2303FB0020437A68
:10C3E800FF2B07D0064A12789A4203D9054A32F839
:10C3F800130000E0808800B2704700BF001D0020D5
:10C4080098240020101B002038B5294D2DED048BF1
:10C4180095EDA48AB0EE480A0446FBF7BBFCF0EEA3
:10C42800408AB0EE480AFBF752FC95EDA59AB0EEAB
:10C43800408AB0EE490AFBF7ADFCF0EE409AB0EE48
:10C44800490AFBF744FC94ED017AD4ED027A94EDA5
:10C45800006A68EE676A27EE088AE7EE286A68EEDF
:10C46800000A67EE807AE6EE290AB0EE660AE7EE81
:10C47800A80A06F083FBDFED0F7A20EE270ADFED2E
:10C488000E7A80EE270ADFED0D7A30EE270AF2EEFB
:10C49800047A80EE270A06F06FFABDEC048B83B2AB
:10C4A8001A0444BF00F5B47083B218B238BD00BF97
:10C4B800CC1F00200000E144DB0F494000000000D1
:10C4C80001380A4B042804D8DFE800F00507090BF7
:10C4D8000D00074A08E0074A06E0074A04E0074A51
:10C4E80002E0074A00E0074A1A607047000100208E
:10C4F800A9A3000871B70008D5A600085BA000082A
:10C50800B99C000831BA0008704708B50B4B0020E9
:10C5180093F82C10FAF760FD094B1B68187A082865
:10C5280001BF084B4FF480521A80102208BF5A806E
:10C53800A0F109035842584108BD00BFCC000020B3
:10C548009823002064220020704770477047FEE758
:10C55800FEE7FEE7704730B50024E3B293420DD200
:10C56800030F092B94BF3033373301F8143001EB34
:10C578004403002500015D700134EEE730BD30B59D
:10C58800002202F1805303F5B8539B0042F40044A3
:10C598001D6840F60F7144F08004294001322143A0
:10C5A800042A1960EDD1024B40F08000186030BDBC
:10C5B8004C5C00402DE9F347884D894C2B68894E27
:10C5C8009BB2A380A28831880A40970507D54FF609
:10C5D800FF53854A2B6013780133DBB21370A388AD
:10C5E8000B40180440F100830023ADF802302B689B
:10C5F8007B4F9AB21804A28040F1F682BB8803F000
:10C608000F03BB71002B40F0C182784A13689BB2BC
:10C618003B803B8803F030037B803B8803F4405326
:10C628003B8011684BF6BF730B4083F4005383F0D3
:10C63800200343F4004343F080031360BB88D9060A
:10C6480021D4116848F60F730B40694913600B68D1
:10C658001A7A022A884601D0042A02D1FAF748FC3D
:10C668005AE2062A40F06B825A78052A08D11A78CD
:10C67800520605D1D878FFF782FFBB681B6A984736
:10C68800E3689B685AE213689BB2ADF80230BDF8C4
:10C6980002301F0540F1D0811168554F40F68F7365
:10C6A8000B40544913600A68534B92B213445B0021
:10C6B80088461A683B68187A092817D092B252003F
:10C6C80002F1804202F5C042117819705178597010
:10C6D8009188C8B2090A41EA002159801189C8B273
:10C6E800090A41EA002199809289DA8001221A72A6
:10C6F800DA8893F80190002A40F0DC801A7812F06A
:10C708007F024AD1B9F1090F0FD1DA78012A00F274
:10C71800B8809978002940F0B4809988002940F0C1
:10C72800B0809A72A3685B68A9E0B9F1050F10D1CF
:10C7380093F90320002A01DA0823B9E09A78002A3D
:10C74800FAD19A88002AF7D19B7A002B00F0A280B0
:10C75800F2E7B9F1030F0ED1DA78012A40F091809F
:10C768009A88002A40F08D805A7A42F020025A7244
:10C77800A368DB6983E0B9F1010F40F08280DA78C1
:10C78800012A7ED19A88002A7BD15B7A980678D5CF
:10C79800FAF744FC00287DD073E0012A2ED1B9F1C4
:10C7A8000B0F6ED1E26858799269D97890473B6847
:10C7B8009A7A002A65D0002863D11A79002A60D1B4
:10C7C8009B78002B5DD1064B9B68DB689847084B2C
:10C7D8001B685A79DA72DA781A735BE0445C0040B5
:10C7E80064220020AC26002013270020005C0040B3
:10C7F80098230020505C004004300020022A40D1D9
:10C80800B9F1010FC4D0B9F1030F3AD1587920F02A
:10C81800800E4FEA8E0202F1804101F5B84110F016
:10C82800800F096814BF01F0300101F44051BEF1D6
:10C83800030F26D8B3F802E0BEF1000F21D101B3EF
:10C848009B7AF3B102F1804202F5B84201061368FF
:10C858004BBF23F4E04323F4804323F0400323F049
:10C8680070034BBF9BB29BB283F0100383F48053D9
:10C8780043F4004343F080031360A3689B6998471F
:10C8880008E0E36848465B69984703280FD000280A
:10C898007FF452AFD8F80020A14B92B213445B004A
:10C8A8001A6800221A6030236380062300E00923F7
:10C8B8003A6847E1B9F1060F12D11A78520678D1D1
:10C8C8009B78012B02D1E368DB6967E0022B02D178
:10C8D800E3681B6A62E0032B6BD1E3685B6A5DE087
:10C8E800B9F1000F38D15988002962D15A6822F469
:10C8F8007F42B2F5003F5CD11A7812F07F0204D172
:10C908009B88002B00F0D58153E0012A08D1E2680A
:10C9180058799269904700284BD13B689B7A17E079
:10C92800022A46D15A7902F00F010BB29B0003F19B
:10C93800804303F5B84312F0800F1B6814BF03F05F
:10C94800300303F44053032933D812F0700F30D169
:10C95800002B40F0AE812CE0B9F1080F04D11B7810
:10C968005B0600F0A88124E0B9F10A0F21D11A78FA
:10C9780002F07F02012A1CD19A7AD2B15988C1B932
:10C988005A6822F47F42B2F5803F12D1E2685879A2
:10C9980092699047002800F090810AE04BB13A680C
:10C9A8004FF00008A2F8128093614046984740462D
:10C9B8000BE0E3683A681B6950789847032804D16C
:10C9C800584B1B6809221A72BDE03A68138A4FF661
:10C9D800FF718B4201D10923B4E0022800D00BB9C2
:10C9E8000823AFE092F9001000291FDAD1880191DD
:10C9F8000198834202D9019B138210E08B420ED228
:10CA0800E16891F82C00834201D2002105E093FBF4
:10CA1800F0F100FB113313B90121434B1970E3689E
:10CA280093F82C309382FAF763FA8CE0032313729D
:10CA38004FF44053238086E0BDF802301BB2002B30
:10CA4800BFF6D5AD116840F68F730B401360354AB9
:10CA580017683B7A022B904671D0042B6FD0032BBA
:10CA680001D0052B66D1BB693A8A8BB9398A00296E
:10CA78003BD04FF4405323802C4B1A68284B92B27A
:10CA880013445B001A6800221A60302363802CE08C
:10CA9800002AEBD0B7F81490914528BF91461FFAA9
:10CAA80089FA504698473B8ACAEB03033B827B8A44
:10CAB80053447B821D4B1A681D4B92B213445B0092
:10CAC80009F101021B689BB203F1005303F54053BF
:10CAD80052105B004FF0000E9645C7D053F82E1049
:10CAE80020F81E100EF1010EF6E7BB8A8B42D8F82B
:10CAF800003001D8032201E011B105221A720BE0BF
:10CB080006221A72094B1A68054B92B213445B004D
:10CB18001A68196030236380D8F800301B7A0FE058
:10CB2800023000209823002012270020505C00408B
:10CB380004300020072B02D1E368DB6898470823FC
:10CB4800D8F800201372FFF7E0FC5E4B1A684BF62A
:10CB5800BF7313402288D704228848BF83F48053C8
:10CB68009004628848BF83F40053D106628848BFA6
:10CB780083F01003920648BF83F0200343F4004378
:10CB880043F080034F4A9BB213602DE09A0002F1F4
:10CB9800804202F5B842116889B2ADF80210BDF8BA
:10CBA800021009B2002909DA106840F68F710140B5
:10CBB8001160013B444A52F823309847BDF80230CF
:10CBC8001F067FF514ADA1798B0003F1804303F5AF
:10CBD800B84348F60F72186802401A603A4B03EBE4
:10CBE80081039B69984702E5A28833881340590559
:10CBF80005D54FF6FF332B60344B5B689847A28806
:10CC080031880A40920444BF4DF6FF732B60A38815
:10CC18002F4A0B40DB0452D54EF6FF732B600023DE
:10CC28001374137C052B41D8DFE803F0030D1418A7
:10CC3800222D6369264D1BB901F08CFF062300E005
:10CC480005232B743BE001F085FF042323740123A3
:10CC5800636134E002236374032328E0637C013BAF
:10CC6800DBB26374637C53BB194B04221A7426E04D
:10CC7800184A13689BB243F010031360052323740A
:10CC88000A2363741BE0637C114A013BDBB26374C3
:10CC9800637C03F0FF0093B90E490C684FF6EF73FD
:10CCA80023400B6006231374506108E006232374A5
:10CCB80005E0094B73E6094B71E6094B6FE602B0D4
:10CCC800BDE8F087005C00402C4D0108CC00002036
:10CCD80064220020405C0040516A0008096B00088B
:10CCE800E56A0008022803D0431E5842584170479D
:10CCF800064B1B681B7823B1054B1868C0F3C0406E
:10CD08007047044B1878C0F380007047000A002071
:10CD1800DC1000201027002010B50A4C5E280146C0
:10CD2800206805D15D21FFF78DF920683E2105E0D7
:10CD38005D2903D1FFF786F920683D21BDE8104041
:10CD4800FFF780B97C22002030B50028104C114A2A
:10CD5800B8BF40423C2590FBF2F304FB0300684354
:10CD68000D4D90FBF2F22D682D7B25B903EB830363
:10CD780003EB830301E0C3EB031302EB83030B8094
:10CD880004FB02024FF47A7392FBF3F24A8030BD3F
:10CD9800806967FF80969800D018002010B5044677
:10CDA800C0B2FFF7B9FFC4F30720BDE81040B3E7EE
:10CDB800024B5E211868FFF745B900BF7C220020AE
:10CDC80038B5064C05465E212068FFF73BF9206818
:10CDD8002946BDE83840FFF735B900BF7C2200205E
:10CDE800674B73B51878674DFFF77CFF2B78834244
:10CDF800044620D0C8B1644B1B68E3B193F9000026
:10CE080002230093614B1B685B78003318BF012332
:10CE1800019304214FF416530022F9F76DFA5C4B85
:10CE2800186040B101232B7005E0594E3068F9F7BE
:10CE380048FA34602C70574B574D1878FFF752FF5B
:10CE48002B788342044618D088B1544B1B68A3B191
:10CE58000022012493F9000000944FF496430192B4
:10CE68000821F9F749FA4E4B186028B905E04C4EED
:10CE78003068F9F726FA34602C704A4B4A4D187816
:10CE8800FFF730FF2B78834204462E4642D0002815
:10CE980037D0464B1A68002A3CD0D37992F9000063
:10CEA800434C002B08BF022302220092002254F8B0
:10CEB800233001921021F9F71FFA3E4B05461860FE
:10CEC80040B33D4C94F84A30022B0BD094F896208E
:10CED800022A01D14C3405E023B1002A04F14C04A4
:10CEE80018BF0024354B1C6044B1204600214C2259
:10CEF80005F033FB0223256084F84A3001233370A0
:10CF080008E02C4E306800F0EBFC3068F9F7D9F9EE
:10CF180034602C702A4B2B4D1878FFF7E3FE2B78E2
:10CF28008342044629D000B3274B1B682BB3274AFA
:10CF380093F9000012685278002A0CBF08220922CF
:10CF48000323009301924FF4614320210022F9F753
:10CF5800D3F91F4B186080B11E4A012313702B7040
:10CF68001D4B1A681D4B1A6007E0194E3068F9F717
:10CF7800A8F9184B34601C702C7002B070BD00BF4B
:10CF8800080A002098110020040A0020D018002068
:10CF98007C220020090A0020F018002074190020C3
:10CFA80064190020140A00207A190020100A0020B1
:10CFB8008C5C01087C190020FC23002080190020CB
:10CFC800200A0020901900201C0A0020180A0020BE
:10CFD8009419002098190020942600209C190020FC
:10CFE8002DE9F04FC34BDA682DED028B1A61C24A66
:10CFF8001168D960C1490B6843F020030B60C04B2E
:10D008001978012990460CBF002201221A70BD4BE5
:10D018001A78910789B040F13F83BB490978042900
:10D0280040F23A83B949097801F0040101F0FF00A0
:10D0380011B922F001021A701B78DB0702D408B17B
:10D04800FEF7DCF9B2490A79531C052293FBF2F288
:10D0580002EB82029A1AAF4B0A711B780393920073
:10D068000023AD4CDFF8D0C2DFF8DC925CF8231067
:10D0780091FBF9F504F1080004F1100640F823507B
:10D08800A64844F8231000FB051142F2107091FBEA
:10D09800F0F080B226F813004FF0140E04F11406D5
:10D0A80004F13C0A0EFB036E5AF823605EF8027026
:10D0B8004EF80210F61B314444344AF82310052672
:10D0C80091FBF6F109FB051144F82310039C012C90
:10D0D8004FEA830BE24605D10238B0F5797F98BF55
:10D0E8004BF80C100BB90123BBE7894CD8F800307A
:10D0F800626D9FED8B7A8B4E8B4D9B1A07EE903AA3
:10D10800F8EE677AD8F800306365C7EE877A7D4B0A
:10D118001B78B7EE008AF4EEC87AF1EE10FA58BF21
:10D12800F0EE487A13F00103C4ED167A12D005AA7E
:10D1380000927E4B06AA01920CCB9AE80300FEF7F8
:10D148005BF86421059A069BB2FBF1F293FBF1F3BD
:10D15800328000E033802B8094F85C306C48002BE0
:10D168003BD0D0ED167A026EDAF80030C8EE276AA6
:10D178009B1A426E022507EE103AB8EEC77ADAF823
:10D18800043027EE267A9B1AFDEEC77AB0F96A209A
:10D1980017EE901A07EE903A654BB8EEE77AD3EDA2
:10D1A800007A67EE277A67EEA67AFDEEE77A17EE41
:10D1B800903A02FA83F3B0F9682093FBF5F302FA88
:10D1C80081F29BB292FBF5F292B2A0F86E30A0F811
:10D1D8006C20A0F86A30A0F86820012384F85C303D
:10D1E800544BDAF804101B88DAF80000484D524E08
:10D1F800616603F030032066002B00F04D8205F1D4
:10D208007803009305F17C0301932A6F6B6FFDF798
:10D21800F3FF72686B6F9B1A07EE903A444B3268C3
:10D2280093ED007A2B6FF8EEE77A9B1AC5F88030F9
:10D23800384B67EE877A1B78FDEEE77A012BC5ED50
:10D24800217A03D0022B00F0E08025E2D5ED297A7F
:10D258003A4BD5ED225A95ED265A95ED166A95ED7D
:10D26800274AD5ED284A36491D68B1EE677ABDEEE2
:10D27800C77AFDEEE77A17EE10EA17EE90CA00209B
:10D28800304A91ED007A52F8207007EE907AF8EE65
:10D29800E77AA2F1140367EEA57A33F81060FDEE81
:10D2A800E77A283217EE903A9B1B9BB222F810308F
:10D2B8001BB207EE903AF8EEE77A3B4467EE857AC0
:10D2C8004400FDEEE77ACDED037A07EE903AF8EEEA
:10D2D800E77ABDF80C8067EE847AA7EE867AFDEED1
:10D2E800C77A17EE902A724532DB6245A8BF6246BC
:10D2F8002FE000BF8401002094260020DC180020C5
:10D308003A110020E0180020E6180020102700201D
:10D318007C2200200C0B002084220020806967FFFB
:10D3280000007A445A1900205C1900203C110020A2
:10D338006C000020A4190020E8180020100B002021
:10D34800400B0020FC22002080969800DB0FC9408B
:10D35800724607EE902AF8EEE77A5FED046AC1EDAF
:10D36800007AFDEEE77A313617EE903A43449AB2E6
:10D37800AB78D1ED027A07EE103AB8EE477A4B68EF
:10D388004F6027EE267AFB1A88EE077AB6B2622E2D
:10D3980006EE903AF8EEE66A37EE067AC6EE866A48
:10D3A80086EE077A76EEE76AE7EE267AC1ED047A2A
:10D3B800C1ED027A0FD964EEA77ABA4EFDEEE77A8C
:10D3C80017EE903AB3F5FA6FA8BF4FF4FA63B34279
:10D3D800B8BF334600E0002313441BB240F6B8320E
:10D3E8009342A8BF1346B04A9342B8BF1346AF4A08
:10D3F800A352AF4A142303FB002351F8142B1A60DD
:10D40800002840F0498101203AE7AA4BD5F87880F6
:10D418001F68D4F87C903E89DFEDA78A4FEA58034D
:10D428009E4228BF1E46B5F8AC301AB29642C3BF1A
:10D43800D5ED167A9FEDA17A67EE877AB6B2C1BFAD
:10D44800FDEEE77A17EE906AF618B6B2C8BFA5F8EF
:10D45800AC60D4F8B050C5EB09052846FDF710FFBD
:10D468000028D8BF404241F293129042CCBF00201E
:10D47800012088B307EE905AB8EEE70A20EE280A92
:10D48800FAF725FC07EE908AF8EE677A40F6B8338B
:10D4980020EE270AFDEEC07ACDED037ABDF80C2008
:10D4A800A4F8B42012B29A42A8BF1A467E4B9A42F8
:10D4B800ACBF09EB02034B4448F6A042934203DD9C
:10D4C800A3F50C43A03B04E0002BBCBF03F50C43C1
:10D4D800A033C4F8B83001E0C4F8B890D4F8B85014
:10D4E800C5F50C53283307EE903AF8EEE77A67EE65
:10D4F800A88AB0EE680AFAF74DFC8DED070AB0EE7F
:10D50800680AFAF7E4FBD4ED327AD4ED2F4AD4ED69
:10D51800165A94ED304A94ED315A65498DED060A54
:10D52800B1EE677ABDEEC77AFDEEE77A0DF1180E17
:10D5380017EE10AA17EE90BA0020614AFEEC016AB5
:10D5480032F91030DFF88C9107EE903A07EE106A46
:10D55800F8EEE77AB8EEC77A3C32D6EE877A4FEA29
:10D56800400CFDEEE77ACDED037ABDF90C30B3F54A
:10D578007A7FA8BF4FF47A734B45B8BF4B461FFA62
:10D5880083F922F810900FFA89F207EE902AF8EE44
:10D59800E77A27EEA47ABDEEC77A8DED037A27EEF7
:10D5A800847AD1ED007ABDF80C90E7EE257AFDEE8D
:10D5B800E77A17EE902A524503DB5A45A8BF5A4628
:10D5C80000E0524607EE902AF8EEE77A9FED3D6AB2
:10D5D800C1ED007ABA7891ED027A06EE902AF8EE5B
:10D5E800666A4A684B6066EE866A9A1AC8EE266AC8
:10D5F800143106EE102AB8EEC66A76EEA56A86EEF3
:10D60800256AC5EEA66A36EE476AA6EE867A01ED69
:10D61800017A01ED037A25EE077ABDEEC77A17EE97
:10D62800103ABDEEE77A4B4417EE102A13441BB2AA
:10D6380040F6B8329342A8BF13461B4A9342B8BF7C
:10D6480013461A4A2CF802301F4A142303FB0023FE
:10D65800C3ED007A08B901206FE73B7923B1642351
:10D6680095FBF3F5194B1D803B8898450DD9D4F8E7
:10D67800B030E06FC01AFDF703FE80EAE072A2EB5B
:10D68800E07242F210739A4206DD114B01221A70C1
:10D698000E4BB4F8CC201A8009B0BDEC028BBDE863
:10D6A800F08F00BF30F8FFFF48F4FFFF940B002015
:10D6B800680B0020100B0020D30237390000C84245
:10D6C800E8220020DB0FC940400B0020C4100020D6
:10D6D8000C0B002018FCFFFF07B5064B0093064B08
:10D6E80001930649064A074B0748FAF7C2FA03B0FE
:10D6F8005DF804FBAE5D0108835D01084D6B010810
:10D70800576B0108A25D01082D6B010808B5037865
:10D7180033B90C4B0C481978BDE80840FAF7A9BA98
:10D7280004F0B6FF02280CD8064B1870074B0C22E1
:10D7380002FB0030064B02301860FAF7BBFC0548C4
:10D74800E5E708BD4C2300205E6B01089C1800200B
:10D75800341100207061010808B503783BB90B4B00
:10D768000B4893F8E816BDE80840FAF782BA04F0C7
:10D778008FFF022808D8054B83F8E806FAF700FC63
:10D78800FAF7BCFC0348E8E708BD00BFB411002065
:10D79800626B01087061010838B5037803BB214B3F
:10D7A8001B6801330F2B07D81F490C2202FB0312F9
:10D7B8001C4695682DBB00E01C4601340F2C01DD8A
:10D7C800002400E005D818490C2202FB04129568D1
:10D7D800BDB99C42F1D11548BDE83840FAF749BABD
:10D7E80004F056FF0F28044605D80F4A0C2303FB04
:10D7F80000239D682DB921460D48BDE83840FAF749
:10D8080038BA084B1C60F9F787F821462A460948B8
:10D81800FAF72FFA0C235C43034B185DBDE8384038
:10D82800F9F790B870000020684D01086F6B010887
:10D83800856B01089D6B010873B5037813B9F8F778
:10D84800E3FB3FE001AA204904F083FF00240246DD
:10D85800264625469AB134B1012C08D1104604F069
:10D8680017FF064603E0104604F012FF054601AA1A
:10D878000020154904F06DFF01340246EAE70B2D3C
:10D8880003D9124812490C230CE0022C11D1A6F539
:10D898007A73B3F57A7F08D90C480E494FF47A7237
:10D8A8004FF4FA63FAF7E5F90CE00B4B03EB450389
:10D8B8005E80094B094803EB45032946B3F902206A
:10D8C800FAF7D7F902B070BDF6660108C36201081D
:10D8D800E2620108AF6801084C230020B46B01081C
:10D8E80038B50D4C23688342054606D1F8F7E9FCA4
:10D8F800204600214C2204F030FEE36CAB4209D1F3
:10D908002846F8F7DEFC054800214C22BDE83840DF
:10D9180004F023BE38BD00BFFC23002048240020AB
:10D92800034B1A68D379591C1344D171187A70477C
:10D938008419002010B5FFF7F3FF84B2FFF7F0FF5A
:10D9480004EB002080B210BD10B5FFF7F3FF0446CA
:10D95800FFF7F0FF04EB004010BD064B10B504467E
:10D9680021461868FEF76EFB034B1B6898796040E8
:10D97800987110BD881900208419002038B5044614
:10D9880024200D46FFF7E9FF4D20FFF7E6FF002CA6
:10D99800084C14BF21203E20FFF7DFFF2368002238
:10D9A80028469A71FFF7D9FF236893F84900BDE824
:10D9B8003840D2E78419002001460020DEE710B580
:10D9C8000446C0B2FFF7C9FF200ABDE81040C4E70B
:10D9D80010B5044680B2FFF7F2FF200CBDE81040F6
:10D9E800EDE737B582888368044610060D4641BFC7
:10D9F8002B4991F8E8164FF4CC7000FB0133D105A0
:10DA080044BF2849097802F03F0244BF01EB4101B5
:10DA180003EB8103042A12D006D8012A0DD0022A6A
:10DA280032D193F9001030E0102A0AD0202A0AD007
:10DA3800082A29D1B3F9001027E0197825E01988B8
:10DA480023E0196821E093ED000A6846F9F7A6FF7C
:10DA580001461548FAF70DF905B3D4ED037A68467F
:10DA6800B8EEE70AF9F79AFF01461048FAF701F904
:10DA780094ED040A6846B8EEC00AF9F78FFF01462C
:10DA88000A48FAF7F6F809E000210948FAF7F1F828
:10DA980025B10848E1682269FAF7EBF803B030BD10
:10DAA800B41100204C230020596401085264010875
:10DAB800C76B0108C36B0108024B0146D869FEF722
:10DAC800C1BA00BF4C23002010B5441E14F8011F32
:10DAD80021B1034BD869FEF7B5FAF7E710BD00BFCF
:10DAE8004C230020F7B52B492B4B08782B4D1C688D
:10DAF8002B4B05EB80001A882A4BD0F8C0101B78F6
:10DB0800294800914FF47A71B4FBF1F1FAF7B1F8B2
:10DB180026484821FAF7ADF8254B1F680026F3B2CE
:10DB280005EB8302D2F8D010E9B101249C403C42B5
:10DB380017D0220715D01F4AD25C0B2000FB032305
:10DB4800164A1D4802EB8303D3F8F020FAF791F840
:10DB5800022C06D1194B93F8281011B11848FAF77E
:10DB680088F80136DBE71748FFF7AEFF164B174872
:10DB78001A68174B9A420CBF164B174B1A88174B4B
:10DB8800198892B240F2147303B0BDE8F040FAF776
:10DB980070B800BF2C19002094260020684D010899
:10DBA800CC180020FC000020CA6B01080D6C01088D
:10DBB800DC180020040100201D6C01084C23002003
:10DBC800256C01086D6C0108D4100020296C01082F
:10DBD80000540040D8100020DA100020D010002097
:10DBE8002DE9F0410024804625460F4EA7594146AD
:10DBF800384604F035FD58B139460C48FAF739F87B
:10DC080030190021FFF7EDFE0948FFF75DFF0135E8
:10DC1800143440F6BC439C42E7D11DB90548BDE821
:10DC2800F04151E7BDE8F081084F0108DF640108C1
:10DC38006D6C0108816401082DE9F04F2DED028B10
:10DC480083B0054604F0CDFC064620B1012818D162
:10DC58002B782A2B15D15C48FFF736FF00245B4D43
:10DC68005B486159FAF705F828193146FFF7B9FEFC
:10DC78005848FFF729FF143440F6BC439C42EED1C4
:10DC88009CE028463D2104F09EFC002800F08F808F
:10DC98000346994613F8012D202AFAD0441C204641
:10DCA80004F0F6FC80462046F9F7EEFDC5EB0909BD
:10DCB800B0EE408A0026DFF834A1142202FB06F4F5
:10DCC8000AF5D07B54F80B70384604F08AFC0346FA
:10DCD8001A4628463946019304F08CFC019B00281B
:10DCE8005BD15FFA89F29A4257D10AEB0402D2ED6E
:10DCF8006B7AF8EEE77A0BEB0405B4EEE78AF1EEFF
:10DD080010FA48DBD2ED6C7AF8EEE77AB4EEE78ADF
:10DD1800F1EE10FA3FD8B2F8A431D2F8A82113F0E6
:10DD2800200F08BF08EE108A1C0641BF2A4991F847
:10DD3800E8164FF4CC7404FB0122D90544BF2749E7
:10DD4800097803F03F0344BF01EB410102EB810274
:10DD5800042B18EE100A0BD004D8013B012B0ED867
:10DD680010700CE0102B05D0202B06D0082B06D104
:10DD7800108004E082ED008A01E082ED008A3946D5
:10DD88001748F9F776FF2846002103B0BDEC028B4F
:10DD9800BDE8F04F25E6134803E00136A32E8AD1EB
:10DDA800114803B0BDEC028BBDE8F04F8CE6284665
:10DDB80003B0BDEC028BBDE8F04F11E703B0BDEC3A
:10DDC800028BBDE8F08F00BF5B6C0108084F0108AB
:10DDD800DF6401086D6C0108B41100204C23002099
:10DDE800706C01087B6C010881640108684D0108AA
:10DDF80070B50546284604F0F4FB064658B9194B99
:10DE080019485A79194B03EB8203BDE87040D3F8DF
:10DE1800581EF9F72EBF28461549324604F0EAFB8A
:10DE280060B91448144CFFF74FFE54F8041F19B199
:10DE38001248F9F71EFFF8E7114805E00024114BD6
:10DE480053F8241019B91048BDE870403CE628463C
:10DE5800324604F0CFFB01340028F0D1014B0B4DC2
:10DE68005C71C7E7B41100209B6C0108684D01087C
:10DE780070640108A76C0108C05B01086C640108A4
:10DE88006D6C0108C45B01088164010870610108B8
:10DE980008B50748FFF718FE064BD869F8F706FAE1
:10DEA800FEF730FAFAF742F8034B044ADA6008BD85
:10DEB800BA6C01084C23002000ED00E00400FA05CC
:10DEC80008B50548FFF700FE00F038F8FAF758F8EB
:10DED800BDE80840DCE700BFC66C010808B5044887
:10DEE800FFF7F2FDFAF74CF8BDE80840D0E700BFAD
:10DEF800DC6C01080F4B1A78692A17D1598840F24F
:10DF08001472914212D11A79BE2A0FD193F81127AF
:10DF1800EF2A4FF000000BD113F8012B5040064AAE
:10DF28009342F9D1B0FA80F0400970470020704759
:10DF3800704700BF00F8030814FF03082DE9F04FED
:10DF48002DED028BEA4D002140F2147285B028466F
:10DF580004F003FBE74B05F508721A60E64A002354
:10DF68001370E64A05F2EA61116069222A700322F9
:10DF78006A714FF48072AA604FF41672A5F8662190
:10DF8800FA22A5F86821BC22A5F864214FF4FA7298
:10DF98002021A5F86E21012285F8622185F86A11F1
:10DFA80085F87E216E2185F88621052285F87C1169
:10DFB80085F81F220A2140F2DC5285F87D11A5F868
:10DFC80098212B2140F24C4285F87F11A5F89A211F
:10DFD800212140F26C7285F88011A5F89C2123213B
:10DFE80040F2753285F88111A5F89E214FF4C87169
:10DFF80040F64302A5F8A021A5F882112A462C462E
:10E00800032BCCBF0121002103F1010382F8A211E7
:10E0180014BF1E217521122B82F8A31102F10202EE
:10E02800EED140F27E424FF4FA63A4F8442140F264
:10E038003A72A4F8C831A4F8CC31A4F8D031A4F8C5
:10E04800D431A4F84621052340F27E5284F8E23107
:10E05800A4F84C21C82340F2EA5201274FF47A78F9
:10E068004FF0320A40F2DC51A4F8E631A4F84E2110
:10E078004FF4C87340F2B4521E204FF0190BA4F8A5
:10E08800EA31A4F84A11A4F85021A4F852A1A4F83E
:10E09800C681A4F8CA81A4F8CE81A4F8D28184F8F4
:10E0A800E47184F8E57184F8E871A4F8488184F88B
:10E0B8009501039084F8E3B10291A4F85431A4F8CF
:10E0C80056A184F8E17184F8EE7184F8F17100F0DA
:10E0D80047FC884A0398136827740026E773A673D9
:10E0E800A681D87218735520D8700F205871222035
:10E0F80098710E2018743520987621204FF0170E4D
:10E10800587453204FF0280983F815E083F816E077
:10E1180083F807B04FF02D0ED87601925A2064226A
:10E128004FF00A0B4FF0780C83F80DE083F804A049
:10E1380018721A771E7083F8019083F80290DE75C2
:10E148009E731E76DE735E7683F812B083F80990AC
:10E1580083F80AC083F814E04FF4FA7EA3F84EE07F
:10E168004FF03C0E83F851E04FF0110E83F850E069
:10E17800DFF8A4E1C3F838E0C3F83CE0DFF89CE13D
:10E18800C3F828E0DFF898E1C3F834E0DFF894C179
:10E19800DFF894E19FED5A8AC3F82CC0C3F830C069
:10E1A800C3F848E0F7EE087ADFF880C102999F7754
:10E1B8004FF04B0E83F85260C3ED087AC3ED097A2D
:10E1C80083ED108AC3F844C083F84CE084F8EA066B
:10E1D800A4F8F4164120042184F8EB0684F8ECA690
:10E1E80084F8ED6684F8F16684F8F26684F8EE66E1
:10E1F80084F8EF6684F8F06683F85C101521A3F8BC
:10E208005860A3F85A60A3F85660C3F860C083F852
:10E2180068103C49D9663C4919673C4983F86490C1
:10E2280083F86590596783F87870394800F0DEFB09
:10E23800019AD2F800A04FF44873AAF81631C823FF
:10E248008AF811618AF812618AF813918AF81471B0
:10E258008AF8186184F8D931642384F8D8B1A4F80D
:10E26800DA8184F8DC61A4F8DE3152460E2303FB20
:10E2780006A36FF0170183F81911032183F81A1107
:10E288006FF02F0183F81B11072183F81C116FF021
:10E29800230183F81D11052183F81E1101365A2127
:10E2A80082F8201182F821116423FF21082E82F8B8
:10E2B8001F3182F8221102F10E02D7D100228AF80A
:10E2C8008921C822AAF88A21AAF8903114224FF489
:10E2D80096738AF88C21AAF892311E2228238AF88C
:10E2E8008D21AAF8943101220A4B8AF88E211FE069
:10E2F800B4110020141100204C23002034110020F8
:10E30800000000009A99193FF6287C3F3D0A773FA4
:10E31800C2770108741200208FC2F53C00006040EB
:10E328006666663FCDCCCC3E000040400000A04071
:10E3380085ED058A10359D42FAD11A4C0023012536
:10E34800514604F56E704FF4CC7284F8103784F897
:10E358000E5784F80F5704F0F5F804F5AA605146F3
:10E368004FF4CC7204F0EEF80F4B1B681A68C4F82F
:10E37800F6265A68C4F8FA269A68C4F8FE261A6877
:10E38800C4F802275A68C4F806279A68C4F80A2706
:10E39800022384F80C5484F8A43505B0BDEC028B34
:10E3A800BDE8F08FB4110020341100201549D1F8D0
:10E3B800883043F47003C1F88830134B1A6842F070
:10E3C80001021A605868114A02405A601A6822F01D
:10E3D800847222F480321A601A6822F480221A6049
:10E3E8005A6822F4FE025A60DA6A22F00F02DA62F0
:10E3F800186B074A02401A6300229A604FF00063C4
:10E408008B60704700ED00E0001002400CC07FF800
:10E41800CCFC00FF38B5094B93F8105765B9084C88
:10E428002068F7F74EFF074B25601B78022B03D1B6
:10E43800BDE8384000F053BA38BD00BFB411002021
:10E44800CC240020CB240020044B93F810371BB9B0
:10E45800034B1868FDF7EABD00207047B41100208F
:10E46800CC24002038B505460446204614F8011B84
:10E4780021B1034B1868FDF7E5FDF6E7401B38BDF1
:10E48800CC2400200FB407B504AB064953F8042B7D
:10E4980001930020F9F700FB03B05DF804EB04B02A
:10E4A800704700BF1BE60008024B01461868FDF7DD
:10E4B800C9BD00BFCC240020F8B5011F06460023C3
:10E4C800083051F8042F02F120043F2C3AD802F109
:10E4D80008040F2C06D80232032A04D9002B08BFDF
:10E4E800012300E002238142EBD1012B30680ED0DA
:10E4F800022B1AD0736803F003039B0000F003009B
:10E5080043EA0010B36803F00303184317E000F070
:10E518000F0040F04000FFF7C7FFB068736800F0D5
:10E528000F0040EA0310C0B209E000F03F0040F0DD
:10E538008000FFF7B9FF3079FFF7B6FF307ABDE802
:10E54800F840B1E706F10C0734463A46002552F880
:10E55800043D03F18001FF294FEA850510D903F531
:10E568000041B1F5803F02D245F0010508E003F50E
:10E578000003B3F1807F34BF45F0020545F0030581
:10E58800B242E4D165F03F00C0B2FFF78DFF05F05D
:10E598000303022B207807D0032B0CD0012B13D1B7
:10E5A800FFF782FF60780FE0FFF77EFF6078FFF7E4
:10E5B8007BFFA07808E0FFF777FF6078FFF774FF2C
:10E5C800A078FFF771FFE0780434FFF76DFFBC42D5
:10E5D8004FEAA505DBD1F8BD10B50446C0B2FFF778
:10E5E80063FFC4F30720BDE810405DE710B504469B
:10E5F8007F2C06D964F07F00C0B2FFF755FFE4090D
:10E60800F6E7E0B2BDE810404EE7430083EAE07069
:10E61800ECE7084648E700BF82B01B4B1B4A8DF861
:10E6280007101968106860B31268052A29D1184ABA
:10E63800106810BB9DF808109DF8073043EA0123C5
:10E6480014490B80144B1968144B89B20B445B00B6
:10E6580019680121196013680B441360104A136884
:10E6680023F4E04323F040039BB283F0300343F4E8
:10E67800004343F08003136003E01A68521A312AFA
:10E68800D5D902B0704700BF94260020F826002094
:10E698009023002080610040505C00400A30002038
:10E6A800045C0040014B5868C0B2704790230020BA
:10E6B800012070477047704720B9034B9B680822B8
:10E6C8001A82704701487047902300207400002088
:10E6D80020B9034B9B6808221A827047014870478B
:10E6E800902300207400002021B901288CBF02204B
:10E6F800002070470220704710B5094B9A68D378FC
:10E70800042B0BD8074C518ADB00234418B99B898A
:10E718005B1A138210BD9B68581810BD002010BDED
:10E728009023002074000020054B9968054B4A8A05
:10E7380018B99B8D9B1A0B827047986A10447047D2
:10E748009023002074000020054B9968054B4A8AE5
:10E7580018B99B8E9B1A0B827047186B1044704730
:10E768009023002074000020074B9B681B7803F05F
:10E778007F03212B06D100F0DF00022814BF0220FE
:10E78800002070470220704790230020212810B5F0
:10E7980008D1114B9B681B7803F07F03212B10D005
:10E7A800022010BD2028FBD10B4B0C4A9B6810702F
:10E7B8001B7803F07F03212B094B18BF00230BB9EB
:10E7C800EEE7084B044A926800249361548220467D
:10E7D8009847204610BD00BF902300201427002032
:10E7E800C1E60008D9E600087047034B1A78202ACA
:10E7F80004BF00221A70704714270020014B04221E
:10E808001A607047F8260020034B9B7D13B1034B19
:10E8180005221A60704700BF90230020F8260020C8
:10E82800F7B51E4B5A681D460AB95C6800E001241A
:10E8380093F828000021CAB2A24201F1010108D2CE
:10E8480002AE2F1816443A4492F8292006F8042CF0
:10E85800F1E75A68121B5A6093F828205D68224431
:10E8680083F82820A5B903204021F8F7B5FB0C4A06
:10E87800136823F4804323F070039BB283F440535E
:10E8880043F4004343F080031360044B83F828509B
:10E89800002CC6D09DF8040003B0F0BD90230020E2
:10E8A8000C5C004010B50446B0F90000FFF7ADFE5F
:10E8B800B4F90200FFF7A9FEB4F90400BDE810405E
:10E8C800FFF7A3BE10B504460068FFF79EFE606818
:10E8D800FFF79BFEA068BDE81040FFF796BE2DE944
:10E8E800F74F0120F7F730FF002488B3012C2FD809
:10E8F800194E4FF04C0909FB04FA06EB0A0808F117
:10E90800B407BD7815B10134E4B2EEE790F90030F0
:10E9180090F804E01846114B03228DE824000121E9
:10E928002A4653F82E30F7F7E7FC834660B106F124
:10E938006C00504429464A4603F00FFE01231C444C
:10E94800C8F86CB0BB70E4B20120F7F7E1FECCE781
:10E9580003B0BDE8F08F00BF902300208C5C010855
:10E9680010B5184C002120461A2203F0F6FDA4F534
:10E97800FA70142380F8F63105230022042180F868
:10E98800FA3180F8FC3180F8023280F8043280F8DD
:10E998000A3280F80C325223012480F8FB1180F8E7
:10E9A800FD2180F8031280F8052280F80B1280F808
:10E9B8000D2280F8F43180F8FE2180F80642A0F894
:10E9C800F84110BDA813002010B5F8F731FC4FF43A
:10E9D8003024012806D11CB1F8F72AFC013CF8E7DD
:10E9E800052010BD002C08BF052010BD70B50646D7
:10E9F800441E14F8011F89B1094D284603F0E3FDB0
:10EA08000028F6D005F1080398423FBF054B401B8C
:10EA1800C018A31B38BF80F88A31EAE770BD00BF71
:10EA2800DD770108B4110020031EB8BF2D2210B5F0
:10EA3800B8BF58420C46B8BF01F8012B0A22F9F7B3
:10EA480017F800230370204610BD07B51C4B03F5CB
:10EA58008472C3F804211B4A92F892215AB1012A00
:10EA680014D1032183F80A11072183F80C2183F8B4
:10EA78000B110C2208E0022183F80A11032183F804
:10EA88000C2183F80B11072283F808210E4B0F4A3B
:10EA98009A634020F7F758FE70B10122002390F9DD
:10EAA800000040218DE80C00094A4FF4E133F7F7E4
:10EAB80023FC003018BF012003B05DF804FB00BF41
:10EAC80090230020B411002074000020E56B00089A
:10EAD800656D000801200021FEF750BFF0B51C4A03
:10EAE80092F80D31D2F8105192F8147192F8206111
:10EAF80092F82CE1022B0ED805EBC304591CA31C79
:10EB0800C9B206D02346A48814F0010F01D02042D0
:10EB180005D10B46EEE782F80D310020F0BD93F9E0
:10EB280002307CB29C4201D1002307E074B29C42BF
:10EB38000CD04FFA8EF49C42EBD1022382F80D11CF
:10EB48000C2101FB0322D2F81801F0BD0123F5E7DF
:10EB5800902300200A4B10B519684FF6FB720A4043
:10EB68001A60084A927D1C46074B0AB1052200E04C
:10EB780001221A60FFF71AFC4FF43643236010BDD8
:10EB8800405C004090230020F82600202DE9F04F3B
:10EB9800A7490B7813F0010F85B003F0040200F0C9
:10EBA8003781002A40F04181A248076817F0806742
:10EBB80040F03B81980700F12B8143F004030B7070
:10EBC8009D4B9E4C1B8823809D4B1A6812F4002F86
:10EBD800984600F0FE809B4B80201F70FFF77EFF59
:10EBE80008B1FEF77DFEA678012E40F0F280964D22
:10EBF80095F80E2722B195F80F370BB19A4203D337
:10EC0800012385F80E370FE01846114630B191FB05
:10EC1800F0FE00FB1E1E01467046F7E792FBF1F27C
:10EC280085F80E2793FBF1F385F80F3795F8103721
:10EC38001BB1854B002283F81027844B95F810A749
:10EC480004221A70BAF1000F1FD18020F7F77CFD5B
:10EC58008146D0B18021F7F751FD99F806207C4B09
:10EC6800E07053F8223099F90000DFF8D091B3F53D
:10EC7800613F0CBF0222002202218DE8060080219C
:10EC88005246F7F739FB606008B90023A0E0514607
:10EC980009F10800142203F060FC09F12803C9F8FF
:10ECA8001C3009F19403C9F8203009F58073C9F8BC
:10ECB8002430684BD8F800101B88A9F86C3195F8F7
:10ECC8009431654895F886910390002B6B79A3F1F0
:10ECD800190BC1F3C03C18BF4FF0010CDBF1000E5B
:10ECE8004EEB0B0E95F80EB7012B95F80F3705680C
:10ECF80008BF4FF0010E9B45584B1B780293C1F398
:10ED0800400A28BF4FF0000B01F4006138BF4FF0F4
:10ED1800010B721ED2B2531E132B35D8DFE803F055
:10ED28000C0C0C0C0C0C0C0C0A37377F2737811293
:10ED380012123137734675E0029B9342B4BF002329
:10ED4800012320E02B78022B0BD105EB820353ED36
:10ED5800027AF5EE407AF1EE10FA14BF012300238F
:10ED680011E0AB185B79003318BF01230BE021B128
:10ED780009F1FF304342434100E00B4603F0010331
:10ED880050E05B464EE013B1012393401F43142E1D
:10ED980002D80136F6B2BCE7039BC4F87071186854
:10EDA80019217930F7F762FD0023C4F87831A4F807
:10EDB8007C31A4F87E31C4F88831294BD4F88421F9
:10EDC8001B68C4F88C3184F87401C4F880210223CC
:10EDD800A370234B1C4A1B6892F8E2214FF47A7106
:10EDE80001FB02331F4A1360D8F800301A0609D510
:10EDF8001D4B1B789B0705D51C4B1B78042B01D991
:10EE0800062000E0052005B0BDE8F04FF7F79ABDF1
:10EE18005AB9012005B0BDE8F04FF7F7B5BD534624
:10EE280000E06346002BAFD1B3E705B0BDE8F08F33
:10EE380010270020DC100020A8110020C824002082
:10EE4800702600209D240020B41100200801002015
:10EE58008C5C0108101C0020141100208A2000205E
:10EE680094260020C00A0020E0180020E6180020A0
:10EE780010B5154A1378590725D523F004031370E4
:10EE8800124B1B681B0319D5114CA378A3F1080278
:10EE9800012A0BD8FF200021FAF714FB0D4B1B6841
:10EEA800C4F88C31FFF7D0FA0A2306E0012B05D904
:10EEB8000A2B03D0FFF7AEFA0123A3700420BDE8A4
:10EEC8001040F7F73FBD10BD102700207026002026
:10EED800C8240020942600200C4B0D49DA6843789A
:10EEE800D243C2F30222C2F10402934002781B010A
:10EEF8000A44DBB282F8003303780122580903F090
:10EF08001F0302FA03F341F82030704700ED00E0D8
:10EF180000E100E073B50546002100680122FCF716
:10EF28002FFB2A6813889BB243F001031380EB7A06
:10EF38008DF804300124002601A88DF805408DF8CD
:10EF480006608DF80740FFF7C7FFEB7A1B2B0BD144
:10EF5800192301A88DF804308DF805408DF8066056
:10EF68008DF80740FFF7B8FF02B070BDF0B5BE4C92
:10EF780023782DED028B013B012B85B000F26F81C8
:10EF88006578854240F06B81A378022B00F0678199
:10EF9800B64B5B5DE37023796D00F2EE048A1BB11A
:10EFA8006319B3F9063009E06319D4ED037AB3F9AC
:10EFB8000630F1EE677AC4ED037A5B4208EE103A48
:10EFC8002369A94EB8EEC88A1A0388EE288A35D56F
:10EFD800D6ED037AFDEEE77A28EE280A17EE903A86
:10EFE800D6ED057A8DF80A30FDEEE77A17EE903AFD
:10EFF8008DF80B3003F006FDFCEEC07A96ED060A9C
:10F0080017EE903A20EE280AADF8083003F0FAFC23
:10F01800FCEEC07A96ED070A17EE903A20EE280A21
:10F02800ADF80C3003F0EEFCFCEEC07A0C2017EEC5
:10F03800903A02A9ADF80E30FAF744FAD4ED077AFF
:10F04800894BF5EE407AF1EE10FA60D1D3ED067AED
:10F05800B4EEE78AF1EE10FA04DDDA6883ED068A89
:10F068005A61E8E0F5EEC07AF1EE10FA40F3E38079
:10F0780093F8202042B1022A00F2DD805A6B83ED1A
:10F08800078AFA329A63D6E0D3ED037A38EE678AB4
:10F09800F7EE007AB4EEE78AF1EE10FAACBF012180
:10F0A8000021D3ED0A7A69B19FED717A27EE877A4C
:10F0B800DFED707AB4EEE77AF1EE10FA58BFF0EEB1
:10F0C800477A03E09FED6C7A67EE877AC3ED0A7A98
:10F0D8002369654A1B0311D58DF80810D378116B85
:10F0E8000B440B205A788DF80920DA7A8DF80A201B
:10F0F8005B7D8DF80B3002A9FAF7E4F90123226B46
:10F1080084F82030E37813440022DA7291E0B4EEF8
:10F11800E78AF1EE10FA48BF83ED078AA16B636BAB
:10F1280094ED067AD4ED076A591AC943C90F77EEE8
:10F13800667A59B9B7EE006AF4EEC67AF1EE10FABB
:10F1480079DDB4EEE68AF1EE10FA74DDD4ED056AE5
:10F15800454BB4EEE67AF1EE10FACCBF0126002654
:10F1680066B1D3ED097A9FED427A67EE877A9FED13
:10F17800427AC3ED097AD3ED0B7A0AE0B0EE007A51
:10F18800F4EEC77AF1EE10FA08DDD3ED0B7A9FEDB5
:10F19800387A67EE877AC3ED0B7A07E0D3ED097A00
:10F1A8009FED357A67EE877AC3ED097AD4ED097A4F
:10F1B800206BE27867EEA87A1044FCEEE77ACDED92
:10F1C800017A9DF804304370D4ED0B7A2769FCEE80
:10F1D800E77A3F03CDED017A9DF8042042750ED5FC
:10F1E80046EA41018DF808108DF80930C37A8DF888
:10F1F8000A300B2002A98DF80B20FAF763F994F86E
:10F208002020194B022A11D1D3ED0A7A9FED1B7ADF
:10F21800196B67EE877A002283F82020FCEEE77AE4
:10F22800DA7817EE903A0A44D37202E0022283F8A1
:10F238002020FCF74FF922790B4B0AB1104A00E065
:10F24800104ADA602544D4ED037AB5F9063000EEA9
:10F25800103AB8EEC00A80EE280A37EEC00A05B0A8
:10F26800BDEC028BF0BD00BF602600204C5D01089C
:10F27800EC51783F6F12833A0AD7833F00007A44F3
:10F288000000A0410000A0C12B4BF0B52B4D1E681B
:10F2980005F110002F78F3192C46597801F0040174
:10F2A800013501F0FF0219B18542F3D10020F0BD0C
:10F2B800224D631B022B0ADD1AB102EB82025200B7
:10F2C800D2B215F8013B303B1A44D2B2F1E7002123
:10F2D800AC420AD919B101EB81014900C9B215F84C
:10F2E800013B303B1944C9B2F2E72E2F16D1013445
:10F2F800042000232578771903EB83037F785B00CC
:10F308007F079BB244BF303D5B1900F1FF3044BF1B
:10F3180001349BB210F0FF00ECD100E00023084854
:10F328004143642000FB03130620B3FBF0F30548B8
:10F3380000FB0230F0BD00BF0C0100209C2600201D
:10F3480040420F008096980030B500231A461049B5
:10F358008C1894F83C40BCB12E2C06D1013298B1DF
:10F368008C180444002584F83C5011440A2491F870
:10F378003C106343A1F13004092C9CBF303B5B185F
:10F388000E2A03D80132E2E7184630BD002030BD0E
:10F39800602600200D4B0E491A680E4B92B213449A
:10F3A8005B000D4A1B68C3F3090310B513601368AB
:10F3B8009BB201335B1000229A4206D0074851F8ED
:10F3C800044B20F812400132F6E710BD505C0040B3
:10F3D800206200401E30002094230020B923002022
:10F3E800014B00221A607047902300202DE9F84352
:10F3F800664B674E1B68DFF8B881664A00254FF0F8
:10F40800C0099D7283F80990DD723560D8F8003024
:10F4180023F4EC4323F0700343F400739BB2C8F861
:10F428000030D8F8003023F4E04323F040039BB2C7
:10F4380048F2800483F010032343C8F8003033688F
:10F4480012FA83F35B0040271A681F6033689BB287
:10F4580003F1005303F540535B0028461A688022E5
:10F468001A60D8F8003023F4F8731B051B0D2343EA
:10F47800C8F80030484B93F82C10F7F7ADFDD8F8D2
:10F488000030464A464923F4804323F070039BB278
:10F4980083F440532343C8F80030136823F4EC4343
:10F4A80023F070039BB21360336811FA83F35B0097
:10F4B80003201968C3F8009013683A4923F4E0431D
:10F4C80023F040039BB283F02003234313601368A7
:10F4D80023F4804323F0700323439BB213605368E3
:10F4E80023F4EC4323F0700343F4C0639BB25360EE
:10F4F800336811FA83F35B0019684FF4807119605F
:10F50800536823F4804323F0700323439BB2536072
:10F51800536823F4E04323F040039BB283F02003B5
:10F5280023435360D8F80C301F4A23F4EC4323F0EC
:10F5380070039BB2C8F80C30336812FA83F35B008F
:10F5480039461A684FF488721A60F7F745FDD8F8FB
:10F558000C3023F4804323F070039BB283F44053B0
:10F568002343C8F80C30D8F80C3023F4E04323F0D8
:10F5780040031C43A4B2C8F80C402846FCF7FFFF20
:10F588000A4B01221A60BDE8F88300BF98230020C7
:10F59800505C004004300020CC000020045C004097
:10F5A80008300020103000201C300020F8260020F1
:10F5B800005C0040134A144B50681B68181810B5BB
:10F5C800146808D011490822FCF7C5FF20461049E5
:10F5D8000422FCF7C0FF0F4B1A68002393720E4AEF
:10F5E800012111600D4913604FF4E0500B60106069
:10F5F8000B480B604FF4364101801160094A1360D3
:10F6080010BD00BFB0F7FF1FACF7FF1FB20000200E
:10F61800C200002098230020405C0040445C004069
:10F62800AC260020F8260020024B4FF480221A60F6
:10F63800704700BF14040140014B33F811007047B4
:10F64800341B002000207047104B1B6803EB40025E
:10F65800117E11B1022910D00BE0022805D9032828
:10F6680007D10B4A1268D20401D5D8897047988A05
:10F678007047084B33F810007047507E00EB80004D
:10F6880000EB800000F2EE2080B27047B026002028
:10F6980070260020101B002008B5FCF781FC054BE4
:10F6A80002221A72044A586012685A61012283F8C9
:10F6B8002D2008BDB02600209426002008B5FCF7B0
:10F6C8006FFC064B02221A725A6900F5B71000F552
:10F6D800587002F2DC5258605A6108BDB02600200A
:10F6E800044B1B6842F201021A420CBF01200020A1
:10F6F800704700BF70260020104B93F83020012A75
:10F7080010B51C460ED008D3022A0FD10C4A938A92
:10F718009BB283F48053938208E0094B4FF48052E4
:10F728009A6103E0064B4FF480521A85FCF738FCC7
:10F7380000F5F42000F59070606310BDB02600203D
:10F748000004004808B5044B1B7803F00503052B9B
:10F7580001D1FCF7D7FDFEE7E8260020D0400B1CBE
:10F768001141203A03D49C46134118436346524240
:10F7780093401843704700BF7BB972B90029BEBFD8
:10F7880000204FF0004106E008BF00281CBF6FF0C2
:10F7980000414FF0FF3000F073B882B0EC462DE91D
:10F7A800005000F03DF8DDF804E002B00CBC7047F2
:10F7B80007EE900AF5EEC07AF1EE10FA01D400F0E7
:10F7C80009B808B580F0004000F004F8404261EB49
:10F7D800410108BDD0B500F0B9F900220E4B06462C
:10F7E8000F4600F007FA00F017FC044600F08CF909
:10F7F80000220A4B00F0FEF902460B463046394615
:10F8080000F044F800F008FC2346002242EA000217
:10F8180010461946D0BD00BF0000F03D0000F04181
:10F828002DE9F041069C154606460F46984600F01D
:10F8380013FC05FB01F300FB0838A5FB0023B21AF3
:10F84800434467EB0303C4E90023BDE8F08100BF2C
:10F858002DE9F041069C904606460F461D4600F0ED
:10F8680049FD00FB05F5A0FB082308FB0155B21A6A
:10F878002B4467EB0303C4E90023BDE8F08100BF14
:10F88800704700BF81F0004102E000BF83F00043F1
:10F8980030B54FEA41044FEA430594EA050F08BF23
:10F8A80090EA020F1FBF54EA000C55EA020C7FEAE7
:10F8B800645C7FEA655C00F0E2804FEA5454D4EB64
:10F8C8005555B8BF6D420CDD2C4480EA020281EA2E
:10F8D800030382EA000083EA010180EA020281EA66
:10F8E8000303362D88BF30BD11F0004F4FEA0131B8
:10F8F8004FF4801C4CEA113102D0404261EB4101C7
:10F9080013F0004F4FEA03334CEA133302D052424C
:10F9180063EB430394EA050F00F0A780A4F1010408
:10F92800D5F1200E0DDB02FA0EFC22FA05F2801842
:10F9380041F1000103FA0EF2801843FA05F3594128
:10F948000EE0A5F120050EF1200E012A03FA0EFCA7
:10F9580028BF4CF0020C43FA05F3C01851EBE371D1
:10F9680001F0004507D54FF0000EDCF1000C7EEBEE
:10F9780000006EEB0101B1F5801F1BD3B1F5001F2C
:10F988000CD349085FEA30004FEA3C0C04F101044B
:10F998004FEA445212F5800F80F09A80BCF1004F74
:10F9A80008BF5FEA500C50F1000041EB045141EAF6
:10F9B800050130BD5FEA4C0C404141EB010111F4F7
:10F9C800801FA4F10104E9D191F0000F04BF0146A2
:10F9D8000020B1FA81F308BF2033A3F10B03B3F180
:10F9E80020020CDA0C3208DD02F1140CC2F10C0210
:10F9F80001FA0CF021FA02F10CE002F11402D8BF6E
:10FA0800C2F1200C01FA02F120FA0CFCDCBF41EA39
:10FA18000C019040E41AA2BF01EB0451294330BD08
:10FA28006FEA04041F3C1CDA0C340EDC04F11404E5
:10FA3800C4F1200220FA04F001FA02F340EA0300BC
:10FA480021FA04F345EA030130BDC4F10C04C4F102
:10FA5800200220FA02F001FA04F340EA03002946E2
:10FA680030BD21FA04F0294630BD94F0000F83F42C
:10FA7800801306BF81F480110134013D4EE77FEA0F
:10FA8800645C18BF7FEA655C29D094EA050F08BF5B
:10FA980090EA020F05D054EA000C04BF194610463C
:10FAA80030BD91EA030F1EBF0021002030BD5FEA80
:10FAB800545C05D14000494128BF41F0004130BDA8
:10FAC80014F580043CBF01F5801130BD01F00045FC
:10FAD80045F0FE4141F470014FF0000030BD7FEA6F
:10FAE800645C1ABF194610467FEA655C1CBF0B466A
:10FAF800024650EA013406BF52EA033591EA030F81
:10FB080041F4002130BD00BF90F0000F04BF002178
:10FB1800704730B54FF4806404F132044FF00005AB
:10FB28004FF0000150E700BF90F0000F04BF002124
:10FB3800704730B54FF4806404F1320410F000458A
:10FB480048BF40424FF000013EE700BF42004FEA85
:10FB5800E2014FEA31014FEA02701FBF12F07F4302
:10FB680093F07F4F81F06051704792F0000F14BFFF
:10FB780093F07F4F704730B54FF4607401F0004543
:10FB880021F0004120E700BF50EA010208BF70479A
:10FB980030B54FF000050AE050EA010208BF70478F
:10FBA80030B511F0004502D5404261EB41014FF4F8
:10FBB800806404F132045FEA915C3FF4DCAE4FF0FC
:10FBC80003025FEADC0C18BF03325FEADC0C18BFE3
:10FBD800033202EBDC02C2F1200300FA03FC20FA34
:10FBE80002F001FA03FE40EA0E0021FA02F1144481
:10FBF800C1E600BF70B54FF0FF0C4CF4E06C1CEA96
:10FC080011541DBF1CEA135594EA0C0F95EA0C0F0A
:10FC180000F0DEF82C4481EA030621EA4C5123EA7D
:10FC28004C5350EA013518BF52EA033541F48011AC
:10FC380043F4801338D0A0FB02CE4FF00005E1FB5F
:10FC480002E506F00042E0FB03E54FF00006E1FBA9
:10FC580003569CF0000F18BF4EF0010EA4F1FF04EC
:10FC6800B6F5007F64F5407404D25FEA4E0E6D412C
:10FC780046EB060642EAC62141EA55514FEAC5203D
:10FC880040EA5E504FEACE2EB4F1FD0C88BFBCF5B9
:10FC9800E06F1ED8BEF1004F08BF5FEA500E50F16A
:10FCA800000041EB045170BD06F0004646EA010130
:10FCB80040EA020081EA0301B4EB5C04C2BFD4EB62
:10FCC8000C0541EA045170BD41F480114FF0000E5B
:10FCD800013C00F3AB8014F1360FDEBF002001F0C9
:10FCE800004170BDC4F10004203C35DA0C341BDC43
:10FCF80004F11404C4F1200500FA05F320FA04F015
:10FD080001FA05F240EA020001F0004221F0004148
:10FD180010EBD37021FA04F642EB06015EEA430EBB
:10FD280008BF20EAD37070BDC4F10C04C4F12005EB
:10FD380000FA04F320FA05F001FA04F240EA02009E
:10FD480001F0004110EBD37041F100015EEA430E6F
:10FD580008BF20EAD37070BDC4F1200500FA05F28F
:10FD68004EEA020E20FA04F301FA05F243EA02030E
:10FD780021FA04F001F0004121FA04F220EA02001D
:10FD880000EBD3705EEA430E08BF20EAD37070BD63
:10FD980094F0000F0FD101F00046400041EB010143
:10FDA80011F4801F08BF013CF7D041EA060195F025
:10FDB800000F18BF704703F00046520043EB0303DF
:10FDC80013F4801F08BF013DF7D043EA06037047CC
:10FDD80094EA0C0F0CEA135518BF95EA0C0F0CD0D7
:10FDE80050EA410618BF52EA4306D1D181EA03011D
:10FDF80001F000414FF0000070BD50EA410606BF17
:10FE08001046194652EA430619D094EA0C0F02D15B
:10FE180050EA013613D195EA0C0F05D152EA0336A0
:10FE28001CBF104619460AD181EA030101F00041BE
:10FE380041F0FE4141F470014FF0000070BD41F007
:10FE4800FE4141F4780170BD70B54FF0FF0C4CF4E1
:10FE5800E06C1CEA11541DBF1CEA135594EA0C0F00
:10FE680095EA0C0F00F0A7F8A4EB050481EA030E4D
:10FE780052EA03354FEA013100F088804FEA033334
:10FE88004FF0805545EA131343EA12634FEA022202
:10FE980045EA111545EA10654FEA00260EF00041C3
:10FEA8009D4208BF964244F1FD0404F5407402D215
:10FEB8005B084FEA3202B61A65EB03055B084FEAA6
:10FEC80032024FF480104FF4002CB6EB020E75EBA3
:10FED800030E22BFB61A754640EA0C005B084FEACB
:10FEE8003202B6EB020E75EB030E22BFB61A754648
:10FEF80040EA5C005B084FEA3202B6EB020E75EB93
:10FF0800030E22BFB61A754640EA9C005B084FEA0A
:10FF18003202B6EB020E75EB030E22BFB61A754617
:10FF280040EADC0055EA060E18D04FEA051545EA06
:10FF380016754FEA06164FEAC30343EA52734FEAAF
:10FF4800C2025FEA1C1CC0D111F4801F0BD141EA28
:10FF580000014FF000004FF0004CB6E711F4801F8D
:10FF680004BF01430020B4F1FD0C88BFBCF5E06F6D
:10FF78003FF6AFAEB5EB030C04BFB6EB020C5FEA7D
:10FF8800500C50F1000041EB045170BD0EF0004ED2
:10FF98004EEA113114EB5C04C2BFD4EB0C0541EA04
:10FFA800045170BD41F480114FF0000E013C90E601
:10FFB80045EA060E8DE60CEA135594EA0C0F08BFC5
:10FFC80095EA0C0F3FF43BAF94EA0C0F0AD150EAC4
:10FFD80001347FF434AF95EA0C0F7FF425AF104657
:10FFE80019462CE795EA0C0F06D152EA03353FF47F
:08FFF800FDAE1046194622E798
:020000040801F1
:1000000050EA410618BF52EA43067FF4C5AE50EAF3
:1000100041047FF40DAF52EA43057FF4EBAE12E7E3
:100020004A0011D212F5001211D20DD56FF4787377
:10003000B3EB62520ED44FEAC12343F0004343EACC
:10004000505323FA02F070474FF00000704750EA17
:10005000013002D14FF0FF3070474FF00000704781
:1000600000292DE9F043C0F2A6800026002BC0F243
:100070009C80884694469E46154604460F46002BB3
:100080003DD18A4259D9B2FA82F33BB1C3F1200281
:100090009F4020FA02F29D4017439C40290C220CFD
:1000A000B7FBF1FEA8B201FB1E7742EA074700FB4F
:1000B0000EF3BB420AD97F190EF1FF3280F00581A1
:1000C000BB4240F20281AEF1020E2F44FF1AA4B2ED
:1000D000B7FBF1F301FB137744EA074700FB03F09A
:1000E000B84208D97F1903F1FF3280F0F080B8429E
:1000F00040F2ED80023B43EA0E43002203E08B42D4
:100100000FD900221346341C18BF012460424FF05F
:10011000000565EB45015840514000196941BDE8B3
:10012000F083B3FA83F2002A40F086808B4202D338
:10013000844500F2DB800123E5E712B90123B3FB1C
:10014000F2F5B5FA85F000283BD1781B4FEA154E41
:100150001FFA85FC0122B0FBFEF8210C0EFB1807EC
:1001600041EA07470CFB08F3BB4207D97F1908F1A6
:10017000FF3102D2BB4200F2BD808846FF1AA4B212
:10018000B7FBFEF30EFB137744EA07470CFB03FCB7
:10019000BC4507D97F1903F1FF3102D2BC4500F2FB
:1001A000A7800B4643EA0843ADE752426FEA0606D2
:1001B00063EB43035DE7404261EB41014FF0FF36E3
:1001C00054E7C0F1200224FA02F107FA00F3854057
:1001D0004FEA154ED7401943B7FBFEF20B0C0EFB4E
:1001E00012771FFA85FC43EA07430CFB02F79F4294
:1001F00004FA00F407D95B1902F1FF3074D29F4270
:1002000072D9023A2B44DF1B89B2B7FBFEF80EFB12
:10021000187341EA03430CFB08F79F4208D95B19A6
:1002200008F1FF315CD29F425AD9A8F102082B4451
:10023000D81B48EA02428EE7C2F120032CFA03F1F0
:100240000EFA02FE20FA03F741EA0E0E08FA02F057
:1002500028FA03F14FEA1E453843B1FBF5F8030CC9
:1002600005FB18111FFA8EF743EA014107FB08F35B
:100270008B420CFA02FC09D911EB0E0108F1FF398F
:1002800030D28B422ED9A8F102087144C91A80B22B
:10029000B1FBF5F305FB131140EA014107FB03F73E
:1002A0008F4208D911EB0E0103F1FF3016D28F42B5
:1002B00014D9023B714443EA0843C91BA3FB0C89D0
:1002C000494509D305D000221DE79646FEE61346B0
:1002D00011E794404445F6D2013BF4E70346EAE7D0
:1002E0008846A5E7C846D1E702468CE713460AE7E9
:1002F000023B57E7A8F102082F443FE72DE9F04100
:10030000002B44D18A42154604464FD9B2FA82F7EF
:100310000E464FB1C7F12003B94020FA03F602FAA6
:1003200007F50E4300FA07F44FEA154E230CB6FB0F
:10033000FEF0AFB20EFB106143EA014307FB00F190
:10034000994209D95B1900F1FF3280F0EC809942A3
:1003500040F2E98002382B445A1AA4B2B2FBFEF3F1
:100360000EFB132244EA024207FB03F7974208D927
:10037000521903F1FF3180F0D880974240F2D580C6
:10038000023B43EA004000263146BDE8F0818B4243
:1003900047D8B3FA83F6002E48D18B4202D382426B
:1003A00000F2CD8001203146BDE8F08112B901256F
:1003B000B5FBF2F5B5FA85F8B8F1000F77D14A1B15
:1003C0004FEA154EAFB20126B2FBFEF0230C0EFB36
:1003D000102143EA014107FB00F38B4207D9491979
:1003E00000F1FF3202D28B4200F2BA801046C91AE5
:1003F000A4B2B1FBFEF30EFB131144EA014407FB68
:1004000003F7A74208D9641903F1FF3280F08F8007
:10041000A74240F28C80023B43EA00403146BDE8EF
:10042000F081002630463146BDE8F081C6F1200457
:1004300022FA04F5B3402B4320FA04FC01FA06F734
:1004400021FA04F54FEA134E4CEA0707B5FBFEF814
:10045000390C0EFB18551FFA83FC41EA05450CFBCD
:1004600008F1A94202FA06F204D9ED1808F1FF34A6
:1004700067D3A0466D1ABFB2B5FBFEF40EFB145550
:1004800047EA05410CFB04FC8C4504D9C91804F16A
:10049000FF355CD32C4644EA0844CCEB0101A4FBB5
:1004A0000223994248D344D0204600266CE7C8F185
:1004B000200401FA08F305FA08F520FA04F7E140F0
:1004C0004FEA154E1F43B1FBFEF63A0C0EFB161118
:1004D0001FFA85FC42EA01430CFB06F29A4200FA3D
:1004E00008F407D95B1906F1FF3137D29A4235D9A2
:1004F000023E2B449B1ABFB2B3FBFEF00EFB10333F
:1005000047EA03430CFB00F1994207D95B1900F15C
:10051000FF3221D299421FD902382B445A1A40EA9D
:100520000646674650E7104616E70B4629E713468E
:1005300072E7B0409042B7D2601E002624E73046F2
:1005400022E7A94295D9A8F102081D4492E78C45FB
:10055000A0D9023C19449EE71046DFE70E46C9E7E2
:100560000238294443E700BF4FEA4102B2F1E043B9
:1005700024BFB3F5001CDCF1FE5C0DD901F0004C8A
:100580004FEAC0024CEA5070B2F1004F40EB8300DA
:1005900008BF20F00100704711F0804F21D113F106
:1005A0003872BCBF01F00040704741F480114FEA3F
:1005B0005252C2F11802C2F1200C10FA0CF320FAC8
:1005C00002F018BF40F001004FEAC1234FEAD323E5
:1005D00003FA0CFC40EA0C0023FA02F34FEA43034F
:1005E000CCE77FEA625307D150EA01331EBF4FF0D8
:1005F000FE4040F44000704701F0004040F0FE40F3
:1006000040F40000704700BF1148124902680060C2
:100610008A4218D0002103E00F4B5B58435004314D
:100620000E480F4B42189A42F6D30E4A02E00023BE
:1006300042F8043B0C4B9A42F9D3FDF7BBFE00F0A5
:1006400019F87047FEE70948D0F800D04068004725
:10065000FC9F0020EFBEADDE087D010800000020F9
:1006600078010020780100201C27002000D8FF1FFF
:10067000FEE700002DE9804897B0EFF785FDAC4C10
:10068000DFF810932378D9F8005033B1A94B1B68D9
:10069000EB1A002BA4BF00232370FFF725F810B13D
:1006A000A54B00221A70A54B19680F0740F18281F3
:1006B000A34B1B681B7A062B00F27081DFE813F056
:1006C000070007003200CC000501300130019D4BCE
:1006D0001A78002A00F0628100221A709A4B1F7863
:1006E0009A4B1B6893F800E0994B93F800C00222E4
:1006F000984EB35C3B4103F00F03734502F10108D0
:100700000CD20B2B9FBFB05C16F8086000EA0C00FF
:1007100006EB00209CBF904E46F823000232102AC0
:10072000E6D102E18D4B1A78002A00F037810022D1
:100730001A708B4B8B4A93F802E0DF7858780EF0F2
:10074000070640EA062007F03F06760146EADE0685
:100750001060187956605E7993F806E0800040EAF0
:10076000971006F0010740EA87209060DF790EF0CD
:100770000F00C00140EA560007F07F06D060360146
:10078000187A46EA1E1693F809E0166140000EF04A
:10079000030640EAD71040EA46209F7A5061D87A93
:1007A00007F01F06B601C00046EA9E0640EA571051
:1007B00093F80DE09F7BD061187B96610EF00706E1
:1007C00040EA062007F03F06760146EADE061062A0
:1007D000D87B56621E7C93F811E0800040EA9710A7
:1007E00006F0010740EA872090629F7C0EF00F0020
:1007F000C00140EA560007F07F06360146EA1E16A1
:10080000D062D87C166393F814E0400040EAD71019
:100810000EF003065F7D40EA4620506307F01F0696
:10082000987DDB7DB60146EA9E06C00040EA57107F
:100830009663DE07D0634CBF40F21470AD201064A5
:1008400098074CBF40F21470AD2013F0080F5064AD
:1008500014BF03230123A2E0434A1378002B00F0C6
:100860009D8000231370414A414F1678414807EBA1
:10087000460EB0F800C09EF803809EF8040040EADF
:100880000820844540F08A807878012804D08128A7
:1008900040F08580032300E00346102E84BF102023
:1008A0001070354817780022D6B2BE4200F102001F
:1008B00075D210F802EC10F8016C46EA0E26DFF84B
:1008C000D8E02EF812600132EEE72C4B1A78002A9D
:1008D00064D000221A702A4B1A78A82A1E465DD1CD
:1008E000DA7C002A5AD106EB42009FED267AC778BF
:1008F000037903EB072307EE903AF8EEE77A224BF1
:10090000C7EE877A9FED217A77EEC77AFCEEE77A19
:1009100017EE900A43F822000132082AE3D104E0DE
:100920001B4B1A78D2B300221A70012337E000BFA4
:100930004F0A002078010020500A00207026002075
:10094000B0260020711B00209A240020942400204F
:100950009B240020611B0020581A0020E21B00206D
:10096000C91B0020C81A0020991B00209C1B0020D6
:100970009D1B00209A1B0020A01B0020921B002022
:100980007D1B0020CDCCCC40881A00200080BB43CA
:10099000541A0020F0260020A81A00200023DA07AD
:1009A00041BF83F002039E4A0120C3F3400344BFCA
:1009B000107023704B0406D59A4A13780BB10020AF
:1009C0001070974A137044F208030B403BB1944BEC
:1009D0001B7823B105F5C333934AA0331360CF07C7
:1009E0000CD5914B5A79187982421FBF012222708F
:1009F00005F5C332A0321CBF1A6058718E0409D5A8
:100A000000238A4A32F81320002A40F07C81013307
:100A10000C2BF6D1824B844C1B7823B9844B1B687A
:100A2000ED1A002D04DBF0F7D5FC0123A3711DE1C5
:100A3000A368013303EAE3730D06A36040F1168156
:100A40007C4D2B682E46A3B9237B013B042B00F27F
:100A50000D81DFE813F0140014001400FB00C70040
:100A6000744B1868FBF7ECFAFAF7CBF808B1FCF70F
:100A7000BBFA3068FBF7E7FA0028F1D1E4E7E26A55
:100A8000694E177817B1012F10D0EFE0012B00F25B
:100A9000ED80727B684B28680C2101FB02335A7889
:100AA000664B53F82210FBF7C8FA5CE02868DFF8C1
:100AB0008481FBF7BFFA002800F0D880337B022B3B
:100AC0003FD0032B4CD0012B40F0D0805C4B1968F9
:100AD000736ACB1AC72B40F2C980336A042B2ED815
:100AE000554AD8F8005071620C2000FB0323A86817
:100AF0005F7896460023514A52F823608642D9B265
:100B000004D00133082BF6D1002300E00B46BB4292
:100B100005D0284652F82710FBF78FFAA6E0627B33
:100B20000C2303FB02E35E6816F8011B19B128468B
:100B3000FBF78CFAF8E7236A0133236296E0022080
:100B400092E0727B3C4BD8F800000C2101FB023391
:100B50005A783A4B53F82210FBF76FFA032083E0E0
:100B6000F36A9B780BB904207EE096F828300BB925
:100B700086F8287094F828302B4E012B12D1336A56
:100B8000B22B0AD82C4A2868134493F83C10FBF780
:100B90005DFA336A0133336204E0002333620223D7
:100BA00086F8283094F828301F4E022B15D1326A6F
:100BB0000F2A0FD8F36A20495B78286803EB0313E8
:100BC0000B44134493F8F010FBF740FA336A0133F7
:100BD000336202E0032386F8283094F82830022B91
:100BE00044D9C0E76369104901336361E36ADB7884
:100BF0004BB14B7B0133DBB20522B3FBF2F202EBCC
:100C000082029B1A4B730E4B1B68A3610D4B002293
:100C10001A700D4A137823F002031370012023E0A9
:100C2000500A0020C610002078010020341B00204C
:100C3000240A0020C81C0020743E01088C5C0108B6
:100C400094260020E6180020E01800208A4BA269B4
:100C50001B689B1A40F6C412934207D9874A13684F
:100C600023F0200313600520FAF7BCFA844DFBF74C
:100C70009BF9EB7BC9F80000266B6BB1814B0FA889
:100C8000DB6898479DF83C30002B44D17E4B1868B8
:100C9000801B64283FD526E0AB89002B3BD0801B0E
:100CA000002838DA1FE09AF80430002B01F0348273
:100CB00061890020F2F79AF801263B689A0601F153
:100CC0006682B9F1050F01F062823B68DB0201F137
:100CD0006B8298F8E0360BB1FBF7C6FA6B4B1B78CA
:100CE000002B01F06F82694B1B78002B7FF4C7AC9F
:100CF000674B1B685B057FF5C2AC614BB3F85201D3
:100D0000F4F75CFBBBE401232370624A05F5C333AF
:100D1000A03313607EE6604AD9F8003012685F485D
:100D20005C4EDFF87881134423635D4B1F68554B9D
:100D30005B689847002800F0C6804046414696F818
:100D40003420F6F737FC574B1B88002B74D0B36B5D
:100D50001B7808EE103A06F13C0A4FF0000B4836BB
:100D6000504B38F91B001988B1F57A7F02BF002378
:100D7000CAF800303361DAF800300344CAF80030B2
:100D8000336907EE900A0133012B4FEA4B02F8EE6C
:100D9000E77A336106D10023C6ED017AC6ED007A09
:100DA000B3601BE0D6ED006A07EE103A37EEE66A54
:100DB000B8EEC77A86EE077A36EE877AD6ED026A03
:100DC00086ED017A77EEC77A86ED007AE6EE276A3D
:100DD000F0EE667AC6ED036AC6ED026A3248002379
:100DE000012928F8023013522E4930D13369079176
:100DF000012BC3BF03F1FF3300EE103AD6ED037AA7
:100E00009FED2A0A0690C8BFB8EEC00A0592C8BF77
:100E100087EE800A01F0B8FE059A0698079918EE49
:100E2000103A5BB1F8EEC87AB4EEE70AF1EE10FAC8
:100E300004DD4FF47A730B80002339E0DAF80030D8
:100E40004FF47A7E03F5FA7393FBFEF383520BF1B2
:100E5000010BBBF1030F0AF1040A06F114067FF43B
:100E60007FAF0888012803D10591F5F76FFD05993B
:100E70000B88013BDFE700BF94260020DC18002030
:100E8000B41100205C1D0020F02600201127002056
:100E9000702600207801002058260020FC10002039
:100EA0001411002008270020FC0100200000000091
:100EB000C64938F8132031F81310521A28F81320B5
:100EC0000133032BF4D1C24B1B6813F0020300F073
:100ED000D082C04EC04B06F18A005B68984700285C
:100EE00000F0E580BD4B06F18A001A780146F6F75E
:100EF00061FBBB4B1B88002B43D0D6F8900000232E
:100F0000B74AB8491288DFF8CCC2B2F5C87F04BF2F
:100F1000002241F823204FEA830E0CF18A0651F893
:100F20000E2036F91380424441F80E20002126F8A5
:100F3000131020F813100133032BE1D1A84E33888E
:100F4000012B1BD1DCF894304FF4C87EC83393FBDF
:100F5000FEF30380DCF89820C83292FBFEF2428058
:100F6000DCF89C30C83393FBFEF3A3F580738380D9
:100F7000A7F85810A7F85A10F7F766FA3388013B1C
:100F80003380994B1B6858077DD5984B1B88322BB3
:100F900013D1D4F890301A88A4F8A0205A889B88DE
:100FA000A4F8A430B7F85830A4F8A630B7F85A30EF
:100FB000A4F8A220A4F8A83001E0002B44D0D4F873
:100FC00090E00023894A834E1288322A884A04BF5F
:100FD000002142F823104FEA830C06F18A0052F8F0
:100FE0000C1030F91380414442F80C10002220F814
:100FF00013202EF813200133032B1146E2D1DFF822
:10100000EC81B8F80030012B19D17A4A11707A4A74
:101010000C201370F5F79AFCD6F89030B6F8A020A3
:101020001A80B6F8A2205A80B6F8A4209A80B6F8A2
:10103000A630A7F85830B6F8A830A7F85A30B8F854
:101040000030013BA8F800306C4B1A78DAB1D4F8C4
:101050009010002232201A70D4F8AC3093FBF0F3D9
:101060000B80D4F8B03093FBF0F34B80D4F8B4305D
:1010700093FBF0F3A3F580738B80A7F85820A7F8B3
:101080005A20F7F7E1F9D4F89020B4F88A301188A3
:101090005B1AA4F88A305188B4F88C305B1AA4F833
:1010A0008C309288B4F88E309B1AA4F88E30FAF700
:1010B0007BFFD4F8B83094ED2F6AD4F8C070C4F830
:1010C000B800C3EB000A07EE90AAB8EE678A0026C4
:1010D00028EE066A97F800C049484A490DF1240EE7
:1010E0003246494B33F9123007EE903AF8EEE77A80
:1010F000464B67EE867AEEEC017ABCF1000F1CD00D
:1011000007EE90CAF8EEE76AB7EE007AC7EE266AF5
:1011100033F9123007EE903AF8EEE77A37EE667A56
:1011200067EEA67AD1ED006AE6EE877AC1ED007A25
:10113000FDEEE77A17EE903A01E033F81230438083
:1011400030F8023F0132032A13FB036601F1040168
:10115000C7D164232E4809A95E43F6F785FE4FF4F4
:10116000803396FBF3F6493EB6B23B2ED7ED016ACB
:1011700011D9B4F9DC30D4ED360A07EE903AF8EE26
:10118000E77A244BF4EEE70AF1EE10FA46DD1A781E
:1011900042F0080245E0F7EE007A36EEA77A1C4AE4
:1011A00087EE877A00231C4931F913100133032B92
:1011B00007EE901A92ED006AF8EEE77AE6EE267AEC
:1011C00067EE877AE2EC017AEDD1D2E7FC010020EC
:1011D000DC180020780100206C2300200E2700205E
:1011E000CA0A00200C02002070260020CC0A002031
:1011F00024020020CE0A0020C70A0020C80A0020CE
:10120000A01100203C020020FC100020020200205F
:1012100048020020E0180020A21100201A7822F0D5
:10122000080294ED350A1A7001F0ACFCDFF8CC83AB
:10123000D4ED357A88ED000A94ED360AD4ED348A7F
:10124000DC4E20EE000AF1EE688AA7EEA70A01F054
:101250009BFCF0EE400AB0EE680A01F093FCDFED73
:10126000D68A88ED010A98ED000A20EE280A01F0DE
:1012700087FB98ED010A308020EE280A01F080FB00
:10128000CE4B70801B68190721D5CD4809A9F6F708
:10129000EBFDD7ED026ACA4AF7EE007A36EEA77A7E
:1012A000002387EE877AC74931F913100133032BE6
:1012B00007EE901A92ED006AF8EEE77AE6EE267AEB
:1012C00067EE877AE2EC017AEDD1BD482AE0BE4EA6
:1012D00009A93046F6F7C8FD96ED010A96ED007AA9
:1012E000D6ED027A20EE000AA7EE070AA7EEA70ABB
:1012F00001F04AFCB5EE400AF1EE10FA11D0D6ED3D
:10130000007AC7EE807AC6ED007AD6ED017AC7EE94
:10131000807AC6ED017AD6ED027A87EE800A86EDF4
:10132000020AA948FBF774F8DFEDA87AA84B9FEDF5
:10133000A97A188068EE278AD8ED007AA44BF1EEDE
:10134000677ACDED0C7AD8ED017AB3F90030F1EE81
:10135000677ACDED0D7A07EE903A9F4BF8EEE77A7B
:10136000B3F9002067EEC77A0FA8CDED0E7A07EE2D
:10137000902AB3F90220B3F90430F8EEE77A0CA909
:10138000CDED0F7A07EE902AF8EEE77ACDED107AE0
:1013900007EE903AF8EEE77ACDED117AF6F764FDB4
:1013A0007B789DED117A012B1DD18C4B1B785A0750
:1013B0000FD4D4F8EC30402293FBF2F29B1A07EEE4
:1013C000903AF8EEE77A77EE877AFDEEE77AC4EDA9
:1013D0003B7AD4F8EC30402293FBF2F307EE903ADC
:1013E000F8EEE77A01E0DFED7E7A94ED3C8A9DED40
:1013F0000F0A37EE677AD4ED3D7A8DED117A78EEEB
:10140000A77A9DED117AC8EEA77A37EE487AA7EE53
:10141000878A84ED3C8A01F0B3FAD4F8F860317819
:10142000F6F74AFCD4F8FC309DED100A1844C4F8D5
:10143000FC0001F0A5FA3178F6F73EFCD4F8003153
:10144000B0EE480A1844C4F8000101F099FA717826
:10145000F6F732FCD4F80431624A18441368C4F831
:10146000040153441360D4F808310133C4F808313F
:1014700005E0A4F88A30A4F88C30A4F88E30FAF78E
:1014800093FDD4F80C31584FDFF874A19FED4F7ADB
:10149000C9F80000C31A9BB207EE903AAAF80030D0
:1014A000F8EE677A3B68DFF85C9193F852304F4A68
:1014B000C4F80C0167EE877ABB46C9ED007A23B900
:1014C0002B7C002B00F0C5802FE0D2ED447AF5EEA6
:1014D000407AF1EE10FA0AD1454B1B68059307EEEE
:1014E000903AF8EE677A67EE877AC2ED447A002682
:1014F000DFF814813F4838F91630D4ED440A00EE85
:10150000103ADBF8003000EBC60093F85210B8EE4A
:10151000C00AF6F793F9FDEEC07A17EE903A28F874
:1015200016300136032EE3D1CAE7BAF80030DFF8EF
:10153000BC80D9ED000AB4F82C6100EE103A08F531
:101540009870B8EE400A0121F6F778F9BCEEC00AAF
:10155000A3798DED050ABDF81400B6FBF0F0461C2A
:10156000B6B2A4F83861002B50D0B8F83AB10023D5
:101570001E49214A01F5A27C01F59E7932F81380BB
:101580003CF813E039F813202CF81380CEEB080E4A
:1015900012FB0BF20FFA86FA92FBFAF2724429F868
:1015A00013200133042BE3D100238B71A1F83A01FE
:1015B00031E000BF662600204C3D0F44DC180020BF
:1015C000580200209211002000000020BD3786350F
:1015D000A811002035FA8E3CA2110020102700200F
:1015E00000008043EC260020141100207801002028
:1015F000582600208C020020101B00205C220020B6
:10160000D0100020E81F0020FC100020B8F83A316C
:10161000013BA8F83A31B4F83A01B54A03B2002BBD
:101620004FF0000313DDB2F93861B24931F81320ED
:10163000083112FB00F231F8131092FBF6F28A1A0D
:10164000AD4921F813200133042BEED101E0A2F8BB
:101650003A31F1F72DFDA94BDFF804831B68A84E42
:1016600013F4801300F0978033881B0600F1E080AC
:10167000A44B1B7803F0040303F0FF0A002B75D082
:10168000A14AA24B117811B194F84C1139B1A0497B
:101690000020086001211973002184F84C111B7B84
:1016A000D8F800901370032B05D14846994954226D
:1016B00000F04CFF53E0012B06D1542295484946D7
:1016C00000F044FF002202E0022B02D10122924BE3
:1016D0001A70924A01231370914A1370914A0023A1
:1016E0001360914A1360914BC3F80090904B99F8A6
:1016F00000201A70884B8F4A1B78D05C8E4B8F4A23
:101700001870834B48441A6042788D4B07EE902A3C
:10171000F8EEE77AB2EE047AC7EE877AC27A9FEDE6
:10172000897AC3ED007A07EE902AF8EEE77A427DD7
:10173000C7EE877A9FED847AC3ED017A07EE902A8F
:10174000F8EEE77A67EE877AC3ED027AFCEEE77A85
:1017500017EE903A43750023C372F9F779FE8020A3
:10176000F6F7D0FB012384F8A43161E0DFF8A09103
:10177000D9ED007AF5EE407AF1EE10FA58D0F6F78E
:1017800063FE0023C9F800305F4B83F800A05F4B75
:1017900001221A734CE0328810063ED55A4A10785E
:1017A000411E012959492DD8DFF894E15F4BDEED48
:1017B000017A9FED647A1A685F4B67EE877A187832
:1017C0009FED627AFCEEE77A104417EE903AC3720E
:1017D000DEED027A67EE877AFCEEE77A17EE903A52
:1017E0004375537807EE903AF8EEE77A77EEA77AEA
:1017F000FCEEE77A17EE903AD370D37A5373537DA9
:10180000D37504E0032802D11370012301E00B7BA0
:10181000013380200B73F6F764FB3A4B1B785907B2
:1018200006D494F8A4311BB1314B012283F84C212A
:10183000474BDFF830911B78B3B12F4B454AB3F9D2
:101840000610B2F89A3199420EDC5379012B01D07F
:10185000192B02D192F8E82132B90E2B04D0082BB3
:101860001CBF0023A9F80430D8F8003093F8188181
:10187000B8F1000F7ED033889A077BD094ED350AFB
:10188000D4ED347A94ED368A20EE000AA7EEA70A4A
:10189000A8EE080A01F078F988EE000ADFED2E7A4A
:1018A000B4EEE70AF1EE10FA5ED901F00DF9104B33
:1018B000D3ED6A7A20EE270A01F062F8B0F5617F75
:1018C000A8BF4FF4617007EE900AB8EEE70ADFEDAB
:1018D000237A80EE270AF6F7FEF907EE908AF8EEF3
:1018E000E77A27EE800A01F04BF880B23DE000BFB6
:1018F00078010020B4020020101B0020DC10002022
:10190000A4190020102700206026002000000020DD
:101910006C260020C80200206126002064260020DA
:10192000802600207C26002078260020902600209B
:10193000622600204C5D0108632600200000A041C3
:101940008426002000007A445555553F9A99993FC6
:1019500010000020B41100208FC2753CEFB6B044D7
:1019600014110020AC1100200020B9F806301844F2
:10197000A9F80600C34B1B689B0640F19E80338884
:1019800003F03003002B00F09880BF4B1B78DE077C
:1019900040F19380BD4BDFEDBE7AB3F90030DFF844
:1019A00034B308EE103AB8EEC88A28EE278AB0EEB3
:1019B000480AF6F790F9F0EE408AB0EE480AF6F7DA
:1019C000EDF9B44B1B68D978B34BB0EE409AB2EE48
:1019D000048A00294DD0B14AB3F902E05688079134
:1019E00030B2C0EB0E0006920593F9F74DFC079953
:1019F000059B069AC1F1000A504503DB8842A8BF47
:101A0000084600E0504600EB06081688B3F90000CF
:101A1000059233B21FFA88F8C01AA2F80280069124
:101A2000F9F732FC5045059A04DB06998842A8BFB5
:101A3000084682465644B6B2168036B207EE106AA1
:101A40000FFA88F8B8EEC70A07EE908A28EEC07A37
:101A5000F8EEE77A20EE090AA7EE897AA7EEA80A3F
:101A600087EE087ABDEEC77A17EE103AABF8003071
:101A70001BE0B3F90220B3F9003000EE103A07EE94
:101A8000102AB8EEC00AB8EEC77A68EEC07A20EE27
:101A9000090AE7EE097AA7EE280AC7EE887AFDEE72
:101AA000E77A17EE903AABF8003080EE080AFDEEC8
:101AB000C07A17EE903AABF80230794B3868B5F837
:101AC0006E210093774B1E68774B196800F158031D
:101AD000B047764B764A1E78032E1AD9D4F8AC312B
:101AE000B3F802E0BEF5FA7F13D2B9F90400B2F9F7
:101AF000047080EAE07CACEBE07CCEF10001CCEB42
:101B000001039F4204DB0EEB0C03BB42A8BF3B4624
:101B100093805788B2F800E0B2F90480B9F8060063
:101B2000D4F8ACC1634A0021B14202F1100232D2B2
:101B30009CF9013052ED045ADFF884915B4208FBB6
:101B400003F307EE903A0FFA8EF306EE903A03B2E3
:101B500006EE103A3BB2B8EEE77A07EE903AF8EEAE
:101B6000E77AB8EEC66A67EEA57A52ED065AE6EE57
:101B7000257AF8EEE66A12ED056AE6EE867A52ED0F
:101B8000036AE7EE267AFDEEE77A17EE903A29F837
:101B900011300131C8E7484B1A7802F0040202F014
:101BA000FF03002A00F0A080444B454ADB780693EF
:101BB00013880121B1421FB207D232F91130BB4262
:101BC000B8BF3B469BB20131F4E73E4A3E4910683C
:101BD000B1F906E042883D49D4F870C2D1F80080DE
:101BE00037499742C8BF9A1A394B1B6803F4805B88
:101BF00003F0100AD4F8AC310593CCBF92B20022A6
